:020000040800F2
:10000000E8B200209D010008793E0108F9280108A6
:100010009D3B01089535000839D901080000000012
:10002000000000000000000000000000216C01083A
:100030002571000800000000714701085976010889
:10004000B7010008B7010008B7010008B7010008B0
:10005000B7010008B701000829710008B7010008BE
:10006000B70100083571000841710008B7010008A8
:10007000856B0008956B0008B7010008B701000800
:10008000B7010008B7010008B7010008B701000870
:1000900099350008A9350008B70100084D7100081E
:1000A0004D770108B7010008B7010008B701000843
:1000B000B7010008B7010008B7010008B701000840
:1000C000B7010008B7010008B7010008B701000830
:1000D000B70100084DA70108B7010008B7010008E3
:1000E000B7010008B7010008B7010008B701000810
:1000F000B7010008B7010008B7010008A56B0008A8
:10010000B7010008B7010008B7010008B7010008EF
:10011000B7010008B7010008B70100085D770108C2
:10012000B7010008B56B0008C56B0008D56B000867
:10013000B7010008B7010008B7010008B7010008BF
:10014000B9350008C9350008B7010008E93E0108C3
:10015000E56B0008F56B0008056C000869A701084D
:10016000B7010008B7010008B7010008B70100088F
:10017000B7010008B7010008B7010008000000003F
:10018000B7010008B7010008DFF80CD000F0C4FB8D
:100190000048004785DC0108E8B200200648804797
:1001A00006480047FEE7FEE7FEE7FEE7FEE7FEE75C
:1001B000FEE7FEE7FEE7FEE72D770108890100086C
:1001C0002DE9F05F0546002092469B46884606468C
:1001D000814640241BE0284641464746224600F01F
:1001E0002DFA53465A46C01A914110D3114618466B
:1001F000224600F014FA2D1A67EB01084F462246FA
:100200000120002100F00BFA17EB00094E41201EDF
:10021000A4F10104DFDC484631462A464346BDE8E6
:10022000F09F00000649074A0868504343F239022C
:10023000104408604008704701490860704700009A
:10024000000000206D4EC64140EA01039B0703D029
:1002500009E008C9121F08C0042AFAD203E011F805
:10026000013B00F8013B521EF9D27047D2B201E0C7
:1002700000F8012B491EFBD270470022F6E710B5AB
:1002800013460A4604461946FFF7F0FF204610BD04
:1002900010B5044604E00B7800F8013B03B1491C9B
:1002A000521EF8D2204610BD421C10F8011B002936
:1002B000FBD1801A704710B5002200E0521C835C0D
:1002C0008C5CA34201D1002BF8D1D8B2E1B2401A24
:1002D00010BD034611F8012B00F8012B002AF9D1BB
:1002E0001846704730B505460020034600E05B1C09
:1002F000934205D2EC5CC85C201A01D1002CF6D1E7
:1003000030BD2DE9FE4F804681EA0300C00F0C4648
:10031000009021F0004123F00045B8EB0200A94114
:1003200005D24046214690461C460B46024623F025
:100330000040104347D0270DC7F30A00C3F30A510A
:100340000290401A019040286BDAC3F3130040F486
:10035000801B0098924620B10023D2EB030A63EB86
:100360000B0B01985946C0F14002504600F057F976
:1003700006460D4650465946019A00F06FF910EBBB
:1003800008006141002487EA115284EAE7731A43A6
:1003900040D0009A62B3019A012A4FEA075215DC55
:1003A000001B61EB02014FF0004202EA0752CDE967
:1003B0000042001C41F5801132462B4600F0A6F9A0
:1003C00003B0BDE8F08F40462146F9E7001B61EB22
:1003D0000201001C41F5801300185B412018A2F5B2
:1003E000001747EB030140EAD570B6196D4111E0E3
:1003F0006D084FEA360645EAC0754FEA0752001B02
:1004000061EB0201001C41F5801149084FEA300000
:100410000019514132462B4603B0BDE8F04F00F0C1
:1004200066B90098012240000023D0EB020263EB82
:10043000E073009821464FEAE074B8EB000061EBEE
:100440000401E9E783F000435BE781F0004158E7EE
:100450002DE9FE4F81EA030404F0004421F000413D
:1004600000944FF0000B23F0004350EA01045ED0EB
:1004700052EA03045BD0C3F30A54C1F30A552C4477
:10048000A4F2F3340194A0FB0254C1F3130141F42C
:100490008011C3F3130343F4801301FB024400FBF8
:1004A000034E840A970A44EA815447EA8357A4FB1F
:1004B000076802958D0A05FB07854FEA932C04FB1C
:1004C0000C542705029D4FEA065847EA1637B5EB4C
:1004D00008056EEB070C870E920E47EA811742EA79
:1004E0008312A7FB0201B6EB0B0164EB00042B0D9A
:1004F00043EA0C335E1844EB1C50DA465146E7FBE6
:100500000201C5F313044FEA0B3343EA14534FEAD5
:100510000432019C43EA0603A4F10C040294009CFB
:10052000CDE900B400F0F2F803B0BDE8F08F002090
:100530000146F9E70EB5C10F80EAE0700844CA072A
:10054000002140F233438DE80E000A460B4600F0CE
:10055000DDF803B000BD70B5C1F30A5201F00045EB
:100560000024C1F3130140F2FF3341F480119A4299
:1005700001DA002070BD40F233439A42A2F23342C6
:1005800003DC524200F05AF800E090402C43F1D0D6
:10059000404270BD00F0004230F000400AD0C10D72
:1005A00001F56071C0F3160042EA0151C20840072C
:1005B0001143704700200146704701F0004330B4FA
:1005C00021F0004150EA010206D00A0DA2F5607246
:1005D000C1F31301002A02DC30BC00207047440F35
:1005E00044EAC104C100E01830BC00EBC25000F086
:1005F00047B830B50B46014600202022012409E00F
:1006000021FA02F59D4205D303FA02F5491B04FACB
:1006100002F52844151EA2F10102F1DC30BD202AAA
:1006200004DB203A00FA02F1002070479140C2F149
:10063000200320FA03F3194390407047202A04DB7B
:10064000203A21FA02F00021704721FA02F3D0404B
:10065000C2F120029140084319467047202A06DB68
:10066000CB17203A41FA02F043EAE07306E041FA80
:1006700002F3D040C2F1200291400843194670476E
:100680000029A8BF7047401C490008BF20F00100A6
:10069000704710B4B0FA80FC00FA0CF050EA010484
:1006A00004BF10BC704749B1CCF1200421FA04F416
:1006B00011FA0CF118BF012121430843A3EB0C01EF
:1006C000CB1D4FEA00614FEA102042BF002010BC52
:1006D000704700EBC35010440029A4BF10BC704702
:1006E000401C490008BF20F0010010BC704710B545
:1006F000141E73F1000408DA401C41F10001921845
:100700005B411A4301D120F0010010BD2DE9F04DED
:1007100092469B4611B1B1FA81F202E0B0FA80F242
:1007200020329046FFF77BFF04460F4640EA0A005E
:1007300041EA0B0153465A46084313D0114653EA87
:10074000010019D0C8F140025046FFF777FF054677
:100750000E46504659464246FFF761FF084305D012
:10076000012004E020463946BDE8F08D0020054315
:1007700046EAE0762C4337430A986305E40AA0EB87
:1007800008000022FD0A44EA47540A3002D500203E
:100790000146E9E7010510196941DDE9084500193D
:1007A0006941BDE8F04DA2E72DE9F04D81EA03046F
:1007B00004F0004B21F0004514464FF0000A23F0EE
:1007C000004150EA050220D054EA01021DD0C5F3D1
:1007D0000A570246C5F31303C1F31300C1F30A56C7
:1007E00040F4801543F48013A7EB0608101BD6468F
:1007F00008F2FD3873EB050002D308F1010801E0AF
:1008000092185B41B8F1000F03DA00200146BDE801
:10081000F08D00204FF48011064684460EE0171B31
:1008200073EB050705D3121B63EB050306434CEA84
:10083000010C49084FEA300092185B4150EA010769
:10084000EDD152EA030012D082EA040083EA0501E6
:10085000084305D0101BAB4106D20122002306E05D
:1008600000224FF0004302E06FF0010253101AEB38
:1008700006004CEB085110EB0A0041EB0B01BDE800
:10088000F04DFFF734BFC1F30A52C1F3130140F238
:10089000FF3341F480119A4202DA0020014670478A
:1008A00040F233439A42A2F2334202DC5242FFF753
:1008B000C5BEFFF7B4BE000030B5041E71F10004E0
:1008C00004DB4FF00044404264EB0101141E73F15D
:1008D000000405DB1C464FF00043524263EB040367
:1008E0008B4208BF824230BD30B5041E71F1000456
:1008F00004DB4FF00044404264EB0101141E73F12D
:10090000000405DB1C464FF00043524263EB040336
:10091000994208BF904230BD064C074D06E0E068A2
:1009200040F0010394E8070098471034AC42F6D336
:10093000FFF72EFCC0610208E06102080EB540F22C
:10094000334102910021CDE900110A460B46FFF721
:10095000DDFE03B000BD70B58D1810F8014B14F02A
:10096000030201D110F8012B231106D110F8013B2D
:1009700003E010F8016B01F8016B521EF9D1ABB125
:1009800010F8012B04F00C048A1A0C2C03D0A2EBF3
:1009900084129B1C08E010F8014BA2EB0422F8E73C
:1009A00012F8014B01F8014B5B1EF9D5A942D4D3D3
:1009B000002070BD80B582B0019042F20030C4F2D8
:1009C000010000900099486820F440304860019888
:1009D0004268009948681043486001980168486877
:1009E00020F480704860019801680269486840EA14
:1009F0000220486001980168486820F04070486013
:100A0000019801688268486810434860019801684D
:100A1000886820F40060886001980168C26888686E
:100A2000104388600198806A0121C0F600718842F5
:100A300019D0FFE701980168886820F0706088602D
:100A400001980168826A886810438860019801688B
:100A5000886820F04050886001980168C26A886800
:100A6000104388600CE001980168886820F070608D
:100A7000886001980168886820F040508860FFE72E
:100A800001980168886820F0020088600198027E61
:100A90000168886840EA42008860019890F8200068
:100AA00060B3FFE70198406A30B1FFE70198406A00
:100AB000082801D8FFE708E045F2E630C0F602005A
:100AC00040F2A6711DF038F8FFE701980168486808
:100AD00040F40060486001980168486820F4604074
:100AE000486001980168426A4EF20000CFF6FF703C
:100AF00000EB423248681043486006E00198016804
:100B0000486820F400604860FFE701980168C86AFF
:100B100020F47000C86201980168C2690020CFF615
:100B2000F07000EB0252C86A1043C8620198016875
:100B3000886820F400708860019890F8302001687F
:100B4000886840EA4220886001980168886820F43B
:100B500080608860019801684269886840EA822064
:100B6000886002B080BD000080B58AB0089007910F
:100B7000089820B9FFE7FF208DF827009BE0079831
:100B800020B9FFE7FF208DF8270094E0079890ED4B
:100B9000000A90ED013A90ED021A90ED032A20EE42
:100BA000030A21EE021A30EE010A30EE000A8DED42
:100BB000060A079890ED010A90ED021A20EE000A4D
:100BC00021EE011A30EE010A30EE001AB7EE000AEB
:100BD0008DED010A30EE410A8DED050A9DED060A04
:100BE000DDED050A22F0E0F89DED011A089880ED90
:100BF000010A079890ED000A90ED013A90ED024A43
:100C000090ED032A20EE040A22EE032A30EE420A77
:100C100030EE000A8DED040A9DED040AB0EEC00A24
:100C2000B4EE410AF1EE10FA0ADBFFE7DDED040A4B
:100C30009FED230A1CF094FF089880ED020A07E05C
:100C40009DED040A21F0AEFD089880ED020AFFE751
:100C5000079890ED000A90ED011A90ED022A90EDB0
:100C6000033A20EE030A21EE021A30EE010A30EEBA
:100C7000000A8DED030A079890ED020A90ED031A21
:100C800020EE000A21EE011A30EE010A30EE001AC1
:100C9000B7EE000A30EE410A8DED020A9DED030A1F
:100CA000DDED020A22F080F8089880ED000A0020AD
:100CB0008DF82700FFE79DF927000AB080BD00BF2F
:100CC000DB0FC93F80B58CB00A9009918DED080A01
:100CD0000A9820B9FFE7FF208DF82F0029E19DED4C
:100CE000081AB7EE000A80EE010A0A9880ED040A9D
:100CF0000A994FF07E5008600A99002048600A99CE
:100D000088600A99C8600998002800F00E81FFE702
:100D10000998016800914068FFF73CFC0246009882
:100D200001920A46019942EC101B8DED020BFFF770
:100D300031FC9DED020B41EC110B21F035FF8DEDE7
:100D4000040B9DF8170080F080008DF817000498C0
:100D50000599FFF732FC0790099890ED000AB5EE6F
:100D6000400AF1EE10FA2BD1FFE7099890ED010A45
:100D7000B5EE400AF1EE10FA22D1FFE7099890EDA6
:100D8000020AB5EE400AF1EE10FA19D1FFE70A990E
:100D900040F2C560C3F64D7008600A9944F62D20F4
:100DA000C3F60D4048600A994AF25640CBF63930F6
:100DB00088600A9944F2AD70C3F61970C860B3E058
:100DC0009DED070A9FED5D1AB4EE410AF1EE10FAAF
:100DD00008DBFFE79DED070AB5EE400AF1EE10FAD9
:100DE00019DDFFE70A9945F66E10C3F67F700860BB
:100DF0000A9945F20C30C3F6B01048600A9948F6DB
:100E0000AB00CBF6BB3088600A9949F28550C3F637
:100E10009750C86087E09DED070A9FED491AB4EE30
:100E2000410AF1EE10FA0ADBFFE79DED070A9FED9C
:100E3000431AB4EE410AF1EE10FA19DDFFE70A9900
:100E400040F2C560C3F64D7008600A9944F62D2043
:100E5000C3F60D4048600A994AF25640CBF6393045
:100E600088600A9944F2AD70C3F61970C86059E001
:100E70009DED070A9FED331AB4EE410AF1EE10FA28
:100E80000ADBFFE79DED070A9FED2D1AB4EE410A3C
:100E9000F1EE10FA19DDFFE70A9940F2C560C3F6DA
:100EA0004D7008600A9944F62D20C3F60D40486045
:100EB0000A994AF25640CBF6393088600A9944F2D2
:100EC000AD70C3F61970C8602BE09DED070A9FED69
:100ED0001D1AB4EE410AF1EE10FA08DBFFE79DEDB2
:100EE000070AB5EE400AF1EE10FA19DDFFE70A999C
:100EF00040F2C560C3F64D7008600A9944F62D2093
:100F0000C3F60D4048600A994AF25640CBF6393094
:100F100088600A9944F2AD70C3F61970C860FFE7A3
:100F2000FFE7FFE7FFE7FFE7FFE700208DF82F006F
:100F3000FFE79DF92F000CB080BD00BFDB0FC93F5C
:100F4000DB0F49400000B44281B0009000990020BE
:100F500088604860086001B07047000080B52DEDE2
:100F6000048BB2B030902F912E922D93309828B9E7
:100F7000FFE7FF208DF8C70000F0F7BD2F9828B9D4
:100F8000FFE7FF208DF8C70000F0EFBD2E9828B9CD
:100F9000FFE7FF208DF8C70000F0E7BD40F28411A5
:100FA000C2F200014EF69E70C3F6275008602D98DD
:100FB00048B9FFE730982F992E9A00F0DDFD8DF8A3
:100FC000C70000F0D2BD2D98006809902D984068A8
:100FD00008902D98806807909DED090AB5EE400AAB
:100FE000F1EE10FA19D1FFE79DED080AB5EE400ABF
:100FF000F1EE10FA11D1FFE79DED070AB5EE400AB8
:10100000F1EE10FA09D1FFE730982F992E9A00F0EF
:10101000B3FD8DF8C70000F0A8BD2F9800680690BA
:101020002F98406805902F98806804902E9800684B
:1010300003902E98406802902E9880680190309816
:101040009DED033A90ED010A90ED022A90ED031A0E
:1010500020EE430A9DED023A22EE032A30EE420AC8
:101060009DED012A21EE021A30EE410AB6EE001A79
:1010700020EE010A8DED270A30989DED034A90ED90
:10108000000A90ED023A90ED032A20EE040A9DED4D
:10109000014A23EE043A30EE030A9DED023A22EEB5
:1010A000032A30EE420A20EE010A8DED260A30981E
:1010B0009DED024A90ED000A90ED013A90ED032A71
:1010C00020EE040A9DED014A23EE043A30EE430A75
:1010D0009DED033A22EE032A30EE020A20EE010AC9
:1010E0008DED250A30989DED014A90ED000A90EDB6
:1010F000013A90ED022A20EE040A9DED024A23EE09
:10110000043A30EE030A9DED033A22EE032A30EE54
:10111000420A20EE010A8DED240A9DED060AB5EE85
:10112000400AF1EE10FA11D1FFE79DED050AB5EE88
:10113000400AF1EE10FA09D1FFE79DED040AB5EE81
:10114000400AF1EE10FA00F09984FFE79DED060ADF
:1011500020EE000A9DED051A21EE011A30EE010A7B
:101160009DED041A21EE011A30EE010A11F04AFC3D
:101170008DED2C0A9DED2C1A9DED060A20EE010A3C
:101180008DED060A9DED2C1A9DED050A20EE010A53
:101190008DED050A9DED2C1A9DED040A20EE010A45
:1011A0008DED040A9DED090A20EE000A9DED081A56
:1011B00021EE011A30EE010A9DED071A21EE011A07
:1011C00030EE010A11F01EFC8DED2C0A9DED2C1A5B
:1011D0009DED090A20EE010A8DED090A9DED2C1AFC
:1011E0009DED080A20EE010A8DED080A9DED2C1AEE
:1011F0009DED070A20EE010A8DED070A309890ED6B
:10120000000A30EE000A9DED091A20EE010A8DED6C
:10121000210A309890ED000A30EE000A9DED081A80
:1012200020EE010A8DED200A309890ED000A30EE94
:10123000000A9DED071A20EE010A8DED1F0A309875
:1012400090ED010A30EE000A9DED091A20EE010A28
:101250008DED1E0A309890ED000A30EE000A8DEDFB
:10126000190A309890ED010A30EE000A8DED180A47
:10127000309890ED020A30EE000A8DED170A309892
:1012800090ED030A30EE000A8DED160A309890EDCD
:10129000000A90ED021A30EE000A20EE010A8DEDF0
:1012A000150A309890ED020A90ED031A30EE000A0C
:1012B00020EE010A8DED140A309890ED000A20EE20
:1012C000000A8DED130A309890ED000A90ED011A96
:1012D00020EE010A8DED120A309890ED000A90ED93
:1012E000021A20EE010A8DED110A309890ED000AE5
:1012F00090ED031A20EE010A8DED100A309890ED62
:10130000010A20EE000A8DED0F0A309890ED010AD7
:1013100090ED021A20EE010A8DED0E0A309890ED44
:10132000010A90ED031A20EE010A8DED0D0A3098A6
:1013300090ED020A20EE000A8DED0C0A309890ED37
:10134000020A90ED031A20EE010A8DED0B0A309887
:1013500090ED030A20EE000A8DED0A0A9DED091AB0
:101360009DED130A21EE000A9DED202A309890EDA4
:10137000025A90ED033A22EE032A30EE420A9DED26
:101380001F2A22EE052A30EE020A9DED0F2A21EED9
:10139000022A30EE020A9DED182A9DED084A22EE3F
:1013A000044A24EE054A30EE040A9DED074A22EE77
:1013B000042A22EE032A30EE020A9DED0C2A21EEC9
:1013C000022A30EE420A9DED0A2A21EE021A30EE80
:1013D000410A8DED230A9DED210A309890ED015AC6
:1013E00090ED024A90ED033A20EE030A9DED081AB3
:1013F0009DED132A21EE022A30EE020A9DED1F2AEE
:1014000022EE052A30EE420A9DED1E2A22EE042A23
:1014100030EE020A9DED0F2A21EE022A30EE420A3A
:101420009DED0C2A21EE022A30EE020A9DED172ACC
:101430009DED074A22EE042A22EE032A30EE020A2C
:101440009DED0A2A21EE021A30EE410A8DED220AA4
:101450009DED230A20EE000A9DED221A21EE011ACD
:1014600030EE010A11F0CEFAB7EE006A86EE000AFD
:101470008DED1D0A9DED210A309890ED012A90ED29
:10148000021A90ED033A20EE011A9DED200A20EE9B
:10149000020A30EE412A9DED071A9DED130A21EE56
:1014A000000A30EE022A9DED1E0A20EE030A30EEFD
:1014B000020A9DED0F2A21EE022A30EE420A9DED2E
:1014C000172A9DED084A22EE042A22EE032A30EE66
:1014D000020A9DED0C2A21EE022A30EE420A9DED11
:1014E0000A2A21EE021A30EE010A8DED1C0A9DED4A
:1014F0001D0A30EE000A8DED1B0A9DED1C0A30EE30
:10150000000A8DED1A0A9DED170ADDED0D0A30EE89
:10151000A02A9DED151A31EE422A9DED061A31EEF4
:10152000021A20EE010A9DED181ADDED123A33EE93
:10153000A32A9DED143A32EE032A9DED053A32EED0
:10154000432A21EE021A70EE014A9DED1C3A3098B2
:1015500090ED011A90ED020AD0ED032A63EE001A15
:101560009DED1D2A9DED0C7AB6EE004A8DED004AE8
:1015700077EE445A9DED0A5A35EE255A62EE055A29
:101580009DED115A75EE606A63EE266A75EEA66AE5
:10159000DDED095A75EEA65A61EEA51A71EEA41A90
:1015A00062EE222A23EE011A31EE621ADDED0E2AD6
:1015B000DDED104A72EEE42A62EE222ADDED0B4ADE
:1015C00073EEA43A63EE233A72EEA32ADDED083AF5
:1015D00072EEE32A21EE221A31EE211A22EE000ADF
:1015E00035EE205A22EE052A9DED0F5A34EE455A6B
:1015F00035EE475A23EE053A32EE032A9DED073ABF
:1016000032EE432A20EE020A30EE010A8DED2B0A5B
:101610009DED160ADDED0D2A32EEA21A9DED152A7A
:1016200031EE421A9DED062A31EE421A20EE010AF1
:101630009DED191ADDED126A36EEA62A9DED143ADB
:1016400032EE032A9DED053A32EE432A21EE021ACC
:1016500030EE011A3098D0ED005AD0ED014AD0EDAD
:10166000023A90ED032AB1EE000A24EE803A9DED95
:101670000F7A37EE075A75EE461ADDED0C0A30EE9A
:10168000A05A75EE211A9DED045A35EE215A23EE2B
:10169000053A31EE031A9DED1C5A65EE027A9DED76
:1016A0001D3A74EE601A9DED0A8A71EEC81A23EE97
:1016B000218ADDED111A32EEE19A25EE099A38EE13
:1016C000098A9DED099A38EE498A67EE887A31EEEB
:1016D000271A63EE233A65EE255A73EEA53ADDED3F
:1016E0000E5ADDED107A75EEE75A63EE255ADDED00
:1016F0000B7A76EEA76A65EE266A75EEA65ADDEDE0
:10170000086A75EEE65A63EEA53A31EE231A23EE27
:10171000022ADDED1A3A63EEA43A32EE632A71EE44
:10172000A21A23EE213A34EE477A37EE607A25EE9C
:10173000075A33EE053A9DED075A33EE453A22EE4D
:10174000032A31EE021A8DED2A1A9DED191ADDEDEC
:101750000D0A30EEA03A9DED152A32EE433A9DED8A
:10176000062A32EE032A21EE021A9DED162ADDED3D
:10177000124A34EEA43A9DED145A33EE053A9DED2B
:10178000055A33EE453A22EE032A31EE022A30980A
:1017900090ED001AD0ED011AD0ED022AD0ED033AF7
:1017A00022EE800A9DED0F5A35EE053A33EE467A69
:1017B0009DED0C6A36EE063A33EE077A9DED043A5B
:1017C00033EE073A20EE030A70EE025A9DED1B0A33
:1017D00020EE620A9DED1C3A23EE012A30EE420A09
:1017E0009DED1D2A34EE467ADDED0A6A37EE667A03
:1017F00062EE076A9DED117A70EEC77A63EE277A82
:1018000076EEA76ADDED097A76EEE76A20EE260A23
:1018100030EE250A62EE211A63EE233A71EEA31A26
:10182000DDED0E3ADDED105A73EEE53A62EE233A45
:10183000DDED0B5A74EEA54A63EE244A73EEA43A2A
:10184000DDED084A73EEE43A61EEA31A30EE210AA8
:1018500022EE011ADDED1A1A61EEA21A31EE611ABA
:1018600037EE207A22EE072A34EE455A35EE465AF4
:1018700023EE053A32EE032A9DED073A32EE432A73
:1018800021EE021A30EE010A8DED290A9DED180AAB
:101890009DED0D7A37EE071A9DED152A31EE421AAD
:1018A0009DED062A31EE421A20EE010A9DED171A2F
:1018B000DDED122A32EEA22A9DED143A32EE032A11
:1018C0009DED053A32EE432A21EE021A70EE013AFE
:1018D0009DED1B1A3098D0ED001A90ED010AD0ED65
:1018E000020A90ED032A21EE022A9DED1C3A23EE16
:1018F000001A31EE421A9DED1D2A9DED0C5A34EE70
:10190000456ADDED0A4A36EE646A62EE064A9DEDEE
:10191000116A77EE465A63EE255A74EEA54ADDED5C
:10192000095A74EEE54A21EE241A31EE231A62EECA
:10193000211A63EE200A70EEE10ADDED0E1ADDEDEC
:10194000103A71EEE31A62EE211ADDED0B3A72EEF7
:10195000A32A63EE222A71EEA21ADDED082A71EEA7
:10196000E21A60EEA10A31EE201A22EE000A36EEEB
:10197000076A22EE062A9DED0F6A34EE464A34EEDF
:10198000454A23EE043A32EE032A9DED073A32EE41
:10199000432A20EE020A30EE010A8DED280A9DED61
:1019A0002B0A20EE000A9DED2A1A21EE011A30EED4
:1019B000010A9DED291A21EE011A30EE010A9DED72
:1019C000281A21EE011A30EE010A11F01BF88DEDF4
:1019D0002C0A9DED2C1A9DED2B0A20EE010A8DEDAF
:1019E0002B0A9DED2C1A9DED2A0A20EE010A8DEDA1
:1019F0002A0A9DED2C1A9DED290A20EE010A8DED93
:101A0000290A9DED2C1A9DED280A20EE010A8DED84
:101A1000280A40F28410C2F2000090ED000A9DED09
:101A20002B1A20EE011A9DED270A30EE410A8DEDAA
:101A3000270A90ED000A9DED2A1A20EE011A9DED6D
:101A4000260A30EE410A8DED260A90ED000A9DED42
:101A5000291A20EE011A9DED250A30EE410A8DED7E
:101A6000250A90ED000A9DED281A20EE011A9DED41
:101A7000240A30EE410A8DED240AFFE79DED271A76
:101A8000309890ED000A90ED042A21EE021A30EE13
:101A9000010A80ED000A9DED261A309890ED010AAA
:101AA00090ED042A21EE021A30EE010A80ED010ABF
:101AB0009DED251A309890ED020A90ED042A21EE52
:101AC000021A30EE010A80ED020A9DED241A3098C8
:101AD00090ED030A90ED042A21EE021A30EE010A7D
:101AE00080ED030A309890ED000A90ED013A90EDF8
:101AF000022A90ED031A20EE000A23EE033A30EE9C
:101B0000030A22EE022A30EE020A21EE011A30EE1A
:101B1000010A10F077FF8DED2C0A9DED2C1A3098FC
:101B200090ED000A20EE010A80ED000A9DED2C1ACE
:101B3000309890ED010A20EE010A80ED010A9DED3A
:101B40002C1A309890ED020A20EE010A80ED020A6C
:101B50009DED2C1A309890ED030A20EE010A80EDDD
:101B6000030A00208DF8C700FFE79DF9C70032B0D7
:101B7000BDEC048B80BD000080B5A0B01E901D910F
:101B80001C921E9820B9FFE7FF208DF87F00D3E25A
:101B90001D9820B9FFE7FF208DF87F00CCE21C984C
:101BA00020B9FFE7FF208DF87F00C5E240F28411E5
:101BB000C2F2000142F60230C3F6075008601D98D9
:101BC00000681B901D9840681A901D9880681990B5
:101BD0001C98006818901C98406817901C988068A2
:101BE00016901E989DED183A90ED010A90ED022A8C
:101BF00090ED031A20EE430A9DED173A22EE032AD8
:101C000030EE420A9DED162A21EE021A30EE410A0C
:101C1000B6EE001A20EE010A8DED100A1E989DED19
:101C2000184A90ED000A90ED023A90ED032A20EE5A
:101C3000040A9DED164A23EE043A30EE030A9DEDA8
:101C4000173A22EE032A30EE420A20EE010A8DED09
:101C50000F0A1E989DED174A90ED000A90ED013A8B
:101C600090ED032A20EE040A9DED164A23EE043A75
:101C700030EE430A9DED183A22EE032A30EE020AB6
:101C800020EE010A8DED0E0A1E989DED164A90ED8C
:101C9000000A90ED013A90ED022A20EE040A9DED33
:101CA000174A23EE043A30EE030A9DED183A22EE6D
:101CB000032A30EE420A20EE010A8DED0D0A9DED59
:101CC0001B0AB5EE400AF1EE10FA11D1FFE79DEDC7
:101CD0001A0AB5EE400AF1EE10FA09D1FFE79DEDC0
:101CE000190AB5EE400AF1EE10FA00F0AE81FFE7F6
:101CF0009DED1B0A20EE000A9DED1A1A21EE011A35
:101D000030EE010A9DED191A21EE011A30EE010A9A
:101D100010F078FE8DED150A9DED151A9DED1B0A4C
:101D200020EE010A8DED1B0A9DED151A9DED1A0A94
:101D300020EE010A8DED1A0A9DED151A9DED190A86
:101D400020EE010A8DED190A1E9890ED000A30EE82
:101D5000000A8DED0C0A1E9890ED010A30EE000A83
:101D60008DED0B0A1E9890ED020A30EE000A8DED03
:101D70000A0A1E9890ED030A30EE000A8DED090A5A
:101D80001E9890ED000AB1EE003A20EE030A8DEDA8
:101D9000080A1E9890ED010A20EE030A8DED070A4D
:101DA0001E9890ED020A20EE030A8DED060A1E9899
:101DB00090ED010AB2EE001A20EE010A8DED050A3F
:101DC0001E9890ED020A20EE010A8DED040A1E987D
:101DD00090ED000A20EE000A8DED030A1E9890EDAA
:101DE000010A20EE000A8DED020A1E9890ED020A0B
:101DF00020EE000A8DED010A1E9890ED030A20EEF8
:101E0000000A8DED000A9DED081A9DED010A21EEF4
:101E1000000A9DED0A2A9DED1B4A22EE042A30EEAF
:101E2000020A9DED022A21EE021A30EE010A9DED12
:101E30000B1A9DED1A2A21EE021A30EE410A8DEDA1
:101E4000140A9DED071A9DED000A21EE000A9DED92
:101E5000092A9DED1B4A22EE042A30EE420A9DED2E
:101E6000032A22EE032A1E9890ED014A22EE042A4C
:101E700030EE020A9DED0C2A9DED1A4A22EE042A4C
:101E800030EE420A30EE410A9DED052A9DED024AF0
:101E900022EE044A30EE040A9DED014A22EE042AA5
:101EA00030EE020A9DED192A21EE021A30EE010AE7
:101EB0008DED130A9DED030A20EE030A1E9890EDA6
:101EC000021A20EE010A9DED0C1A9DED1B2A21EE4F
:101ED000021A30EE010A9DED061A9DED002A21EE50
:101EE000022A30EE020A9DED092A9DED1A4A22EEE1
:101EF000042A30EE420A30EE410A9DED042A9DED9F
:101F0000024A22EE044A30EE040A9DED014A22EE16
:101F1000042A30EE020A9DED192A21EE021A30EE53
:101F2000010A8DED120A9DED020A20EE030A1E98A9
:101F300090ED032A20EE020A9DED0B1A9DED1B4A3F
:101F400021EE041A30EE410A9DED011A21EE031A2A
:101F500021EE021A30EE010A9DED0A1A9DED1A2AB1
:101F600021EE021A30EE410A8DED110A9DED140AA0
:101F700020EE000A9DED131A21EE011A30EE010A3F
:101F80009DED121A21EE011A30EE010A9DED111A93
:101F900021EE011A30EE010A10F034FD8DED150A24
:101FA0009DED151A9DED140A20EE010A8DED140A1F
:101FB0009DED151A9DED130A20EE010A8DED130A11
:101FC0009DED151A9DED120A20EE010A8DED120A03
:101FD0009DED151A9DED110A20EE010A8DED110AF5
:101FE00040F28410C2F2000090ED000A9DED141A38
:101FF00020EE011A9DED100A30EE410A8DED100A17
:1020000090ED000A9DED131A20EE011A9DED0F0AC6
:1020100030EE410A8DED0F0A90ED000A9DED121A87
:1020200020EE011A9DED0E0A30EE410A8DED0E0AEA
:1020300090ED000A9DED111A20EE011A9DED0D0A9A
:1020400030EE410A8DED0D0AFFE79DED101A1E9846
:1020500090ED000A90ED042A21EE021A30EE010AFA
:1020600080ED000A9DED0F1A1E9890ED010A90ED8B
:10207000042A21EE021A30EE010A80ED010A9DEDDC
:102080000E1A1E9890ED020A90ED042A21EE021A13
:1020900030EE010A80ED020A9DED0D1A1E9890EDBA
:1020A000030A90ED042A21EE021A30EE010A80EDB7
:1020B000030A1E9890ED000A90ED013A90ED022A75
:1020C00090ED031A20EE000A23EE033A30EE030AE5
:1020D00022EE022A30EE020A21EE011A30EE010A47
:1020E00010F090FC8DED150A9DED151A1E9890EDDF
:1020F000000A20EE010A80ED000A9DED151A1E98D7
:1021000090ED010A20EE010A80ED010A9DED151AFD
:102110001E9890ED020A20EE010A80ED020A9DED64
:10212000151A1E9890ED030A20EE010A80ED030AAD
:1021300000208DF87F00FFE79DF97F0020B080BD73
:1021400084B002900191029820B9FFE7FE208DF83B
:102150000F001CE0019820B9FFE7FE208DF80F006A
:1021600015E0029900200090C1F81B0088614861C9
:102170000861C860886048600199886148610861A9
:10218000C8608860486008608DF80F00FFE79DF91F
:102190000F0004B07047000080B582B00090009836
:1021A00020B9FFE7FE208DF807002AE042F26860C0
:1021B000C2F200000078C00720B1FFE7FD208DF8D3
:1021C00007001EE01CF078F943F2A441C2F20001BE
:1021D000086020B9FFE7FE208DF8070011E042F209
:1021E0008542C0F600020220032101F037F942F2D5
:1021F0006861C2F200010120087000208DF807001C
:10220000FFE79DF9070002B080BD000080B582B0F5
:10221000019000910199C42081F826000199DDF810
:1022200000C0DCF80000DCF80420DCF80830DCF842
:102230000CC0C1F833C0C1F82F30C1F82B20C1F851
:1022400027000199002081F83700019890F84A0092
:10225000012808D1FFE7019991F8370040F001000B
:1022600081F837001DE0019890F84A00022808D153
:10227000FFE7019991F8370040F0020081F837003C
:102280000EE0019890F84A00032808D1FFE7019971
:1022900091F8370040F0040081F83700FFE7FFE7CE
:1022A000FFE70198273021214FF6FF7202F0DEFB95
:1022B0000199A1F84800002002B080BD80B582B02D
:1022C000019000910199A820C8770198203004213D
:1022D0004FF6FF7202F0CAFB01998884002002B019
:1022E00080BD000080B584B0029001910298043056
:1022F0001B2102F0D7FB08B9FFE724E002988068B1
:102300000199486002984068019908600298C06885
:10231000019988600298007CC0F3C000019908769A
:102320000298D0F811000199C8600298D0F8150001
:10233000019908610298D0F81900019948610020BC
:102340008DF80F000AE041F25441C2F20001086822
:1023500001300860FF208DF80F00FFE79DF90F00A6
:1023600004B080BD80B582B00090022001F016F864
:10237000009904311B2210F061F920B9FFE7002019
:102380008DF8070003E0FF208DF80700FFE79DF9B7
:10239000070002B080BD000080B584B002908DF8C7
:1023A00007109DF80700C00790B1FFE7022000F07A
:1023B000F5FF02991F312B2210F0D0F920B9FFE769
:1023C00000208DF80F0015E0FF208DF80F0011E0C0
:1023D000022000F0E3FF02992631242210F0BEF91A
:1023E00020B9FFE700208DF80F0003E0FF208DF8F3
:1023F0000F00FFE79DF90F0004B080BD80B54FF4DA
:102400008040012100221BF0C9FFA0F58040B0FAF6
:1024100080F0400980BD000084B08DED030ACDED51
:10242000020A9DED030A9DED021AB1EE411AB4EEC7
:10243000410AF1EE10FA07DAFFE79DED020AB1EE6C
:10244000400A8DED010A18E09DED030A9DED021A88
:10245000B4EE410AF1EE10FA05DDFFE79DED020A48
:102460008DED000A04E09DED030A8DED000AFFE703
:102470009DED000A8DED010AFFE79DED010A04B014
:102480007047000080B543F2A440C2F2000000682B
:102490004FF480411BF030FF80BD000080B543F257
:1024A0009440C2F20000006802211BF025FF80BDAD
:1024B00080B582B040F61C32C2F2000200200190CA
:1024C0001221132300F06EFA019802B080BD0000C3
:1024D00080B5082001214FF0FF321BF05FFF80BD67
:1024E00081B000909FED010A01B070470000C84321
:1024F00080B543F29440C2F20000006801211BF055
:10250000FBFE80BD82B00190019890ED000A002092
:102510009FED141AB4EE410AF1EE10FA00901BDAA6
:10252000FFE7019890ED010A00209FED0E1AB4EE2E
:10253000410AF1EE10FA00900EDAFFE7019890EDF3
:10254000020A9FED081A0020B4EE410AF1EE10FADB
:10255000B8BF01200090FFE7009800F0010002B032
:10256000704700BF8FC2F53C80B540F61C30C2F208
:102570000000C21D01200221062300F013FA0020F2
:1025800080BD000080B5042001214FF0FF321BF018
:1025900005FF80BD80B58CB00A9009910A9820B9DA
:1025A000FFE7FE208DF82F00B5E0099820B9FFE77E
:1025B000FE208DF82F00AEE042F26460C2F200000F
:1025C0000078C00720B1FFE7FD208DF82F00A2E0C2
:1025D0001BF072FF43F29441C2F20001086020B97F
:1025E000FFE7FE208DF82F0095E009980A99C86151
:1025F000002008907E21B622069200F087FA069A03
:102600000120142100F082FA1E20079000F01CFB2C
:102610000799089800F00CFA0899084600F008FAA3
:102620001E2804D0FFE7FC208DF82F0073E0012066
:10263000002100F0FDF90F2804D0FFE7FC208DF801
:102640002F0068E01020039000F0A6FB20200490EB
:1026500000F0A2FB42F62D12C0F600020121029109
:10266000084600F079FE039842F29D41C0F6000151
:1026700000F006FC049842F2F141C0F6000100F0BF
:10268000FFFB002005904021AA2200F03FFA029AA9
:102690000598412100F03AFA05985321082200F0EC
:1026A00035FA059858210422019200F02FFA019A78
:1026B00005987D2100F02AFA322000F0C5FA029A2E
:1026C0000F21104600F022FA02980399032200F02D
:1026D0001DFA0298059A162100F018FA029A18219C
:1026E000104600F013FA02981521802200F00EFA2D
:1026F0000A2000F0A9FA0299039842F26462C2F239
:102700000002117000F082FB049800F07FFB059836
:102710008DF82F00FFE79DF92F000CB080BD000061
:1027200084B00290029820B9FFE7FE208DF80F00D8
:102730006AE040F61C31C2F20001B1F80100ADF8C8
:102740000600B1F80300ADF80400B1F80500ADF8DB
:102750000200BDF9060000EE100AB8EEC00A0298A9
:1027600080ED000ABDF9040000EE100AB8EEC00AC0
:10277000029880ED010ABDF9020000EE100AB8EEE1
:10278000C00A029880ED020A029890ED000A9FEDBF
:10279000201A80EE010A80ED000A029890ED010AED
:1027A00080EE010A80ED010A029890ED020A80EEA7
:1027B000010A80ED020A487C897CC00040EA511081
:1027C000ADF80000BDF90000B0F5806F07DBFFE752
:1027D000BDF80000A0F50060ADF80000FFE7BDF90E
:1027E000000000EE100AB8EEC00AB4EE001A20EEA7
:1027F000010AB3EE071A30EE010A029880ED060ACC
:1028000000208DF80F00FFE79DF90F0004B070471E
:1028100000A0AA4584B00290029820B9FFE7FE20EC
:102820008DF80F007AE040F61C30C2F20000B0F8DC
:102830000710ADF80610B0F80910ADF80410B0F8A4
:102840000B00ADF80200BDF9060000EE100AB8EE6C
:10285000C00A029880ED030ABDF9040000EE100AD8
:10286000B8EEC00A029880ED040ABDF9020000EE3D
:10287000100AB8EEC00A029880ED050A029890EDA1
:10288000030A9FED281A80EE010A80ED030A0298E0
:1028900090ED040A80EE010A80ED040A029890EDA2
:1028A000050A80EE010A80ED050A029890ED030A00
:1028B0009FED1D1A20EE010A80ED030A029890EDAB
:1028C000040A20EE010A80ED040A029890ED050A40
:1028D00020EE010A80ED050A0298C16991ED001A07
:1028E00090ED030A30EE410A80ED030A0298C169B7
:1028F00091ED011A90ED040A30EE410A80ED040AD0
:102900000298C16991ED021A90ED050A30EE410A74
:1029100080ED050AFE208DF80F00FFE79DF90F00FE
:1029200004B070476F12034235FA8E3C80B5002028
:10293000C4F20200102108F02DFF80B9FFE700204B
:10294000C4F202001021012208F04EFF43F294402D
:10295000C2F20000006808211BF0CEFCFFE740F245
:102960000040C4F20200012108F014FF88B9FFE71B
:1029700040F20040C4F202000122114608F034FF88
:1029800043F29440C2F20000006804211BF0B4FC42
:10299000FFE780BD80B5032001214FF0FF321BF01F
:1029A000FDFC80BD80B586B08DF817008DF816103F
:1029B00004928DF80F30049808B9FFE736E09DF8CF
:1029C00017000146029120B1FFE70298012808D0C4
:1029D00010E00020C4F202001021002208F004FFE1
:1029E00008E040F20040C4F202000121002208F099
:1029F000FBFEFFE79DF8160040F0800040F62F3107
:102A0000C2F20001009108700120019000F084FCE6
:102A10000099019A14230CF025F9019800F07CFC30
:102A200004999DF80F200BF0DFFFFFE706B080BD93
:102A300080B586B08DF816008DF81510012000F0D5
:102A400003F99DF816000146049120B1FFE70498B0
:102A5000012808D010E00020C4F20200102100225A
:102A600008F0C2FE08E040F20040C4F2020001217A
:102A7000002208F0B9FEFFE79DF8150040F0800045
:102A800040F62F31C2F20001019108700120009040
:102A900000F042FC009A0199142302930CF0E2F832
:102AA000009800F039FC0199029B02220BF084FE91
:102AB0009DF816000146039120B1FFE70398012815
:102AC0000FD01EE00020C4F202001021012208F005
:102AD0008BFE40F62F30C2F2000040788DF81700D0
:102AE0000FE040F20040C4F202000122114608F05B
:102AF0007BFE40F62F30C2F2000000788DF8170000
:102B0000FFE79DF8170006B080BD000080B584B0D7
:102B10008DF80F008DF80E108DF80D209DF80E0029
:102B200000F07F0040F62F31C2F2000108709DF8DE
:102B30000D004870012000F087F89DF80F00014655
:102B4000029120B1FFE70298012808D010E0002090
:102B5000C4F202001021002208F046FE08E040F214
:102B60000040C4F202000121002208F03DFEFFE710
:102B7000012000F0D1FB40F62F31C2F20001022209
:102B800014230CF06FF89DF80F000146019120B15D
:102B9000FFE70198012808D010E00020C4F20200ED
:102BA0001021012208F020FE08E040F20040C4F2AB
:102BB00002000122114608F017FEFFE704B080BDB5
:102BC00083B08DF807009DF807000146009150B1D1
:102BD000FFE7009801280CD1FFE741F6F010C2F2A0
:102BE0000000029008E041F6C810C2F20000029016
:102BF00002E000200290FFE7029803B07047000057
:102C000082B08DF806008DF805100092009820B96A
:102C1000FFE7FE208DF8070011E000989DF80610F0
:102C200040F25843C2F20003342211FB02319DF8F6
:102C3000052041F8220000208DF80700FFE79DF9EC
:102C4000070002B07047000080B586B004901BF00A
:102C5000DBF801464FF47A70B0FBF1F00390049872
:102C60000399B0FBF1F002901BF090F80146481C6C
:102C7000019198B1FFE70198022820D3FFE701985E
:102C800002280FD0FFE701980338022806D3FFE798
:102C900001986FF00041884215D1FFE7FF208DF8C1
:102CA000170014E0029818B1FFE70298009002E0C4
:102CB00001200090FFE700981BF022F803E0049841
:102CC00007F0FCFFFFE700208DF81700FFE79DF9F4
:102CD000170006B080BD000080B588B00790079847
:102CE000E0B1FFE707980B2818D8FFE70798049092
:102CF00000200290022006900120059008F03EF985
:102D0000FFE7322004F0D8FC08B1FFE7F9E702A89A
:102D100001A907F0F5FF08F0A3F8FFE708B080BDB0
:102D200080B584B003900291019202980399019AB0
:102D3000FDF78AFA04B080BD80B584B0039002919B
:102D4000019208F01BF9FFE70198C0B1FFE7FFE728
:102D5000322004F0B1FC08B1FFE7F9E703990298CB
:102D600002780023184608F085F803980130039094
:102D7000029801300290019801380190E4E708F0D0
:102D80006FF804B080BD000080B582B0019001985A
:102D90001DF078F902B080BD80B582B0ADF80400B6
:102DA000BDF804000138014600911F2822D800997F
:102DB000DFE801F0182020202020201C20202020E7
:102DC0002020201020202020202020202020202013
:102DD000202020140A2009F02FF90FE0172009F015
:102DE0002BF90BE0062009F027F907E0092009F08C
:102DF00023F903E0FF208DF8070003E000208DF8A1
:102E00000700FFE79DF9070002B080BD80B582B0E2
:102E1000ADF80400BDF804000138014600911F28F8
:102E200022D80099DFE801F0182020202020201C63
:102E300020202020202020102020202020202020A2
:102E400020202020202020140A2009F00DF90FE076
:102E5000172009F009F90BE0062009F005F907E051
:102E6000092009F001F903E0FF208DF8070003E0D5
:102E700000208DF80700FFE79DF9070002B080BD34
:102E800083B0ADF808000191019820B9FFE7FE205A
:102E90008DF80B0025E000208DF80300FFE79DF87A
:102EA00003000F2819DCFFE7BDF808009DF80310A8
:102EB000C840C00750B1FFE701989DF8032040F2D9
:102EC000DC41C2F2000141F8220006E0FFE79DF874
:102ED000030001308DF80300E1E700208DF80B00BE
:102EE000FFE79DF90B0003B07047000080B588B084
:102EF000082004900120059000200690079041F6DC
:102F00008010C2F2000004A905F08CF818B1FFE7A8
:102F100004F022F9FFE741F68010C2F200000190B0
:102F200005F0BAFC0198052105F020FC019805F098
:102F3000D9F903909DED030AB8EE400A40F24C40E7
:102F4000C2F2000090ED001A20EE010A9FED041A73
:102F500020EE010A8DED020A9DED020A08B080BD47
:102F60005D74214180B588B0102004900120059047
:102F700000200690079041F63810C2F2000004A924
:102F800005F050F818B1FFE704F0E6F8FFE741F666
:102F90003810C2F20000019005F07EFC0198052176
:102FA00005F0E4FB019805F09DF903909DED030AFF
:102FB000B8EE400A40F24C40C2F2000090ED001A18
:102FC00020EE010A8DED020A9DED020A9FED061A20
:102FD00030EE010A9FED051A20EE010AB3EE091A40
:102FE00030EE010A08B080BD5C8F42BF0000C843CC
:102FF00080B588B006AA0392024603988DF81E2079
:103000008DF81D1080ED000A90ED000AB7EE001A51
:10301000B4EE410AF1EE10FA04DDFFE7FF208DF86F
:103020001F0097E0039890ED000A9FED4C1A20EEE8
:10303000010ABDEEC00A10EE100AADF812009DF8AC
:103040001E0001460291F0B1FFE70298012804D06A
:10305000FFE7029802280BD020E0BDF8120042F2F0
:103060008441C2F200010968C8630820059015E098
:10307000BDF8120042F28441C2F20001096888637F
:10308000042005900AE0BDF8120042F28441C2F229
:1030900000010968486300200590FFE79DF81D00C6
:1030A0000146019140B1FFE70198012814D0FFE7E4
:1030B0000198022820D049E0059942F28440C2F2EA
:1030C00000000EF0FFF9059A42F27C61C2F20001A5
:1030D00008681043086039E0059942F28440C2F262
:1030E00000000EF0D1FB059A42F27C61C2F20001B1
:1030F00008689043086029E042F27C60C2F2000058
:1031000000680599084210D0FFE7059942F2844013
:10311000C2F200000EF0B8FB059A42F27C61C2F2E6
:1031200000010868904308600FE0059942F284406E
:10313000C2F200000EF0C6F9059A42F27C61C2F2BA
:103140000001086810430860FFE7FFE700208DF8E2
:103150001F00FFE79DF91F0008B080BD00FF7F47FB
:1031600080B582B0019001981CF068FC02B080BD6F
:1031700080B586B004A90291014602988DF8161018
:1031800080ED000A90ED000AB7EE001AB4EE410A95
:10319000F1EE10FA04DDFFE7FF208DF817006AE07A
:1031A000029890ED000AB5EE400AF1EE10FA03DA4B
:1031B000FFE700200490FFE79DF81600014601910B
:1031C00020B1FFE70198012815D029E0029890ED81
:1031D000000A42F2AC30C2F20000006890ED0B1A17
:1031E000B8EE411A20EE010ABDEEC00A10EE100A38
:1031F000ADF80E0014E0029890ED000A42F264303F
:10320000C2F20000006890ED0B1AB8EE411A20EEF1
:10321000010ABDEEC00A10EE100AADF80E00FFE77D
:10322000BDF80E0001281DDBFFE79DF816000146E2
:10323000009120B1FFE70098012809D011E0BDF806
:103240000E0042F2AC31C2F200010968486308E0A6
:10325000BDF80E0042F26431C2F200010968486311
:10326000FFE704E09DF8160000F02CF8FFE70020CF
:103270008DF81700FFE79DF9170006B080BD00002C
:1032800080B582B08DF807009DF8070001460091D7
:1032900020B1FFE70098012808D00FE042F2AC30DF
:1032A000C2F2000000210EF00DF907E042F2643096
:1032B000C2F2000000210EF005F9FFE7002002B085
:1032C00080BD000080B584B08DF80F009DF80F0020
:1032D0000146029120B1FFE70298012808D00FE0D3
:1032E00042F2AC30C2F2000000210EF0CDFA07E04D
:1032F00042F26430C2F2000000210EF0C5FAFFE78E
:1033000041F20040C4F2020040210022019208F084
:103310006BFA019804B080BD83B08DF807009DF86A
:1033200007000146009120B1FFE70098012806D070
:103330000BE042F20C30C2F20000029008E042F2D0
:10334000B420C2F20000029002E000200290FFE7E9
:10335000029803B07047000082B08DF806008DF827
:1033600005100092009820B9FFE7FE208DF80700B5
:1033700010E000989DF8062040F2A051C2F2000132
:1033800001EB42119DF8052041F8220000208DF844
:103390000700FFE79DF9070002B0704783B08DF882
:1033A00007009DF807000146009140B1FFE7009833
:1033B00001280AD0FFE7009802280CD011E042F261
:1033C000A050C2F2000002900EE042F25C50C2F245
:1033D0000000029008E042F2E450C2F200000290C5
:1033E00002E000200290FFE7029803B0704700005F
:1033F00080B582B00190019800680068C00600287E
:103400002AD5FFE7FFE700200090019800680068D8
:10341000009001980068406800900098FFE70198CC
:1034200016F078FA00EBC00140F22060C2F2000012
:1034300000EB8100006A70B1FFE7019816F06AFAAC
:1034400000EBC00140F22060C2F2000000EB8100FE
:10345000006A8047FFE7FFE702B080BD82B08DF8C9
:1034600006008DF805100092009820B9FFE7FE20B5
:103470008DF8070012E000989DF8061001EBC102DC
:1034800040F22061C2F2000101EB82019DF80520AB
:1034900041F8220000208DF80700FFE79DF90700A2
:1034A00002B0704783B080B585B009930892079148
:1034B00003900020ADF8060007A80290039A029B33
:1034C00049F2FC60C2F2000040F2FF311FF024F923
:1034D000ADF80600BDF8060001280CDBFFE7BDF8DB
:1034E000061049F2FC60C2F2000000F02FF8002044
:1034F0008DF8130003E0FE208DF81300FFE79DF91F
:10350000130005B0BDE8804003B0704749F27C600D
:10351000C2F200000078704780B582B00090009839
:1035200020B9FFE7FE208DF807000BE0009841F27C
:10353000AC41C2F20001086000F05AFE00208DF894
:103540000700FFE79DF9070002B080BD80B582B09B
:103550000190ADF8021000208DF80100FFE70198FE
:10356000BDF8021000F06AFE48B1FFE79DF80100C7
:1035700001308DF801000A20FFF766FB00E005E04E
:10358000FFE79DF801000328E9DBFFE7002002B018
:1035900080BD0000FFE7FEE780B541F6C810C2F22B
:1035A000000005F09DFE80BD80B541F6C810C2F256
:1035B000000005F095FE80BD80B541F6F010C2F226
:1035C000000005F08DFE80BD80B541F6F010C2F21E
:1035D000000005F085FE80BD80B582B0002001901E
:1035E000FFF7EEFA019942F64C42C2F20002009255
:1035F00002F11C0305F06AFD0099019B41F2B04005
:10360000C2F200000068D0F804011A461AF092FDD8
:1036100002B080BD80B582B001200090FFF7D0FAE3
:10362000009942F67042C2F20002019202F11C03BC
:1036300005F04CFD019941F2B040C2F20000006873
:10364000D0F8040100231A461AF074FD02B080BDC0
:1036500083B0029001918DED000A0299002008715B
:1036600000980199086003B07047000082B0019093
:1036700000910098008800EE100AB8EEC00A9FED95
:10368000151A80EE010A019880ED000A0098408822
:1036900000EE100AB8EEC00A80EE010A019880ED33
:1036A000010A0098808800EE100AB8EEC00A80EE89
:1036B000010A019880ED020A0098C08800EE100A05
:1036C000B8EEC00A80EE010A019880ED030A02B04C
:1036D000704700BF0000C84280B586B005900491D5
:1036E00005988088ADF80E0042F69441C2F20001C0
:1036F00000914FF4C0600860002002908860C860AC
:1037000004220A619DF80F300A4602F8183F019220
:10371000BDF80E204A768876C8760498D0F8F00076
:103720004079FFF74DFA0099019A049B03F58073E5
:1037300005F00AFA029806B080BD000080B586B098
:103740000590049105984089ADF80E0042F6944129
:10375000C2F20001009140F2036008600020029074
:103760008860C86004220A619DF80F300A4602F89A
:10377000183F0192BDF80E204A768876C8760498E4
:10378000D0F8F0004079FFF71BFA0099019A049BEA
:1037900003F5807305F0D8F9029806B080BD0000EB
:1037A00080B584B0039042F69441C2F200010191C9
:1037B00040F2116008600020029088600222CA6016
:1037C00008610398D0F8F0004079FFF7F9F9019902
:1037D000039A02F5807301F1180205F0B5F9029819
:1037E00004B080BD80B584B0039042F69441C2F22B
:1037F0000001019140F21260086000200290886090
:103800000222CA6008610398D0F8F0004079FFF7FF
:10381000D7F90199039A02F5807301F1180205F0B6
:1038200093F9029804B080BD80B586B005900491EC
:103830000598C088ADF80E0042F69441C2F200012E
:10384000009140F201600860002002908860C8602A
:1038500004220A619DF80F300A4602F8183F0192CF
:10386000BDF80E204A768876C8760498D0F8F00025
:103870004079FFF7A5F90099019A049B03F580733D
:1038800005F062F9029806B080BD000080B586B0F0
:103890000590049105980089ADF80E0042F6944118
:1038A000C2F20001009140F2026008600020029024
:1038B0008860C86004220A619DF80F300A4602F849
:1038C000183F0192BDF80E204A768876C876049893
:1038D000D0F8F0004079FFF773F90099019A049B42
:1038E00003F5807305F030F9029806B080BD000042
:1038F00083B001900091019820B9FFE700208DF876
:103900000B000AE00198006800990840401AB0FADC
:1039100080F040098DF80B00FFE79DF80B0003B025
:103920007047000083B001900091019820B9FFE733
:10393000FE208DF80B0008E0009A0199086890437A
:10394000086000208DF80B00FFE79DF90B0003B025
:103950007047000082B000900098006846F60001B1
:10396000C4F20001884204D1FFE701208DF807006E
:1039700010E00098006846F20041C4F2000188425D
:1039800004D1FFE700208DF8070003E003208DF845
:103990000700FFE79DF8070002B0704780B592B0BE
:1039A00010900F91109820B9FFE7FE208DF8470086
:1039B0007DE042F26560C2F200000078C00720B1ED
:1039C000FFE7FD208DF8470071E01AF075FD43F226
:1039D0009841C2F20001086020B9FFE7FE208DF88F
:1039E000470064E020202421002204921AF022FBE8
:1039F0001099C1F804010F981099C1F8F00005A8BA
:103A000002902821FCF739FC04980A900590069052
:103A10000B90012103910C91079008900D910E21BC
:103A200001910E910990FFF7CBF8029905F0B0F9DA
:103A30000498FFF7C5F806F05DFA049843F2D952EE
:103A4000C0F600020621FFF7DBF80498FFF7B8F88C
:103A5000022105F03DF8019903980A910990FFF7BA
:103A6000AFF8029905F094F90398FFF7A9F806F06A
:103A700041FA039843F21562C0F600020821FFF7ED
:103A8000BFF80398FFF79CF8102105F021F803997F
:103A90000498109A41F2B043C2F200031A6042F255
:103AA0006562C2F2000211708DF84700FFE79DF9D0
:103AB000470012B080BD000080B590B08DF83E0088
:103AC0000E910D920E9820B9FFE7FE208DF83F0071
:103AD0003AE19DF83E000146079158B1FFE707988B
:103AE0000138022869D3FFE7079803380228C0F09D
:103AF000B58024E10E9890ED000A9FED951A20EE16
:103B0000010ABDEEC00A10EE100AADF832000E98A0
:103B100090ED010A20EE010ABDEEC00A10EE100A77
:103B2000ADF830000E9890ED020A20EE010ABDEECD
:103B3000C00A10EE100AADF82E000E9890ED030AA0
:103B400020EE010ABDEEC00A10EE100AADF82C00FE
:103B500042F69441C2F2000105914FF400700860F2
:103B600000208860C860082008619DF8332008465E
:103B700000F8182F0690BDF8320048769DF8310005
:103B80008876BDF83000C8769DF82F000877BDF81C
:103B90002E0048779DF82D008877BDF82C00C87757
:103BA0000D98D0F8F0000078FFF70AF80599069A0A
:103BB0000D9BF43304F0C8FFC2E00E9890ED040AA8
:103BC0009FED651A20EE010ABDEEC00A10EE100A44
:103BD000ADF82A000E9890ED050A20EE010ABDEE20
:103BE000C00A10EE100AADF8280042F69441C2F265
:103BF0000001039140F2FF20086000208860C86047
:103C000008220A619DF82B300A4602F8183F0492F8
:103C1000BDF82A204A769DF829208A76BDF828200A
:103C2000CA76087748778877C8770D98D0F8F0007B
:103C30004078FEF7C5FF0399049A0D9BF83304F012
:103C400083FF0D98D0F8F0008078FEF7B9FF039954
:103C5000049A0D9BF83304F077FF71E00E9890ED15
:103C6000070A9FED3B1A20EE010ABDEEC00A10EED6
:103C7000100AADF826000E9890ED080A20EE010A11
:103C8000BDEEC00A10EE100AADF824000E9890EDBB
:103C9000090A20EE010ABDEEC00A10EE100AADF8C6
:103CA00022000E9890ED0A0A9FED2A1A20EE010AD2
:103CB000BDEEC00A10EE100AADF8200042F69441A5
:103CC000C2F20001019140F2FF10086000208860FC
:103CD000C860082008619DF82720084600F8182FC2
:103CE0000290BDF8260048769DF825008876BDF83C
:103CF0002400C8769DF823000877BDF82200487795
:103D00009DF821008877BDF82000C8770D98D0F87D
:103D1000F000C078FEF754FF0199029A0D9BFC3326
:103D200004F012FF0D98D0F8F0000079FEF748FF7C
:103D30000199029A0D9BFC3304F006FF00E0FFE7B7
:103D400000208DF83F00FFE79DF93F0010B080BDD7
:103D50000000804600401C460060EA4683B00290A6
:103D6000019101980178407840EA0120ADF8020005
:103D700001980179407940EA0120ADF80000BDF8D2
:103D8000020000EE100AB8EEC00A9FED191A80EE8C
:103D9000010A9FED181A20EE010A029880ED000A30
:103DA00001988178C07840EA012000B200EE100A44
:103DB000B8EEC00A029880ED010ABDF9000000EBE0
:103DC0008000800000EE100AB8EEC00A9FED0A1ACB
:103DD00080EE010A029880ED020A0198807900EED7
:103DE000100AB8EE400A029880ED030A03B070474B
:103DF00000000046DB0FC9400000804680B586B059
:103E000004900391049820B9FFE7FE208DF8170075
:103E100085E1039820B9FFE7FE208DF817007EE1C9
:103E2000039800680190A0F2012004284FD3FFE717
:103E30000198A0F20520042860D3FFE70198A0F2C2
:103E40000920022872D3FFE7019840F2112188422D
:103E500000F08480FFE70198B0F5207F00F08A80B1
:103E6000FFE70198B0F5C06F00F09080FFE7019880
:103E700040F20161884200F09880FFE7019840F22B
:103E80000261884200F0A080FFE7019840F20361E0
:103E9000884200F0A880FFE70198B0F5C26F00F0FB
:103EA000B180FFE7019840F21161884200F0C380C1
:103EB000FFE7019840F21261884200F0E180FFE7DD
:103EC000019840F21361884200F0FF8022E10398DC
:103ED0000068A0F2012002900498029900EB011002
:103EE000043003991C31FFF739FF0299012000FAD1
:103EF00001F204990868104308600CE10398006817
:103F0000A0F2052002900298811D012000FA01F222
:103F100004990868104308600498029900EB0110A6
:103F2000643003991C31FFF719FFF4E0039800682F
:103F3000A0F2092002900298011D012000FA01F26E
:103F400004990868104308600498029900EB011076
:103F5000443003991C31FFF701FFDCE00499086845
:103F600040F4007008600498AC3003991C31FFF7EE
:103F70007DFBD0E00499086840F4806008600498F4
:103F8000E83003991C3100F0CFF8C4E00398017FBA
:103F9000407F40EA012142F2A060C2F200000180AD
:103FA00000880499A1F8BC00B5E00398017F407F28
:103FB00040EA012142F2A060C2F200004180408844
:103FC0000499A1F8BE00A6E00398017F407F40EA73
:103FD000012142F2A060C2F2000081808088049931
:103FE000A1F8C00097E00398017F407F40EA0121DB
:103FF00042F2A060C2F20000C180C0880499A1F81A
:10400000C20088E00398017F407F40EA012142F22C
:10401000A060C2F2000001810189049AA2F8C410D4
:1040200003998A7FC97F41EA02214181408904992D
:10403000A1F8C6006FE00398017F407F40EA0121AC
:1040400042F2A060C2F200000182018A049AA2F842
:10405000CC1003998A7FC97F41EA0221818181893D
:10406000049AA2F8C810039991F8202091F8211021
:1040700041EA0221C181C0890499A1F8CA004AE03D
:104080000398017F407F40EA012142F2A060C2F222
:104090000000C182C18A049AA2F8D21003998A7FD3
:1040A000C97F41EA02214182418A049AA2F8CE10D6
:1040B000039991F8202091F8211041EA0221818290
:1040C000808A0499A1F8D00025E00398017F407F01
:1040D00040EA012142F2A060C2F200000183018B9C
:1040E000049AA2F8D41003998A7FC97F41EA022179
:1040F0004183418B049AA2F8D610039991F82020AD
:1041000091F8211041EA02218183808B0499A1F862
:10411000D80000E0FFE700208DF81700FFE79DF9C9
:10412000170006B080BD000082B001900091009899
:10413000017842788078000440EA0220084400EECA
:10414000100AB8EEC00A9FED0A1A80EE010A019823
:1041500080ED000A0098C0780199087100990879EB
:10416000497940EA01200199C88002B0704700BF38
:1041700000007A4484B08DF80F000291ADF806205B
:104180009DF80F000146009123281DD80099DFE813
:1041900001F012131415161B1B1B1B1B1B1B1B1BD7
:1041A0001B1B1B1B1B1B1B1B1B1B1B1B1B1B1B1B5F
:1041B0001B1B1718191A08E007E006E005E004E0E9
:1041C00003E002E001E000E0FFE7002004B07047F8
:1041D0000020704780B541F26860C2F2000049F2E9
:1041E0007C61C2F2000116F0C3FC002080BD00001B
:1041F00080B541F26860C2F2000016F073FC002046
:1042000080BD000080B582B00190009141F2AC40C9
:10421000C2F20000006801211AF06EF8002002B01E
:1042200080BD000083B0029001918DF80320002032
:104230008DF802009DF9020003B0704780B586B08A
:104240000490ADF80E1000208DF80D0041F268606A
:10425000C2F20000D0F8BC0202900298D0F814021A
:1042600020B1FFE701208DF8170013E00499BDF895
:104270000E2041F26860C2F20000019016F092FC3C
:10428000019816F07DFD8DF80D009DF80D008DF85C
:104290001700FFE79DF8170006B080BD80B588B015
:1042A000069005918DF8132005989DF8131000F0E5
:1042B0008DF88DF8120005989DF8131000F078F82D
:1042C0008DF811009DF8120010280DD1FFE7069817
:1042D000007F00F001008DF810000598807A00F052
:1042E00001008DF80F0025E09DF8120011280DD176
:1042F000FFE70698407F00F001008DF81000059858
:10430000C07A00F001008DF80F0012E00698C08B13
:104310009DF81210C84000F001008DF810000598BB
:1043200040889DF81210C84000F001008DF80F0081
:10433000FFE7FFE79DF811000146029140B1FFE75A
:104340000298012817D0FFE70298022824D02AE01B
:104350009DF810100020C907019031B1FFE79DF8CA
:104360000F0080F001000190FFE7019800F00100CC
:104370008DF81F0017E09DF810100020C90700906D
:1043800021B9FFE79DF80F000090FFE7009800F0CB
:1043900001008DF81F0006E09DF8100000F00100FC
:1043A0008DF81F00FFE79DF81F0008B080BD0000DA
:1043B00082B001908DF80310019800699DF80310F8
:1043C00000EB4100007A02B07047000082B001901B
:1043D0008DF80310019800699DF8031000EB41006F
:1043E000407A02B07047000081B000900098407899
:1043F00000F0010001B0704783B001900091019876
:1044000020B9FFE7FF208DF80B000FE0009820B9DE
:10441000FFE7FF208DF80B0008E0019900200870ED
:104420000099019A11618DF80B00FFE79DF90B00CF
:1044300003B0704783B001908DF803109DF803001E
:10444000102807D1FFE70198007F00F001008DF8E8
:104450000B0015E09DF80300112807D1FFE7019834
:10446000407F00F001008DF80B0009E00198C08B3F
:104470009DF80310C84000F001008DF80B00FFE725
:104480009DF80B0003B0704784B0029001918DED50
:10449000000A029820B9FFE7FF208DF80F0025E001
:1044A000019820B9FFE7FF208DF80F001EE0029869
:1044B000006801998862029840680199C862029870
:1044C000007EC00748B1FFE70199022081F834005F
:1044D0000199012081F8360004E00199012081F85A
:1044E0003400FFE700208DF80F00FFE79DF90F0073
:1044F00004B0704780B584B0029001918DED000A40
:10450000029820B9FFE7FF208DF80F0056E00198D0
:1045100020B9FFE7FF208DF80F004FE0029804213B
:10452000FFF788FF80B1FFE702980521FFF782FFC0
:1045300050B1FFE702980621FFF77CFF20B1FFE7AB
:10454000019901200870FFE702980421FFF772FF2C
:1045500080B1FFE702980521FFF76CFF50B1FFE73C
:1045600002980721FFF766FF20B1FFE701990020BD
:104570000870FFE70298407D20B1FFE70298007DB8
:1045800020B9FFE7019800F021FA13E001980078C4
:10459000C00738B1FFE7029801999DED000A00F0CD
:1045A00011F806E0029801999DED000A00F08AF9E1
:1045B000FFE7FFE700208DF80F00FFE79DF90F00F0
:1045C00004B080BD80B584B0039002918DED010AE6
:1045D0000299012081F824000398B0F9160000EE3A
:1045E000100AB8EEC00A9DED011A20EE010A0298E9
:1045F000016991ED001A20EE010A80ED0A0A039884
:10460000B0F9180000EE100AB8EEC00A9DED011ACC
:1046100020EE010A0298016991ED001A20EE010ACC
:1046200080ED0B0A02980022C26102988261029812
:1046300080F8382003980299FFF730FE58B1FFE761
:104640000298016991ED091A90ED070A30EE010A0E
:1046500080ED070AFFE7039802990122FFF71EFE8B
:1046600058B1FFE70298016991ED091A90ED070A28
:1046700030EE410A80ED070AFFE703980299022213
:10468000FFF70CFE58B1FFE70298016991ED091A96
:1046900090ED060A30EE410A80ED060AFFE7039826
:1046A00002990322FFF7FAFD58B1FFE7029801696A
:1046B00091ED091A90ED060A30EE010A80ED060A26
:1046C000FFE7039802990422FFF7E8FDA8B1FFE78E
:1046D0000298016991ED0A1A90ED060A20EE010A8E
:1046E00080ED060A0298016991ED0A1A90ED070A19
:1046F00020EE010A80ED070AFFE7039802990522E0
:10470000FFF7CCFDA8B1FFE70298016991ED0B1A04
:1047100090ED060A20EE010A80ED060A0298016972
:1047200091ED0B1A90ED070A20EE010A80ED070AC1
:10473000FFE7039802990622FFF7B0FD48B1FFE7B3
:104740000299022081F834000299012081F8360094
:1047500008E00299022081F834000299002081F8D3
:104760003600FFE7039802990722FFF797FDB0B1E3
:10477000FFE7029991F83500013081F83500029980
:1047800091F835004AF6AB22CAF6AA22A0FB023203
:10479000520802EB4202801A81F83500FFE70398C5
:1047A00002990B22FFF77AFD38B1FFE70299042046
:1047B0000875029902204875FFE7039802990A22BA
:1047C000FFF76CFD40B1FFE7029991F83720012017
:1047D000904381F83700FFE7039802990822FFF71A
:1047E0005DFD20B3FFE70298007B02280BD1FFE7B5
:1047F00002983930042100F0F7F80299002048703F
:104800000299087312E00298007B012801D1FFE7AA
:104810000BE002983930032100F0E6F802990220FB
:104820000873029901204870FFE7FFE7FFE703984C
:1048300002990922FFF732FDD8B1FFE70298007B09
:1048400001280BD1FFE702990020487002990873F4
:1048500002983930022100F0C7F809E002980121DE
:104860000173029841700298393000F0BDF8FFE7FB
:1048700003E0029900204870FFE7039802990C2298
:10488000FFF70CFD28B1FFE70299012081F83800FD
:10489000FFE7039802990D22FFF700FD20B1FFE723
:1048A000029902200875FFE70398C08B029948809F
:1048B0000299039AD2F81600D2F81A208A6048604A
:1048C00004B080BD85B0049003918DED020A049878
:1048D000407D01460191032817D80199DFE801F0D6
:1048E00011020A060399012008750EE003990220BF
:1048F00008750AE00399042008750399002048759B
:1049000003E0039900200875FFE70498007D014645
:104910000091032831D80099DFE801F02702170A37
:104920000399012081F82400039981F8340024E0E0
:104930000399012081F824000399002081F83600B2
:104940000399022081F8340017E00399012081F8CF
:104950002400039A022182F83410039A002182F87D
:104960003510039981F8360007E00399002081F89B
:104970002400039981F83400FFE704980068039944
:104980008861049840680399C861049890ED020A10
:104990009DED021A20EE010A0398016991ED011ABA
:1049A00020EE010A80ED0A0A049890ED030A9DEDBD
:1049B000021A20EE010A0398016991ED011A20EE16
:1049C000010A80ED0B0A05B07047000081B000902D
:1049D000009900200875009981F82400009981F859
:1049E000340001B07047000083B001908DF80310CF
:1049F000019820B9FFE7FF208DF80B001BE001981C
:104A0000C078022806DCFFE70198C078B0F1FF3FCC
:104A100004DCFFE7FF208DF80B000CE09DF803009D
:104A20000199CA7888540199C8780130C87000206B
:104A30008DF80B00FFE79DF90B0003B070470000F5
:104A400081B0ADF802008DF80110BDF802109DF89C
:104A500001004840C2B244F6A060C0F6020030F83F
:104A6000120080EA112001B07047000080B584B0C8
:104A700003900291ADF80620FFE70298411E0291D3
:104A800058B1FFE7BDF8060003994A1C0392097864
:104A9000FFF7D6FFADF80600EFE7BDF8060004B05B
:104AA00080BD000080B584B002900191019801287A
:104AB00004D8FFE700208DF80F001BE00298019951
:104AC00002394FF6FF72FFF7D1FFADF80200BDF8D3
:104AD0000200029A019901F001031A4421F0010138
:104AE000114431F8021C401AB0FA80F040098DF8E8
:104AF0000F00FFE79DF80F0004B080BD83B0029067
:104B000001918DF80320FFE70198411E019178B1D2
:104B1000FFE79DF8030002994A1C02920978414080
:104B200045F2A000C0F60200405C8DF80300EBE700
:104B30009DF8030003B0704780B584B002900191E6
:104B40000198012804D8FFE700208DF80F0015E038
:104B5000029801990139FF22FFF7D0FF8DF8030079
:104B60009DF80300029A0199114411F8011C401AA2
:104B7000B0FA80F040098DF80F00FFE79DF80F00B4
:104B800004B080BD85B002A900910146009880ED77
:104B9000010AC0ED000A8DF8071090ED010AB5EE8C
:104BA000400AF1EE10FA03D1FFE7002004906DE017
:104BB0009DF80700C007A0B3FFE7009890ED010A39
:104BC000B2EE0E1AB4EE410AF1EE10FA06D1FFE78A
:104BD0004FF20000C4F29150049057E0009890ED1D
:104BE000010AB3EE021AB4EE410AF1EE10FA06D150
:104BF000FFE748F20000C4F2A250049046E000989B
:104C000090ED010AB3EE0E1AB4EE410AF1EE10FA7D
:104C100006D1FFE74BF20000C4F2E550049035E006
:104C200022E0009890ED010AB2EE041AB4EE410AB7
:104C3000F1EE10FA06D1FFE741F20000C4F28B500A
:104C4000049023E0009890ED010AB3EE001AB4EE50
:104C5000410AF1EE10FA06D1FFE744F20000C4F277
:104C6000B550049012E0FFE7009890ED010A9FED27
:104C70000A1A20EE010A90ED001A9FED082A21EE93
:104C8000021A80EE010A80ED020AFFE7009890ED1B
:104C9000020A05B0704700BF00007042DB0FC94038
:104CA00080B584B0039002910298FEF779FD01204F
:104CB000019019F025F80298FEF794FD019819F07B
:104CC0001FF803980299FEF707FD019819F018F8EC
:104CD00003980299FEF7A8FD019819F011F80398BE
:104CE0000299FEF7D3FD019819F00AF8039802998A
:104CF000FEF724FD04B080BD81B000900099022031
:104D00008880009941F28830C88000994FF416607D
:104D1000088100996420488101B0704780B584B053
:104D200003900291019202980078012805D0FFE7D4
:104D300002988068019908600CE0029890ED010AE1
:104D4000D0ED020A90ED031A0FF044FD019880EDBA
:104D5000000AFFE70399012008710398B0F92A00BF
:104D600000EE100AB8EEC00A0398B0F9240001EE74
:104D7000100AF8EEC10AB2EE081A00F0B9F803986A
:104D800080ED000A04B080BD82B0019000910198CE
:104D9000006800990860019800790099087102B0D4
:104DA0007047000084B08DED030A9DED030A20EEEC
:104DB000000A8DED010A9DED010A9DED031A20EE1A
:104DC000010A8DED000A9DED030A9FED3E1AB4EE37
:104DD000410AF1EE10FA03DAFFE70020029053E0F7
:104DE0009DED030A9FED381AB4EE410AF1EE10FA78
:104DF0001DDAFFE79DED000A9FED391A20EE010A4A
:104E00009DED011A9FED372A21EE021A30EE010ABC
:104E10009DED031A9FED342A21EE021A30EE010AAD
:104E20009FED321A30EE010A8DED020A2BE09DED66
:104E3000030A9FED261AB4EE410AF1EE10FA1DDACC
:104E4000FFE79DED000A9FED221A20EE010A9DED7D
:104E5000011A9FED202A21EE021A30EE010A9DED83
:104E6000031A9FED1D2A21EE021A30EE010A9FED72
:104E70001B1A30EE010A8DED020A03E04FF07E505E
:104E80000290FFE7FFE7FFE79DED020AB5EE400A5B
:104E9000F1EE10FA03DAFFE7002002900EE09DED3C
:104EA000020AB7EE001AB4EE410AF1EE10FA04DD80
:104EB000FFE74FF07E500290FFE7FFE79DED020A0B
:104EC00004B0704700009C413333AF410000CC4137
:104ED00061E0B93C46B6D3BF295C21423333A4C359
:104EE0001399B93BFB5CADBEE17AD84014AE34C235
:104EF00084B08DED030ACDED020A8DED011A9DED12
:104F0000030A9DED012A30EE420A9DED021A31EEB0
:104F1000421A80EE010A8DED000A9DED000AB5EE01
:104F2000400AF1EE10FA03DAFFE7002000900EE0ED
:104F30009DED000AB7EE001AB4EE410AF1EE10FA48
:104F400004DDFFE74FF07E500090FFE7FFE79DEDA7
:104F5000000A04B07047000080B588B08DED070AE4
:104F6000CDED060A05909DED050AB8EE400A10EE5B
:104F7000100AFBF70FFB41EC100B9FED2B1B53ECC2
:104F8000112B51EC100BFBF763FA41EC100B51ECB9
:104F9000100BFBF712FB00EE100A1EF005FA9FED56
:104FA000261A20EE010A10EE100AFBF7F3FA41EC84
:104FB000100B51EC100B9FED1E0B52EC103BD20F5F
:104FC00062F3DF7141EC100B8DED020B0798FBF7DC
:104FD000E1FA9DED021B41EC100B51EC110B53EC6F
:104FE000102BFBF78EF941EC100B51EC100BFBF77B
:104FF000E4FA04909DED040A9FED101AB4EE410A04
:10500000F1EE10FA05DDFFE79DED060A8DED010AD0
:1050100004E09DED040A8DED010AFFE79DED010A14
:1050200008B080BD00BF00BFFCA9F1D24D62503F67
:105030000000000000000000CDCC4C3ECDCC4C3F29
:1050400080B58EB007AB05930C900B910A920C982B
:1050500020B9FFE7FE208DF8370067E10B9820B9F3
:10506000FFE7FE208DF8370060E10A990C9802688E
:10507000891A00EE101AB8EE400A9FEDAE1A80EEC3
:10508000010A80ED010A0A980C9908600C980B99A6
:1050900009780A9A00F02EFB0C98007C01460491D6
:1050A00000B3FFE7049801280DD0FFE70498023809
:1050B000032817D3FFE7049805280AD0FFE70498D0
:1050C00006280FD04CE00C99002048610C998861AB
:1050D00046E00B9840680C9948610B9840680C9921
:1050E00088613DE005980C9991ED080AC96891ED39
:1050F000001A30EE410A80ED020A90ED020A1EF01D
:105100000FF8059880ED010A90ED020A1EF04CF9A7
:10511000059880ED000A90ED010A0B9991ED011AB6
:1051200091ED022A20EE010A90ED001A21EE021AFA
:1051300030EE410A0C9981ED050A90ED000A0B99B9
:1051400091ED011A91ED022A20EE010A90ED011A6B
:1051500021EE021A30EE010A0C9880ED060AFFE7F4
:105160000C98007C01460391062848D80399DFE893
:1051700001F00404081A300408000C990020C861EA
:105180003DE00C9901F13800CA6892ED000AD1EDBA
:10519000011AD1ED080A9FED6B1A0FF07FF80C98F9
:1051A00080ED070A2BE00C9901F13800CA6892EDF6
:1051B000000A9FED631A30EE010AD1ED011AD1ED1C
:1051C000080A9FED601A0FF069F80C9880ED070A45
:1051D00015E00C9890ED0B0A8DED020A0A989FEDF0
:1051E000560ADFED560AFFF7B7FEB0EE401A9DED06
:1051F000020A20EE010A0C9880ED070AFFE70C9BDB
:1052000003F1120003F114011A6B93F911309FEDB1
:105210004E0A0EF0C7FC00208DF81B00FFE79DF83A
:105220001B000C9991F9111088427BDAFFE70C986A
:10523000416A406F9DF81B2000EB421001EB820198
:1052400091ED000A0DF01AFC0C98406A9DF81B10B5
:1052500000EB810080ED000A0C98007C0146019172
:10526000E0B3FFE701980138052804D3FFE7019870
:10527000062821D03AE00C99486B9DF81B30C3EB0F
:10528000031200EB82000A6B02EB830292ED000A2C
:105290004A6A02EB8302D2ED000AD1ED011A9FEDBA
:1052A000291A0EF0FBFF0C98C06F9DF81B1000EB45
:1052B000810080ED000A19E00C989DF81B10026B2C
:1052C000C06F02EB810292ED000A9FED201A80EE82
:1052D000010A00EB810080ED000A07E00C98C16F25
:1052E0009DF81B20002041F82200FFE70C999DF853
:1052F0001B20886FC96F00EB421001EB820191ED1A
:10530000000A0DF0BBFB0C98C06F9DF81B1000EB62
:10531000810080ED000AFFE79DF81B0001308DF849
:105320001B007CE700208DF83700FFE79DF9370070
:105330000EB080BD00007A449A99193FCDCC4C3F05
:10534000AB611C3F0000000000C0DA4500A00C4625
:1053500083B00290019100208DF80300FFE79DF8D3
:105360000300029991F91110884210DAFFE70298C0
:10537000C06F9DF8032050F82200019941F82200E7
:10538000FFE79DF8030001308DF80300E7E703B065
:105390007047000082B0019000910198007C009954
:1053A0000870019890ED080AC06890ED001A30EE80
:1053B000410A009880ED010A02B0704780B58AB0BA
:1053C00005AB03930346039808930791069280ED7B
:1053D000000A089820B9FFE7FE208DF827001CE19D
:1053E0000798089988600899002008740698089919
:1053F000C860079890F84C00C00728B1FFE70898EC
:10540000C06800F0DBFAFFE7089880680078014682
:105410000291062832D80299DFE801F0040B121835
:105420001F2C250008990420487400208DF81300D3
:1054300024E008990420487401208DF813001DE031
:105440000899022048748DF8130017E00899042089
:10545000487403208DF8130010E008990420487464
:105460008DF813000AE008990120487405208DF892
:10547000130003E0FC208DF82700CEE0089890F997
:1054800011008000FDF76CFE089948620898406A98
:1054900008B9FFE7A5E0089890F911008000FDF732
:1054A0005FFE089988620898806A08B9FFE798E06B
:1054B000089890F911008000FDF752FE08990863E2
:1054C0000898006B08B9FFE78BE0089890F9110085
:1054D000C0EB00108000FDF743FE08994863089870
:1054E000406B08B9FFE77CE0089890F91100800054
:1054F000FDF736FE0899C8670898C06F08B9FFE73E
:105500006FE0089890F911004001FDF729FE089915
:1055100048670898406F08B9FFE762E0089890F97B
:1055200011004001FDF71CFE089988670898806FFC
:1055300008B9FFE755E000208DF81200FFE79DF85D
:105540001200089991F91110884233DAFFE7039AA3
:1055500008988168406B9DF81230C3EB031300EB91
:10556000830092ED000A0A1D00210FF00FF8039A44
:1055700008988168406F9DF8123000EB431092ED5F
:10558000000AD1ED110A0DF0D5FA039A0898816846
:10559000806F9DF8123000EB431092ED000AD1EDC0
:1055A000120A0DF0C7FAFFE79DF8120001308DF8DE
:1055B0001200C4E7039A089901F1380092ED000A3D
:1055C000896801F12402002101910EF0DFFF0898A3
:1055D00012309DF813100EF037FC01988DF827005B
:1055E0001BE00898406AFDF7CFFB0898006BFDF7B9
:1055F000CBFB0898406BFDF7C7FB0898C06FFDF721
:10560000C3FB0898406FFDF7BFFB0898806FFDF75C
:10561000BBFBFE208DF82700FFE79DF927000AB0AD
:1056200080BD000080B584B00390029101920020FB
:10563000009001980078012805D0FFE70020C4F20F
:10564000FA40009042E002980079012833D1FFE748
:10565000029890ED000A9FED231AB4EE410AF1EE94
:1056600010FA28DDFFE7029890ED000AB7EE001A65
:10567000B4EE410AF1EE10FA05DDFFE70020CBF6AB
:105680008070009016E0019890ED010A029890ED6C
:10569000001A9FED152A31EE021A9FED142A81EEB1
:1056A000021A9FED132A21EE021A30EE010A8DED47
:1056B000000AFFE709E0019890ED010AD0ED020A27
:1056C0000FF038F98DED000AFFE7FFE79DED000AC6
:1056D000039A516AD06F92F911200FF0B7F80020A9
:1056E00004B080BD9A99993E9A9999BE3333333F5D
:1056F0000000C84280B586B004908DF80F10029269
:10570000049820B9FFE7FE208DF8170066E09DF8A9
:105710000F000499097C884204D1FFE700208DF82E
:1057200017005BE09DF80F0004281CD1FFE70498E8
:10573000007C042817D0FFE70298FAF77DFDFAF7FE
:1057400071FD00EBD07121F00101411A0120002907
:1057500018BF4FF0FF3000EE100AB8EEC00A0498F0
:1057600080ED0B0AFFE700208DF80700FFE79DF8AA
:105770000700049991F91110884227DAFFE704988D
:10578000406B9DF80710C1EB011100EB81000EF09A
:10579000C9FF0498406F9DF8071000EB41109FED82
:1057A000110A8DED000A0DF063FA9DED000A0498D0
:1057B000806F9DF8071000EB41100DF059FAFFE7DC
:1057C0009DF8070001308DF80700D0E79DF80F0025
:1057D0000499087400208DF81700FFE79DF9170061
:1057E00006B080BD0000000084B0029001910298D4
:1057F00020B9FFE7FE208DF80F0048E0019820B99E
:10580000FFE7FE208DF80F0041E00298806890F8D5
:105810004C00C00758B1FFE7019890ED111A9FEDB9
:105820001E0A30EE410A029880ED080A04E0019851
:10583000406C02990862FFE700208DF80300FFE743
:105840009DF80300029991F9111088421BDAFFE7D5
:1058500001989DF8032000EB021080680299496AC4
:1058600041F8220001989DF8032000EB0210C06867
:105870000299896A41F82200FFE79DF80300013090
:105880008DF80300DCE700208DF80F00FFE79DF99D
:105890000F0004B0704700BFDB0FC94084B0039015
:1058A0008DED020ACDED010A039890ED000A9DED01
:1058B000021A30EE010A8DED000A9DED010AB5EEE7
:1058C000400AF1EE10FA26DDFFE79DED000A9DED9E
:1058D000011AB4EE410AF1EE10FA09DBFFE79DED83
:1058E000011A9DED000A30EE410A8DED000A11E02B
:1058F0009DED000AB5EE400AF1EE10FA09DAFFE775
:105900009DED011A9DED000A30EE010A8DED000AB1
:10591000FFE7FFE7FFE700980399086004B07047CE
:1059200085B08DED040ACDED030A8DED021A9DEDD3
:10593000040A9DED031A30EE410A8DED010A9DED3A
:10594000020AB5EE400AF1EE10FA32DDFFE79DEDF6
:10595000020AB0EE001A80EE010A8DED000A9DEDFC
:10596000010A9DED001AB4EE410AF1EE10FA09DDCC
:10597000FFE79DED021A9DED010A30EE410A8DED23
:10598000010A15E09DED010A9DED001AB1EE411AE4
:10599000B4EE410AF1EE10FA09DAFFE79DED021AC2
:1059A0009DED010A30EE010A8DED010AFFE7FFE7E8
:1059B000FFE79DED010A05B07047000081B000903F
:1059C000009890ED001A9FED040A30EE410A80ED38
:1059D000000A01B0704700BFDB0FC94083B00290DE
:1059E0008DED010ACDED000A029890ED000A9DEDC3
:1059F000001AB4EE410AF1EE10FA04DDFFE7009858
:105A000002990860FFE7029890ED000A9DED011AE7
:105A1000B4EE410AF1EE10FA04DAFFE701980299B8
:105A20000860FFE703B0704780B5B4B032903191A1
:105A30003092329818B9FFE700203390FDE1319899
:105A4000013831900020ADF84E0040F2C040C2F263
:105A50000000007801461291072800F2C8811299CF
:105A6000DFE811F008001A002C00970036016101F0
:105A7000A301B4013298319945F69C62C0F6020246
:105A80001CF01CFE40F2C041C2F200010878013057
:105A9000087001203390D0E13298319945F6CA520E
:105AA000C0F602021CF00AFE40F2C041C2F2000140
:105AB00008780130087001203390BEE143F2DC2009
:105AC000C2F200001190C06818F0E6FD1198806BDA
:105AD00014A90022052318F04DFAC0B1FFE732984F
:105AE000319945F69C52C0F602021CF0E7FD40F2E7
:105AF000C041C2F200010720087043F2DC20C2F26C
:105B00000000C06818F0A8FD0120339095E143F231
:105B1000DC20C2F20000C06818F09EFD14A8FCF75B
:105B2000F1FC90B1FFE73298319945F67262C0F608
:105B300002021CF0C3FD40F2C041C2F2000108782D
:105B4000013008700120339077E140F2C140C2F289
:105B50000000017801310170007802280FDCFFE7B6
:105B60003298319945F6E852C0F602021CF0A6FDC3
:105B700040F2C041C2F200010120087006E040F28C
:105B8000C041C2F2000107200870FFE701203390F6
:105B900053E13298319945F6BD62C0F602021CF01D
:105BA0008DFD17A8109000F01BFF1098002129917F
:105BB0002A912B9100F0D2FFFFE7BDF84E00B0F51F
:105BC0007A7F4BDAFFE743F2DC20C2F20000806B01
:105BD00014A90F910022052318F0CCF901460F9863
:105BE000B1FA81F149098DF84D10FCF78BFC8DF865
:105BF0004C009DF84D00C00778B3FFE79DF84C00BE
:105C0000C00750B3FFE79DED141A40F2C440C2F242
:105C1000000090ED000A30EE010A80ED000A9DEDD3
:105C2000151A40F2C840C2F2000090ED000A30EEB2
:105C3000010A80ED000A9DED161A40F2CC40C2F236
:105C4000000090ED000A30EE010A80ED000ABDF878
:105C50004E000130ADF84E00FFE7AEE7BDF84E0054
:105C600000EE100AB8EE401A40F2C440C2F2000042
:105C700090ED000A80EE010A80ED000ABDF84E00AA
:105C800000EE100AB8EE401A40F2C840C2F200001E
:105C900090ED000A80EE010A80ED000ABDF84E008A
:105CA00000EE100AB8EE401A40F2CC40C2F20000FA
:105CB00090ED000A80EE010A80ED000A40F2C0413A
:105CC000C2F2000108780130087001203390B4E07E
:105CD0003298319945F64462C0F602021CF0EEFC9F
:105CE00017A80E9000F07CFE0E9840F2C441C2F25C
:105CF00000010968299140F2C841C2F20001096817
:105D00002A9140F2CC41C2F2000109682B9100F0C7
:105D100025FF40F2C041C2F200010878013008704E
:105D20000120339089E032980C9031980D9040F228
:105D3000C440C2F200000068FAF72CFC41EC100BE2
:105D40008DED0A0B40F2C840C2F200000068FAF77D
:105D500021FC41EC100B8DED080B40F2CC40C2F25F
:105D600000000068FAF716FC9DED081B9DED0A0B7C
:105D700002460C980B460D9943EC122B6A4682EDB5
:105D8000042B82ED021B82ED000B45F60072C0F67B
:105D900002021CF093FC40F2C041C2F200010878FC
:105DA000013008700120339047E03298319945F670
:105DB0003162C0F602021CF081FC40F2C041C2F226
:105DC0000001082008700120339036E032983199A4
:105DD00045F6B552C0F602021CF070FC40F2C0411C
:105DE000C2F20001082008700120339025E040F243
:105DF000C441C2F2000100200790086040F2C8418F
:105E0000C2F20001086040F2CC41C2F20001086019
:105E100040F2C141C2F2000108703298319945F652
:105E2000D072C0F602021CF049FC079840F2C04153
:105E3000C2F2000108703390FFE7339834B080BDA0
:105E400080B5B0B02E902D912C922E9818B9FFE706
:105E500000202F9060E22D9801382D902C98012180
:105E60002BAA01F081FC28902C9802212AAA01F08B
:105E70007BFC27902C98032129AA01F075FC269021
:105E800028982B9A45F2F361C0F60201FAF72AFA34
:105E9000A0B9FFE72E982D9946F21C12C0F6020217
:105EA00045F6A313C0F602031CF008FC40F2D041F3
:105EB000C2F20001002008702F902DE228982B9A42
:105EC00046F23A11C0F60201FAF70CFA00285BD14B
:105ED000FFE7279818B9FFE7269808B1FFE70BE21C
:105EE00040F2D040C2F20000007801460A9120B191
:105EF000FFE70A98012810D045E02E982D9946F228
:105F00004F02C0F602021CF0D9FB40F2D041C2F2AF
:105F10000001012008702F90FEE10DA80990642176
:105F2000FAF7ABF945F28F70C0F60200089000F066
:105F30009DFD189045F29270C0F60200069000F0A8
:105F4000D7FD069A014609981791142107911CF074
:105F5000B5FB0799089A099814301CF0AFFB099813
:105F600000F0FCFD2E982D9946F20B02C0F60202BD
:105F70001CF0A4FB40F2D041C2F2000102200870E4
:105F800001202F90C8E19DE128982B9A46F24B11F1
:105F9000C0F60201FAF7A6F9002840F0CF80FFE72B
:105FA000279818B1FFE7269808B1FFE7A4E12798E2
:105FB0002A9A46F24511C0F60201FAF793F9002831
:105FC00057D1FFE700F088FD0C9040F2D040C2F2BC
:105FD000000000780146059120B1FFE705980128EF
:105FE00010D045E02E982D9946F2BA02C0F6020272
:105FF0001CF064FB40F2D041C2F2000101200870A5
:106000002F9089E10C9840F2D141C2F20001097849
:1060100050F83100E0B1FFE72E982D990C9A40F22C
:10602000D143C2F2000304931B7852F8333046F296
:106030001812C0F602021CF041FB049908780130E6
:10604000087040F2D041C2F20001012008700CE05B
:1060500040F2D141C2F200010020087040F2D0416C
:10606000C2F2000102200870FFE701202F9053E1E7
:1060700063E027982A9A46F23F11C0F60201FAF728
:1060800031F9002857D1FFE700F02CFD0B9040F2CA
:10609000D040C2F2000000780146039120B1FFE732
:1060A0000398012810D045E02E982D9946F2D10290
:1060B000C0F602021CF002FB40F2D041C2F2000125
:1060C000012008702F9027E10B9840F2D141C2F2D5
:1060D0000001097850F83100E0B1FFE72E982D99C2
:1060E0000B9A40F2D143C2F2000302931B7852F89C
:1060F000333046F21812C0F602021CF0DFFA0299A1
:1061000008780130087040F2D041C2F2000101204D
:1061100008700CE040F2D141C2F20001002008708A
:1061200040F2D041C2F2000102200870FFE70120D6
:106130002F90F1E000E0DFE0FFE7C2E028982B9A23
:1061400046F22511C0F60201FAF7CCF8002840F01B
:10615000B780FFE7279818B1FFE7269808B9FFE74F
:10616000CAE027982A9A46F23F11C0F60201FAF7D0
:10617000B9F800283ED1FFE740F2D040C2F200005B
:106180000078B0BBFFE70DA800F02AFC269800F0CD
:10619000AFFC88B9FFE72E982D9946F21302C0F69E
:1061A00002021CF08BFA40F2D041C2F20001022040
:1061B000087001202F90AFE02E982D9945F6D372EC
:1061C000C0F602021CF07AFA269B46F21C12C0F6B8
:1061D00002020DA8019014211CF070FA019800F041
:1061E000BDFC40F2D041C2F20001012008702F90A6
:1061F00092E04BE027982A9A46F24511C0F6020138
:10620000FAF770F800283FD1FFE740F2D040C2F221
:1062100000000078B8BBFFE70DA800F0E1FB26986E
:1062200000F024FC88B9FFE72E982D9946F2A202CF
:10623000C0F602021CF042FA40F2D041C2F2000164
:106240000220087001202F9066E02E982D9945F6C7
:10625000D372C0F602021CF031FA0DA8009014307F
:10626000269B46F21C12C0F6020214211CF026FAEC
:10627000009800F073FC40F2D041C2F2000101200E
:1062800008702F9048E000E036E0FFE740F2D04091
:10629000C2F200000078012811D1FFE72E982D9955
:1062A00046F27502C0F602021CF008FA40F2D04134
:1062B000C2F200010220087001202F902CE0FFE7BD
:1062C000FFE7FFE7FFE740F2D040C2F200000078AE
:1062D000022810D1FFE72E982D9945F2EE62C0F604
:1062E00002021CF0EBF940F2D041C2F200010020A2
:1062F00008702F9010E0FFE72E982D9945F63D523B
:10630000C0F602021CF0DAF940F2D041C2F20001FC
:10631000002008702F90FFE72F9830B080BD00005C
:1063200080B588B0069005910492069818B9FFE7E9
:10633000002007908DE005980138059042F2112069
:10634000ADF80E00BDF80E00ADF80C009DF80E0083
:106350009DF80F1040EA0120ADF80A0040F2D2404B
:10636000C2F20000007801460191032861D801992A
:10637000DFE801F00214283C0698059945F6BD7245
:10638000C0F602021CF09AF940F2D241C2F20001BA
:10639000087801300870012007905AE006980599A6
:1063A000BDF80C3045F69072C0F602021CF086F97A
:1063B00040F2D241C2F20001087801300870012099
:1063C000079046E006980599BDF80A3045F66372D5
:1063D000C0F602021CF072F940F2D241C2F2000192
:1063E0000878013008700120079032E0BDF80C00F9
:1063F000BDF80A10884209D1FFE70698059945F6CD
:106400004B72C0F602021CF059F908E00698059993
:1064100045F63E72C0F602021CF050F9FFE740F26A
:10642000D241C2F2000108780130087001200790C3
:106430000FE00698059945F6D072C0F602021CF0EE
:106440003DF940F2D241C2F20001002008700790ED
:10645000FFE7079808B080BD80B5E8B06690659109
:106460006492669818B9FFE700206790C9E06598C4
:106470000138659040F2D340C2F200000078014636
:106480000891042800F2AD800899DFE801F00324A8
:106490007788990009A800F0A3FA66980690659895
:1064A00007902198FAF776F8024606980B46079966
:1064B00043EC102B6A4682ED000B45F62E72C0F6B7
:1064C00002021CF0FBF840F2D341C2F200010120AD
:1064D0000870679095E043F2DC20C2F2000005905E
:1064E000C06818F0D9F80598006F22A900220A2385
:1064F00017F040FD80B1FFE743F2DC20C2F200005C
:10650000C06818F0A9F840F2D341C2F2000103209C
:1065100008700120679074E009A8029000F060FA0A
:1065200043F2DC20C2F20000C06818F095F802982F
:106530003799219100F012FB029800F051FA669809
:106540000390659804902198FAF724F8024603987E
:106550000B46049943EC102B6A4682ED000B45F67E
:10656000FE72C0F602021CF0A9F840F2D341C2F25A
:106570000001022008700120679042E0669865994A
:1065800046F27502C0F602021CF098F840F2D341C0
:10659000C2F20001052008700120679031E0669882
:1065A000659945F66D52C0F602021CF087F840F27C
:1065B000D341C2F20001052008700120679020E05D
:1065C0006698659946F22B02C0F602021CF076F836
:1065D00040F2D341C2F2000105200870012067900B
:1065E0000FE06698659945F6D072C0F602021CF07D
:1065F00065F840F2D341C2F20001002008706790B4
:10660000FFE7679868B080BD80B5F2B070906F9179
:106610006E92709818B9FFE700207190C2E06F98F1
:1066200001386F9040F2D440C2F200000078014679
:10663000129148B1FFE71298012817D0FFE712988E
:10664000022800F08E809DE070986F9945F6D76221
:10665000C0F602021CF032F840F2D441C2F200014E
:10666000087801300870012071909BE013A800F0B9
:10667000B7F943F2DC20C2F200001190C06818F0B4
:106680000BF81198006F2CA90022052317F072FC5B
:10669000C0B1FFE770986F9945F68152C0F60202CB
:1066A0001CF00CF840F2D441C2F200010220087044
:1066B00043F2DC20C2F20000C06817F0CDFF0120D9
:1066C00071906FE043F2DC20C2F20000C06817F066
:1066D000C3FF3D9828904198299013A800F03EFAF6
:1066E00070980F906F9810902898299906912A9980
:1066F0000891F9F74FFF0246069807920A46079954
:1067000042EC101B8DED0C0BF9F744FF0246089884
:1067100009920A46099942EC101B8DED0A0BF9F714
:1067200039FF9DED0A1B9DED0C0B02460F980B46A1
:10673000109943EC122B6A4682ED042B82ED021B6A
:1067400082ED000B45F6DE72C0F602021BF0B6FFCA
:1067500040F2D441C2F20001032008700120719080
:1067600020E070986F9945F6B552C0F602021BF012
:10677000A5FF40F2D441C2F20001032008700120BD
:1067800071900FE070986F9945F6D072C0F60202D2
:106790001BF094FF40F2D441C2F2000100200870C7
:1067A0007190FFE7719872B080BD000080B596B01F
:1067B000149013911292149818B9FFE700201590C5
:1067C0000AE113980138139040F2D540C2F200005C
:1067D000007801460A91092800F2EE800A99DFE864
:1067E00001F00517243643557385BCCE1498139ACF
:1067F00045F6A021C0F60201F9F74AFD40F2D54165
:10680000C2F2000108780130087001201590E3E021
:1068100014981AF015F840F2D541C2F20001087838
:106820000130087001201590D6E01498139A45F6AF
:106830002F41C0F60201F9F72BFD40F2D541C2F21B
:10684000000108780130087001201590C4E0149808
:1068500019F064FF40F2D541C2F20001087801301E
:10686000087001201590B7E01498139A45F62F315F
:10687000C0F60201F9F70CFD40F2D541C2F2000169
:1068800008780130087001201590A5E00BA819F0D8
:1068900061FC149813990B9AC2F5C04C6B46C3F86F
:1068A00004C01A6045F61A72C0F602024FF4C043E3
:1068B0001BF004FF40F2D541C2F20001087801301C
:1068C00008700120159087E01498139A45F6B031AE
:1068D000C0F60201F9F7DCFC40F2D541C2F200013A
:1068E0000878013008700120159075E01498089020
:1068F0001398099043F2DC20C2F20000D0F8AC10EB
:106900000491D0F8B400F9F745FE024604980592C8
:106910000A46059942EC101B8DED060BF9F73AFE7D
:106920009DED060B024608980B46099943EC112B86
:106930006A4682ED021B82ED000B45F62672C0F618
:1069400002021BF0BBFE40F2D541C2F20001087802
:1069500001300870012015903EE01498139A45F616
:10696000BC41C0F60201F9F793FC40F2D541C2F2F6
:106970000001087801300870012015902CE014986F
:10698000139943F2DC22C2F2000202F1CC03EC467E
:10699000CCF8003002F1B80345F65A72C0F6020294
:1069A0001BF08CFE40F2D541C2F2000108780130A4
:1069B0000870012015900FE01498139945F6D072D5
:1069C000C0F602021BF07AFE40F2D541C2F200018D
:1069D000002008701590FFE7159816B080BD0000E4
:1069E00080B582B0019001990020C0F60E006422AB
:1069F000FCF796F90198143000F038F80199C86254
:106A0000019800F075F8019988620198806A38B998
:106A1000FFE7019940F28810C2F200008862FFE7A8
:106A20000198C06A38B9FFE7019944F6D850C0F61A
:106A30000200C862FFE70198806A013038B9FFE7B9
:106A4000019940F28810C2F200008862FFE70198C5
:106A5000C06A013038B9FFE7019944F6D850C0F652
:106A60000200C862FFE702B080BD000080B584B0BC
:106A70000290029818B9FFE70020039029E0002057
:106A80000190FFE7019945F2E410C0F6020050F8CA
:106A90003100D8B1FFE7019945F2E410C0F60200D9
:106AA00050F831000299F9F706FC50B9FFE7019957
:106AB00045F2E410C0F6020000EBC100406803900C
:106AC00007E0FFE7019801300190DBE70020039029
:106AD000FFE7039804B080BD45F2E410C0F6020061
:106AE0007047000045F2FC10C0F60200704700003D
:106AF00080B584B00290029818B9FFE70020039097
:106B000029E000200190FFE7019945F2FC10C0F652
:106B1000020050F83100D8B1FFE7019945F2FC10AE
:106B2000C0F6020050F831000299F9F7C4FB50B9E1
:106B3000FFE7019945F2FC10C0F6020000EBC1002E
:106B40004068039007E0FFE7019801300190DBE720
:106B500000200390FFE7039804B080BD80B582B0A9
:106B6000019017F079F90B20FCF7B6F80199002095
:106B7000C0F60E006422FCF7DFF817F0C3F902B08C
:106B800080BD000080B541F66040C2F2000003F015
:106B9000F7FB80BD80B541F68020C2F2000003F013
:106BA000EFFB80BD80B541F62020C2F2000003F06B
:106BB000E7FB80BD80B541F6C040C2F2000003F0A3
:106BC000DFFB80BD80B541F6E020C2F2000003F09B
:106BD000D7FB80BD80B541F64030C2F2000003F023
:106BE000CFFB80BD80B541F6A030C2F2000003F0BB
:106BF000C7FB80BD80B541F62050C2F2000003F013
:106C0000BFFB80BD80B541F60040C2F2000003F03A
:106C1000B7FB80BD82B001900198007810384AF629
:106C2000AB21CAF6AA21A0FB01100009009000992F
:106C300044F6D830C0F60200405C0199C86500985F
:106C4000042807D3FFE701990868042262F30900CA
:106C5000886506E00199086840F2FF329043886534
:106C6000FFE70198806D02B07047000086B0059084
:106C700000208DF813000598806A039005988069BC
:106C800010BBFFE70398029003281BD80299DFE8A6
:106C900001F0020D0218059890F82F00C00720B1EE
:106CA000FFE701208DF81300FFE70CE00598C06AAC
:106CB000B0F1C07F04D1FFE701208DF81300FFE79A
:106CC00001E000E0FFE745E005988069B0F5005F6E
:106CD00025D1FFE70398019003281ED80199DFE82A
:106CE00001F00206021101208DF8130016E005984C
:106CF00090F82F00C00720B1FFE701208DF81300A6
:106D0000FFE70BE00598C06AB0F1C07F04D1FFE750
:106D100001208DF81300FFE700E0FFE719E003987A
:106D20000090032804D3FFE70098032804D00EE066
:106D300001208DF813000BE0059890F82F00C00794
:106D400020B1FFE701208DF81300FFE700E0FFE727
:106D5000FFE7FFE79DF8130006B0704784B003908B
:106D600002910192009303980168086820F4802042
:106D70000860009803990968486003988068402873
:106D800009D1FFE70198039909688860029803997F
:106D90000968C86008E0029803990968886001984A
:106DA00003990968C860FFE704B0704782B000909B
:106DB000009820B9FFE701208DF8070074E00098E3
:106DC00000886FF3DF20B0F5B67F09D3FFE70098A6
:106DD00000886FF3DF2040F29561884204D3FFE71B
:106DE00001208DF807005FE000980068C0F3CA201A
:106DF000B0F5B67F09D3FFE700980068C0F3CA205A
:106E000040F29561884204D3FFE701208DF8070026
:106E10004AE0009881880068800D40EA81206FF385
:106E2000DF20B0F5B67F0DD3FFE7009881880068BA
:106E3000800D40EA81206FF3DF2040F295618842A7
:106E400004D3FFE701208DF807002DE0009880882B
:106E5000C0F34A00B0F5B67F09D3FFE700988088F9
:106E6000C0F34A0040F29561884204D3FFE7012055
:106E70008DF8070018E0009881880020B0EB913F62
:106E800004D1FFE701208DF807000DE0009880880D
:106E9000000B800720B9FFE701208DF8070003E011
:106EA00000208DF80700FFE79DF8070002B070474B
:106EB00080B584B002900191029820B9FFE7FE20CE
:106EC0008DF80F000EE0019820B9FFE7FE208DF845
:106ED0000F0007E001982421F9F7CFF900208DF881
:106EE0000F00FFE79DF90F0004B080BD80B584B0AE
:106EF0000290029820B9FFE7FE208DF80F002BE0EA
:106F000042F26660C2F200000078C00720B1FFE7DD
:106F1000FD208DF80F001FE017F0CEFA43F29C41E0
:106F2000C2F20001086020B9FFE7FE208DF80F00D3
:106F300012E047F2C502C0F60002002001900321D2
:106F4000FCF78CFA019842F26662C2F2000201215B
:106F500011708DF80F00FFE79DF90F0004B080BDA0
:106F600080B584B002900191029820B9FFE7FE201D
:106F70008DF80F009FE00298FFF718FF20B1FFE7A0
:106F8000FF208DF80F0096E001982421F9F775F99C
:106F9000FFE70020C4F2A5400090029800886FF33C
:106FA000DF2000EE100AB8EE400A9FED451A30EEE1
:106FB000410A30EE000A9DED002A80EE020A019897
:106FC00080ED020A02980068C0F3CA2000EE100AA1
:106FD000B8EE400A30EE410A30EE000A9DED002A7C
:106FE00080EE020A019880ED030A02988188006809
:106FF000800D40EA81206FF3DF2000EE100AB8EE2A
:10700000400A30EE410A30EE000A9DED002A80EE83
:10701000020A019880ED000A02988088C0F34A00B5
:1070200000EE100AB8EE400A30EE410A30EE000AD7
:107030009DED002A80EE020A019880ED010A029877
:107040008088800B0199487502988088C0F30130D0
:10705000019908750298C0880199C8820298008930
:107060000199088302984089019948830298007B1E
:10707000002818BF0120019908770298407B00285A
:1070800018BF0120019948770298C0890199C883E7
:107090000298008A00EE100AB8EE400A30EE410A6B
:1070A0009DED001A80EE010A019880ED040A00208F
:1070B0008DF80F00FFE79DF90F0004B080BD00BF01
:1070C0000000804480B543F29C40C2F2000000689A
:1070D000802117F011F980BD80B582B000900020AA
:1070E000FCF75CF9009912220BF0A8FA20B9FFE72F
:1070F00000208DF8070003E0FF208DF80700FFE770
:107100009DF9070002B080BD80B582B00190019A60
:107110008020012117F042F98038B0FA80F0400950
:1071200002B080BD7047000080B5012003F086FFEB
:1071300080BD000080B5082003F080FF80BD000006
:1071400080B5102003F07AFF80BD000080B52020BC
:1071500003F074FF80BD0000FFE700BFFDE7000003
:1071600080B584B003908DF80B1000200190039837
:1071700060B3FFE70398012828D0FFE703980228AF
:1071800024D0FFE70398032820D0FFE703980428C2
:107190001CD0FFE70398052818D0FFE703980628BE
:1071A00014D0FFE70398072810D0FFE703980828BA
:1071B0000CD0FFE70398092808D0FFE703980A28B6
:1071C00004D0FFE703980B2801D1FFE708E045F260
:1071D000FD20C0F6020040F2DB3116F0ADFCFFE707
:1071E0009DF80B0078B1FFE79DF80B0001280AD04D
:1071F000FFE79DF80B00022805D0FFE79DF80B0084
:10720000032801D1FFE708E045F2FD20C0F60200A7
:107210004FF4777116F090FCFFE79DF80B0018B95A
:10722000FFE70020019017E09DF80B00012804D132
:10723000FFE74FF4807001900DE09DF80B000228ED
:1072400004D1FFE74FF40070019003E04FF4407069
:107250000190FFE7FFE7FFE743F61041C4F20201A8
:10726000086820F440700860019A086810430860BC
:10727000086820F0F8000860039A086840EAC20035
:1072800040F002000860086840F48030086004B0F4
:1072900080BD000043F60040C4F202000068800593
:1072A00000281FD5FFE743F60041C4F20201086839
:1072B00020F400700860FFE743F60041C4F20201C9
:1072C000086840F400600860086820F40060086006
:1072D000FFE743F60041C4F20201086840F4007081
:1072E0000860FFE743F60040C4F202000068400572
:1072F00000281FD5FFE743F60041C4F202010868E9
:1073000020F480600860FFE743F60041C4F2020108
:10731000086840F480500860086820F480500860D5
:10732000FFE743F60041C4F20201086840F48060C0
:107330000860FFE77047000080B582B08DF8070055
:1073400000919DF8070078B1FFE79DF8070001283C
:107350000AD0FFE79DF80700022805D0FFE79DF857
:107360000700032801D1FFE708E045F2FD20C0F641
:1073700002004FF46F7116F0DFFBFFE70098012861
:1073800001D1FFE708E045F2FD20C0F6020040F21F
:10739000BD3116F0D1FBFFE743F61041C4F2020104
:1073A000086820F440700860086840F00400086035
:1073B0009DF80720086840EA022040F48030086009
:1073C00002B080BD80B582B001908DF803100198A5
:1073D000B0F1006F05D3FFE70198B0F1016F10D352
:1073E000FFE7019847F60001C1F6FF71884209D313
:1073F000FFE7019847F60F21C1F6FF71884201D8D7
:10740000FFE708E045F2C320C0F6020040F2BB21CE
:1074100016F092FBFFE743F61041C4F20201086840
:1074200020F44070086008680860086840F00100B7
:1074300008609DF803000199087002B080BD00004B
:1074400080B584B00390019300920398B0F1006F6F
:1074500005D3FFE70398B0F1016F10D3FFE703985E
:1074600047F60001C1F6FF71884209D3FFE7039890
:1074700047F60F21C1F6FF71884201D8FFE708E007
:1074800045F2C320C0F6020040F2672116F054FB1B
:10749000FFE743F61041C4F20201086820F440708F
:1074A0000860086840F440700860086840F0010017
:1074B0000860009803990860BFF36F8F01980399E3
:1074C000486004B080BD000080B582B00190ADF886
:1074D00002100198B0F1006F05D3FFE70198B0F1F9
:1074E000016F10D3FFE7019847F60001C1F6FF7165
:1074F000884209D3FFE7019847F60F21C1F6FF71D3
:10750000884201D8FFE708E045F2C320C0F6020038
:1075100040F2A22116F010FBFFE743F61041C4F23F
:107520000201086820F440700860086840F4807028
:107530000860086840F001000860BDF80200019989
:10754000088002B080BD000080B582B0019000913B
:107550000198B0F1006F05D3FFE70198B0F1016F1A
:1075600010D3FFE7019847F60001C1F6FF7188428A
:1075700009D3FFE7019847F60F21C1F6FF71884252
:1075800001D8FFE708E045F2C320C0F6020040F250
:10759000892116F0D1FAFFE743F61041C4F2020147
:1075A000086820F440700860086840F400700860C3
:1075B000086840F00100086000980199086002B076
:1075C00080BD000043F60C40C4F202000068C00613
:1075D00000280FD5FFE742F28061C2F20001C869BE
:1075E00040F01000C86143F60C41C4F202011020C3
:1075F0000860FFE743F60C40C4F202000068800612
:1076000000280FD5FFE742F28061C2F20001C8698D
:1076100040F00800C86143F60C41C4F2020120208A
:107620000860FFE743F60C40C4F202000068400621
:1076300000280FD5FFE742F28061C2F20001C8695D
:1076400040F00400C86143F60C41C4F2020140203E
:107650000860FFE743F60C40C4F202000068000631
:1076600000280FD5FFE742F28061C2F20001C8692D
:1076700040F00200C86143F60C41C4F202018020D0
:107680000860FFE743F60C40C4F202000068800780
:1076900000280FD5FFE742F28061C2F20001C869FD
:1076A00040F02000C86143F60C41C4F20201022000
:1076B0000860FFE77047000080B584B002900020AA
:1076C000019042F28061C2F20001C86104F0C8F882
:1076D0000190FFE743F60C40C4F202000068C003CB
:1076E000002815D5FFE70298013080B1FFE7029826
:1076F00040B1FFE704F0B4F80199401A02998842BA
:1077000004D9FFE703208DF80F0023E0FFE7E1E74E
:1077100043F60C40C4F202000068C00738B1FFE72E
:1077200043F60C41C4F2020101200860FFE743F672
:107730000C40C4F20200006810F0F20F06D0FFE720
:10774000FFF740FF01208DF80F0003E000208DF8C7
:107750000F00FFE79DF80F0004B080BD40F6313008
:10776000C2F200007047000088B0079006910592B1
:1077700000200490039005990860FFE7049806999B
:10778000884260D2FFE7FFE7079801780020029067
:1077900039B1FFE707980078203818BF0120029020
:1077A000FFE70298C00720B1FFE707980130079074
:1077B000EAE7FFE7079801780020019041B1FFE771
:1077C000079800782038B0FA80F040090190FFE770
:1077D0000198C00720B1FFE7079801300790E9E75B
:1077E0000798007868B3FFE7049801300490049884
:1077F0000699884224D1FFE707980390FFE707988E
:1078000001780020009039B1FFE707980078203810
:1078100018BF01200090FFE70098C00740B1FFE7C4
:107820000599086801300860079801300790E6E77D
:107830000598006818B9FFE700200390FFE702E011
:1078400000E000E09AE7039808B0704780B586B082
:107850000590049103920120029040F2D840C2F2B8
:1078600000000068002859D1FFE740F2D841C2F279
:10787000000140F25040C2F200000860FFE740F211
:10788000D840C2F200000068002846D0FFE740F26E
:10789000D840C2F2000000680068006801900198BA
:1078A000F8F702FD009005980099405C202805D06B
:1078B000FFE705980099405C30BBFFE70598019908
:1078C000009AF8F70FFDF0B9FFE740F2D840C2F296
:1078D00000000068006890F90C00002812D4FFE74F
:1078E000059817F041FA40F2D841C2F20001096848
:1078F000096891F90C10884203D0FFE7002002903C
:10790000FFE7FFE709E0FFE7FFE740F2D841C2F2F7
:107910000001086840680860B1E7FFE740F2D8401E
:10792000C2F20000006890B1FFE7029878B9FFE763
:107930000498039A45F21B61C0F60201F8F7A8FC0F
:1079400040F2D841C2F200010020086029E040F274
:10795000D840C2F200000068B8B1FFE740F2D8405A
:10796000C2F2000000680068836804980399059AD1
:1079700098470290029838B9FFE740F2D841C2F226
:10798000000100200860FFE70AE00498039A45F22E
:107990007361C0F60201F8F77BFC00200290FFE75C
:1079A000FFE7029806B080BD80B586B00390002046
:1079B0000190039858B9FFE74FF0500080F3118809
:1079C000BFF36F8FBFF34F8F0490FFE7FEE70820F0
:1079D00018F034F80290029858B9FFE74FF05000C1
:1079E00080F31188BFF36F8FBFF34F8F0590FFE7D0
:1079F000FEE70298B0B1FFE718F0F2FA0398029997
:107A00000860029900204860029840F22401C2F206
:107A100000010A6850600298086018F00DFB012010
:107A20000190FFE7019806B080BD000080B584B0EA
:107A300047F61020C1F6FF700068039047F6142047
:107A4000C1F6FF700068029047F61820C1F6FF707B
:107A5000006801900199039808440390039888B145
:107A6000FFE7039840F26811C2F200010091023171
:107A700008220AF08BFF00990298123104220AF0C2
:107A800085FFFFE704B080BD80B58EB006AB0493E0
:107A90000C900B910A920C9820B9FFE7FF208DF80B
:107AA000370054E10B9820B9FFE7FF208DF837002D
:107AB0004DE10A990C980268891A00EE101AB8EE86
:107AC000400A9FEDA51A80EE010A80ED010A0A988E
:107AD0000C9908600C980B99097800F0EDF90B9857
:107AE00090ED020AB1EE400A80ED020A0B9890ED8B
:107AF000010AB1EE400A80ED010A0C9810300B9992
:107B000091ED010ADFED950ACDED020AFDF7C6FE03
:107B10009DED021A0C9890ED054A90ED430A90ED08
:107B20005B3A90ED5E2A32EE042A72EE430AFDF7CC
:107B3000F7FE9DED021A049880ED030A0C9890ED73
:107B4000054A90ED440A90ED5B3A90ED5E2A32EEE4
:107B5000042A72EE430AFDF7E3FE049981ED020A5E
:107B60000B98083091ED020AD1ED030AFDF736FFBC
:107B70000B9890ED021A0C9890ED050A30EE010A70
:107B800080ED050A0B980430F9F7DEF90C98007BBC
:107B90000146039140B1FFE7039801281DD0FFE79C
:107BA000039802285CD074E000208DF81700FFE7EE
:107BB0009DF8170001280FDCFFE70C989DF81710BF
:107BC00000EB81010020C1F85401FFE79DF8170088
:107BD00001308DF81700EBE75BE00C9901F15800DC
:107BE000D1ED011A91ED040AD1ED5A0A9FED5C1A0C
:107BF0008DED011A0CF052FB049A9DED011A82EDF5
:107C0000010A0C9901F11C0092ED010AD1ED011A53
:107C1000D1ED590A0CF042FB9DED011A0C9880ED54
:107C2000550A0C9901F1D000D1ED011A91ED050A28
:107C3000D1ED5B0A0CF032FB049A9DED011A82ED46
:107C4000000A0C9901F1940092ED000AD1ED011A9D
:107C5000D1ED570A0CF022FB0C9880ED560A18E083
:107C600000208DF81600FFE79DF8160001280FDCB4
:107C7000FFE70C989DF8161000EB81010020C1F879
:107C80005401FFE79DF8160001308DF81600EBE770
:107C9000FFE700208DF81500FFE79DF8150001288B
:107CA0001BDCFFE70C999DF8152001EB421000F555
:107CB0008A7001EB820191ED550A0AF0DFFE0C9803
:107CC0009DF8151000EB810080ED550AFFE79DF847
:107CD000150001308DF81500DFE70C98806890F8EA
:107CE0008C00C00740B1FFE70C9890ED550AB1EE4B
:107CF000400A80ED550AFFE70C98806890F88D00E7
:107D0000C00740B1FFE70C9890ED560AB1EE400A6B
:107D100080ED560AFFE70C9890ED550AB5EE400A43
:107D2000F1EE10FA02DAFFE700BFFFE70C9890EDE2
:107D3000560AB6EE001AB4EE410AF1EE10FA02DD70
:107D4000FFE700BFFFE700208DF83700FFE79DF950
:107D500037000EB080BD00BF00007A44DB0FC94081
:107D60000000000082B0019000910198D0F8540109
:107D7000009908600198D0F858010099486002B055
:107D80007047000082B0019000910198007B00993B
:107D9000087002B07047000080B58AB005AA03924F
:107DA000024603980892079180ED010AC0ED000A8F
:107DB000089820B9FFE7FF208DF8270076E00798A4
:107DC000089988600899002008730898806890F8DE
:107DD0008D00C00720B1FFE706A8FDF7EFFDFFE724
:107DE000039890ED010A089880ED430A089880ED09
:107DF000440A089901F58870896891ED220AB1EE6C
:107E0000400ADFED2C0AFDF749FD039A089901F1BC
:107E1000580092ED000A896801F1200200210291C8
:107E20000CF0B4FB039A089901F11C0092ED000AD2
:107E30008A68012101910CF0A9FB039B0299089A21
:107E400002F1D00093ED000A926860320CF09EFBC4
:107E5000039B0199089A02F1940093ED000A92683D
:107E600040320CF093FB02988DF81300FFE79DF869
:107E70001300012816DCFFE7039A08999DF8130008
:107E800001EB401000F58A7092ED000A8968D1ED8F
:107E9000200A0AF04FFEFFE79DF8130001308DF82D
:107EA0001300E4E700208DF82700FFE79DF9270085
:107EB0000AB080BDDB0FC94080B584B002908DF858
:107EC0000710029820B9FFE7FF208DF80F0065E04A
:107ED0009DF807000299097B884204D1FFE7002042
:107EE0008DF80F005AE000208DF80600FFE79DF89E
:107EF0000600032811DCFFE702989DF80610C1EB8D
:107F0000011100EB81001C300CF00CFCFFE79DF828
:107F1000060001308DF80600E9E700208DF8050025
:107F2000FFE79DF80500012812DCFFE702989DF8A5
:107F3000051000EB411000F58A709FED1A0A0AF057
:107F400097FEFFE79DF8050001308DF80500E8E792
:107F500002981030F8F7F8FF0298007BB0B9FFE7FD
:107F60009DF80700012805D1FFE70299D1F86801C3
:107F700008610AE09DF80700022805D1FFE7029991
:107F8000D1F874010861FFE7FFE7FFE79DF80700FC
:107F90000299087300208DF80F00FFE79DF90F008C
:107FA00004B080BD0000000080B584B00290019153
:107FB000029820B9FFE7FF208DF80F002EE001980E
:107FC00020B9FFE7FF208DF80F0027E00198406CF3
:107FD0000299C1F874010198406D0299C1F87801C5
:107FE0000298806890F88C00C00730B1FFE70298D3
:107FF00000F5BA70FDF7E2FCFFE70298806890F8A0
:108000008D00C00730B1FFE7029800F5BC70FDF7A6
:10801000D5FCFFE700208DF80F00FFE79DF90F006A
:1080200004B080BD80B586B004900391002002901A
:1080300003980068122801D8FFE708E045F2E6300F
:10804000C0F6020040F2896115F076FDFFE7039863
:10805000406830B1FFE703984068102801D8FFE777
:1080600008E045F2E630C0F6020040F28A6115F001
:1080700063FDFFE70398806818B3FFE70398806803
:1080800001281ED0FFE703988068022819D0FFE777
:1080900003988068032814D0FFE7039880680428B9
:1080A0000FD0FFE70398806805280AD0FFE7039800
:1080B0008068062805D0FFE703988068072801D16B
:1080C000FFE708E045F2E630C0F6020040F28B61BF
:1080D00015F032FDFFE7FFE7049890F83C00012817
:1080E00004D1FFE702208DF81700F7E00499012082
:1080F00081F83C00FFE7FFE7039800680A281CD3DB
:10810000FFE70398008800EB4000A0F11E01072064
:1081100000FA01F204980168C8689043C8600399A6
:108120008868098801EB41011E3900FA01F20498C0
:108130000168C8681043C86018E00398008800EB25
:108140004001072000FA01F2049801680869904391
:10815000086103998868098801EB410100FA01F27E
:1081600004980168086910430861FFE703984068B4
:1081700006281BD8FFE70398406800EB8000411FEA
:108180001F2000FA01F204980168486B904348638D
:1081900003990888496801EB8101053900FA01F269
:1081A00004980168486B104348633DE003984068B9
:1081B0000C281CD8FFE70398406800EB8000A0F172
:1081C00023011F2000FA01F204980168086B904314
:1081D000086303990888496801EB8101233900FA93
:1081E00001F204980168086B104308631BE00398D0
:1081F000406800EB8000A0F141011F2000FA01F26D
:1082000004980168C86A9043C8620399088849685D
:1082100001EB8101413900FA01F204980168C86A52
:108220001043C862FFE7FFE742F20030C4F20100EA
:1082300001900498006842F20001C4F201018842F2
:108240000BD1FFE703980068122806D1FFE70199D8
:10825000486840F480004860FFE70498006842F2F4
:108260000001C4F2010188422ED1FFE703980068A3
:10827000102805D0FFE703980068112824D1FFE7F4
:108280000199486840F4000048600398006810288D
:1082900019D1FFE740F22800C2F2000000684DF655
:1082A0008361C4F21B31A0FB0110800C00EB800045
:1082B00040000290FFE7029820B1FFE702980138E2
:1082C0000290F8E7FFE7FFE7FFE70499002081F855
:1082D0003C00FFE700208DF81700FFE79DF817002E
:1082E00006B080BD81B0009000980068C06C01B0FD
:1082F0007047000080B584B0029000208DF8070020
:10830000029820B9FFE701208DF80F00C7E102981D
:10831000006842F20001C4F20101884212D0FFE776
:108320000298006842F20011C4F20101884209D0AB
:10833000FFE70298006842F20021C4F2010188427E
:1083400001D1FFE708E045F2E630C0F6020040F256
:10835000431115F0F1FBFFE70298406890B1FFE789
:1083600002984068B0F5803F0CD0FFE70298406863
:10837000B0F5003F06D0FFE702984068B0F5403FF7
:1083800001D1FFE708E045F2E630C0F602004FF405
:10839000A27115F0D1FBFFE70298806890B1FFE76A
:1083A00002988068B0F1807F0CD0FFE70298806867
:1083B000B0F1007F06D0FFE702988068B0F1407FFF
:1083C00001D1FFE708E045F2E630C0F6020040F2D6
:1083D000451115F0B1FBFFE70298006928B1FFE7EE
:1083E00002980069012801D1FFE708E045F2E63074
:1083F000C0F602004FF4A37115F09EFBFFE7029850
:10840000007E28B1FFE70298007E012801D1FFE736
:1084100008E045F2E630C0F6020040F2471115F0E0
:108420008BFBFFE70298806A002862D0FFE7029882
:10843000806AB0F1807F5CD0FFE70298806AB0F17B
:10844000007F56D0FFE70298806AB0F1407F50D09D
:10845000FFE70298806AB0F1806F4AD0FFE7029888
:10846000806AB0F1A06F44D0FFE70298806AB0F153
:10847000C06F3ED0FFE70298806AB0F1E06F38D05D
:10848000FFE70298806AB0F1006F32D0FFE70298F0
:10849000806AB0F1106F2CD0FFE70298806AB0F1CB
:1084A000206F26D0FFE70298806AB0F1306F20D0AD
:1084B000FFE70298806AB0F1406F1AD0FFE7029898
:1084C000806AB0F1506F14D0FFE70298806AB0F173
:1084D000606F0ED0FFE70298806AB0F1706F08D02D
:1084E000FFE70298806A0121C0F60071884201D13D
:1084F000FFE708E045F2E630C0F602004FF4A47151
:1085000015F01AFBFFE70298C06830B1FFE7029848
:10851000C068B0F5006F01D1FFE708E045F2E63032
:10852000C0F6020040F2491115F006FBFFE7029881
:10853000C06930B1FFE70298C069102801D8FFE791
:1085400008E045F2E630C0F602004FF4A57115F0E0
:10855000F3FAFFE7029890F8300030B1FFE7029895
:1085600090F83000012801D1FFE708E045F2E6303D
:10857000C0F6020040F24B1115F0DEFAFFE7029858
:108580004069012809D0FFE70298406928B1FFE758
:1085900002984069022801D1FFE708E045F2E63081
:1085A000C0F602004FF4A67115F0C6FAFFE7029874
:1085B00090F8200030B1FFE7029890F820000128E1
:1085C00001D1FFE708E045F2E630C0F6020040F2D4
:1085D0004D1115F0B1FAFFE70298806A0121C0F64B
:1085E0000071884221D0FFE70298C06A90B1FFE78E
:1085F0000298C06AB0F1805F0CD0FFE70298C06AB1
:10860000B0F1005F06D0FFE70298C06AB0F1405FAA
:1086100001D1FFE708E045F2E630C0F6020040F283
:10862000511115F089FAFFE7FFE70298006C50B985
:10863000FFE7029800F038F8029900204864029998
:1086400081F83C00FFE70298006CC006002817D4B0
:10865000FFE70298006C40F0020020F48850029975
:1086600008640298F8F7A6F9029900204864029875
:10867000006C40F0010020F002000299086403E061
:1086800001208DF80700FFE7FFE70299002081F83D
:108690003C00FFE79DF807008DF80F00FFE79DF80D
:1086A0000F0004B080BD000080B58AB009900020A2
:1086B000089007900690059004900998006842F28F
:1086C0000001C4F20101884212D1FFE7FFE7002058
:1086D000039043F64400C4F20200016841F4807143
:1086E0000160006800F4807003900398FFE73AE0AF
:1086F0000998006842F20021C4F20101884231D198
:10870000FFE7FFE70020029043F64400C4F20200B6
:10871000016841F480610160006800F480600290AB
:108720000298FFE7FFE70020019043F63000C4F213
:108730000200016841F020010160006800F02000A3
:1087400001900198FFE74FF48060049003200590AA
:108750000020069041F20040C4F2020004A902F099
:1087600089FCFFE7FFE70AB080BD000080B584B058
:1087700002900191002000900298006880684005F6
:10878000002816D5FFE7029800688068C005002819
:108790000FD5FFE70299086C40F020000864FFE75E
:1087A0000299002081F83C00FFE701208DF80F00BE
:1087B0006DE003F055F80090FFE70298006800684C
:1087C00000F00200022829D0FFE70198013020B311
:1087D000FFE7019840B1FFE703F042F80099401A23
:1087E0000199884218D9FFE702980068006800F0F4
:1087F000020002280FD0FFE70299086C40F0040045
:108800000864FFE70299002081F83C00FFE703209D
:108810008DF80F003BE0FFE7FFE7CEE70298016825
:108820006FF0120008600299086C40F40070086450
:1088300002980068806810F0405F24D1FFE702983A
:10884000007E00BBFFE702980068C06A10F4700F5A
:1088500007D0FFE70298006880684005002812D41E
:10886000FFE70299086C20F4807008640298006C9D
:10887000C004002806D4FFE70299086C40F001000C
:108880000864FFE7FFE700208DF80F00FFE79DF881
:108890000F0004B080BD000080B584B002900020BD
:1088A00001900298007E28B1FFE70298007E01281F
:1088B00001D1FFE708E045F2E630C0F6020040F2E1
:1088C000D32115F039F9FFE70298C06A90B1FFE7AC
:1088D0000298C06AB0F1805F0CD0FFE70298C06ACE
:1088E000B0F1005F06D0FFE70298C06AB0F1405FC8
:1088F00001D1FFE708E045F2E630C0F602004FF490
:10890000357115F019F9FFE7FFE7029890F83C0080
:10891000012804D1FFE702208DF80F00D4E002996E
:10892000012081F83C00FFE7FFE7029800688068BB
:10893000C007F0B9FFE702980168886840F00100BD
:10894000886040F22800C2F2000000684DF68361A2
:10895000C4F21B31A0FB0110800C00EB4000019021
:10896000FFE7019820B1FFE7019801380190F8E78F
:10897000FFE7029800688068C007002800F0958033
:10898000FFE70298006C40F4807040F20161884378
:10899000029908640298006840684005002809D5DB
:1089A000FFE70298006C40F4805020F400500299D8
:1089B0000864FFE70298006CC004002806D5FFE7B2
:1089C0000299486C20F00600486403E002990020F8
:1089D0004864FFE7FFE70299002081F83C00FFE7C9
:1089E00042F20030C4F201000090029801686FF07A
:1089F0002200086000984068C006E8BBFFE70298C4
:108A0000006842F20001C4F20101884224D0FFE76D
:108A10000298006842F20011C4F20101884208D1B4
:108A2000FFE742F20430C4F201000068C00698B1CA
:108A3000FFE70298006842F20021C4F20101884277
:108A400019D1FFE742F20430C4F20100006800F0DF
:108A50001F000F280FD8FFE702980068806810F009
:108A6000405F07D1FFE702980168886840F08040C6
:108A70008860FFE7FFE717E00298006842F2000114
:108A8000C4F2010188420ED1FFE7029800688068B5
:108A900010F0405F07D1FFE702980168886840F056
:108AA00080408860FFE7FFE70AE00299086C40F029
:108AB000100008640299486C40F001004864FFE728
:108AC00000208DF80F00FFE79DF80F0004B080BD77
:108AD00080B584B002900191029890F820008DF842
:108AE0000300019848F67F71C0F20301884201D863
:108AF000FFE708E045F21E40C0F602004FF4D061E7
:108B000015F01AF8FFE79DF80300012805D0FFE7EC
:108B10009DF8030002280AD1FFE7019A0298016834
:108B200048691043486100208DF80F0008E0029961
:108B3000486A40F48020486201208DF80F00FFE76A
:108B40009DF80F0004B080BD80B588B006900591F7
:108B500004920393069890F820008DF80700069879
:108B60000068806800900598806828B1FFE7059844
:108B70008068042801D1FFE708E045F21E40C0F6F6
:108B8000020040F2E94114F0D7FFFFE70598C06802
:108B900028B1FFE70598C068022801D1FFE708E087
:108BA00045F21E40C0F6020040F2EA4114F0C4FF54
:108BB000FFE705980069082801D8FFE708E045F2BB
:108BC0001E40C0F6020040F2EB4114F0B5FFFFE793
:108BD0000598806890B9FFE7059801680020B0EB20
:108BE000D12F01D1FFE708E045F21E40C0F6020098
:108BF00040F2EE4114F0A0FFFFE711E00598416854
:108C00000020B0EB517F01D1FFE708E045F21E40A4
:108C1000C0F6020040F2F24114F08EFFFFE7FFE7DA
:108C20000598007D28B1FFE70598007D012801D156
:108C3000FFE708E045F21E40C0F6020040F2F441B2
:108C400014F07AFFFFE79DF80700012806D0FFE740
:108C50009DF80700022840F08D80FFE79DF8030093
:108C6000400700280CD4FFE79DF803000007002808
:108C700006D4FFE79DF80300C006002871D5FFE782
:108C80000098C0F3016002900298032809D3FFE71F
:108C90000699486A40F40000486201208DF81F00E0
:108CA00071E0029901208840039908600598806866
:108CB00068B9FFE705980168C06840EA4150069925
:108CC0000968029A01EB0211C1F880010EE00599D2
:108CD0004A688868C96840EAC2000843069909687A
:108CE000029A01EB0211C1F88001FFE705980069C3
:108CF00006990968029A01EB0211C1F884010598EE
:108D0000007D01280CD1FFE706980068029900EB6E
:108D10000111D1F8840140F48070C1F88401FFE7AB
:108D20000498406806990968029A01EB0211C1F89B
:108D30008C010498006806990968029A01EB0211F7
:108D4000C1F8880106980068029900EB0111D1F87A
:108D5000800140F00100C1F8800100208DF81F0063
:108D600011E00699486A40F40010486201208DF82D
:108D70001F0008E00699486A40F4802048620120FC
:108D80008DF81F00FFE79DF81F0008B080BD0000B0
:108D900080B586B00490039104980068019004980F
:108DA00090F820008DF803009DF80300012806D0FC
:108DB000FFE79DF80300022840F05281FFE7039887
:108DC000408808B9FFE708E045F21E40C0F60200FF
:108DD0004FF4547114F0B0FEFFE70398C08808B94F
:108DE000FFE708E045F21E40C0F6020040F25131B4
:108DF00014F0A2FEFFE70398408908B9FFE708E0F6
:108E000045F21E40C0F6020040F2523114F094FECA
:108E1000FFE70398C08908B9FFE708E045F21E4064
:108E2000C0F6020040F2533114F086FEFFE70398CB
:108E3000806928B1FFE703988069012801D1FFE725
:108E400008E045F21E40C0F602004FF4557114F0E0
:108E500073FEFFE70398C06928B1FFE70398C06974
:108E6000012801D1FFE708E045F21E40C0F60200EC
:108E700040F2553114F060FEFFE70398006928B115
:108E8000FFE703980069012801D1FFE708E045F2F8
:108E90001E40C0F6020040F2563114F04DFEFFE7CE
:108EA0000398006A28B1FFE70398006A012801D1FE
:108EB000FFE708E045F21E40C0F6020040F25731DD
:108EC00014F03AFEFFE746F20040C4F200000190C1
:108ED000039840691B2801D8FFE708E045F21E40CF
:108EE000C0F6020040F2723114F026FEFFE703984C
:108EF000406A1B2801D8FFE708E045F21E40C0F693
:108F0000020040F2733114F017FEFFE70199D1F827
:108F1000000240F00100C1F800020199D1F80002FE
:108F200020F47C50C1F800020398426A0199D1F8FC
:108F3000000240EA0220C1F800020398406900F0F4
:108F40001F01012088400290029A0199D1F81C0269
:108F50009043C1F81C020398C069F0B9FFE7029A78
:108F60000199D1F80C029043C1F80C02039A908841
:108F7000D168526940EA0140019901EBC201C1F890
:108F80004002039A10889168526940EA01400199B1
:108F900001EBC201C1F84402FFE70398C069012850
:108FA0001ED1FFE7029A0199D1F80C021043C1F8D3
:108FB0000C02039A90881168526940EA01400199B5
:108FC00001EBC201C1F84002039A9089916852698D
:108FD00040EA0140019901EBC201C1F84402FFE7F8
:108FE0000398806940B9FFE7029A0199D1F8040219
:108FF0009043C1F8040207E0029A0199D1F80402F3
:109000001043C1F80402FFE70398006940B9FFE785
:10901000029A0199D1F814029043C1F8140207E0B2
:10902000029A0199D1F814021043C1F81402FFE723
:109030000398006A012808D1FFE7029A0199D1F844
:109040001C021043C1F81C02FFE70199D1F800028D
:1090500020F00100C1F8000200208DF8170008E0A0
:109060000499486A40F48020486201208DF8170076
:10907000FFE79DF8170006B080BD000080B582B004
:1090800001900198FAF766FC8DF803009DF8030043
:10909000032819D0FFE79DF8030040F25842C2F2BE
:1090A0000002342110FB0120006B60B1FFE79DF846
:1090B000030040F25842C2F20002342110FB0120AA
:1090C000006B8047FFE7FFE702B080BD80B586B048
:1090D0000490039102920193049890F820008DF877
:1090E0000300039820B1FFE70398012801D1FFE7AF
:1090F00008E045F21E40C0F602004FF4BE6114F0D5
:109100001BFDFFE79DF80300012806D0FFE79DF84F
:109110000300022840F0D780FFE7039880B9FFE7FB
:1091200004980068C068800748B9FFE70499486A56
:1091300040F40010486201208DF81700CCE00FE0E9
:10914000049800680069800748B9FFE70499486AF5
:1091500040F40010486201208DF81700BCE0FFE7E2
:1091600004980068039900EB0110D0F8B00100F0FA
:109170000400029988600298806858B9FFE7049853
:109180000068039900EB0110D0F8B001400D02997E
:1091900008600AE004980068039900EB0110D0F819
:1091A000B001C00802994860FFE70498006803997D
:1091B00000EB0110D0F8B00100F002000299C86085
:1091C00004980068039900EB0110D0F8B40100F096
:1091D0000F000299086104980068039900EB0110E0
:1091E000D0F8B40180B2000A02998861049800683E
:1091F000039900EB0110D0F8B401000C029948610A
:1092000004980068039900EB0110D0F8B8010199A7
:10921000087004980068039900EB0110D0F8B801B9
:10922000000A0199487004980068039900EB011046
:10923000D0F8B801000C019988700498006803996F
:1092400000EB0110D0F8B801000E0199C870049825
:109250000068039900EB0110D0F8BC010199087176
:1092600004980068039900EB0110D0F8BC01000AD3
:109270000199487104980068039900EB0110D0F837
:10928000BC01000C0199887104980068039900EBF7
:109290000110D0F8BC01000E0199C871039838B9CB
:1092A000FFE704980168C86840F02000C86006E045
:1092B00004980168086940F020000861FFE7002079
:1092C0008DF8170008E00499486A40F4802048624D
:1092D00001208DF81700FFE79DF8170006B080BD4C
:1092E00080B58AB00990002008900998006840690C
:1092F000079009980068406806900998006880689F
:10930000059009980068C068049009980068006991
:10931000039009980068806902909DF81C00C007BE
:10932000002800F09480FFE79DF81400C00758B3B0
:10933000FFE709980168012088609DF81400800704
:10934000002804D5FFE7099800F042FE1BE09DF8D5
:1093500014004007002805D5FFE7089840F4006096
:1093600008900FE09DF814000007002805D5FFE7DE
:10937000089840F48050089003E0099800F000FE3F
:10938000FFE7FFE7FFE7FFE79DF81500C00760B3C1
:10939000FFE7099801684FF4807088609DF8150018
:1093A0008007002804D5FFE7099800F05FFE1BE066
:1093B0009DF815004007002805D5FFE7089840F400
:1093C000005008900FE09DF815000007002805D513
:1093D000FFE7089840F48040089003E0099800F007
:1093E0001DFEFFE7FFE7FFE7FFE79DF81600C00758
:1093F00060B3FFE7099801684FF4803088609DF8FA
:1094000016008007002804D5FFE7099800F07EFECB
:109410001BE09DF816004007002805D5FFE70898D7
:1094200040F4004008900FE09DF816000007002867
:1094300005D5FFE7089840F48030089003E00998CC
:1094400000F03CFEFFE7FFE7FFE7FFE7FFE79DF8DF
:109450001C000007002810D5FFE79DF81000C0068B
:10946000002809D5FFE7089840F400700890099893
:1094700001681020C860FFE7FFE79DF81C00400767
:1094800000280FD5FFE79DF810000007002808D539
:10949000FFE7099801680820C860099800F062FC9D
:1094A000FFE7FFE79DF81C00800700280BD5FFE7CA
:1094B00009980068C068800720B1FFE7099800F0AC
:1094C00079FCFFE7FFE79DF81C004006002810D557
:1094D000FFE79DF80C00C006002809D5FFE70898B3
:1094E00040F4806008900998016810200861FFE747
:1094F000FFE79DF81C00800600280FD5FFE79DF8C8
:109500000C000007002808D5FFE70998016808202B
:109510000861099800F076FCFFE7FFE79DF81C0062
:10952000C00600280BD5FFE709980068006980078E
:1095300020B1FFE7099800F08DFCFFE7FFE79DF8F9
:109540001E00800700280FD5FFE79DF81800C00611
:10955000002808D5FFE7099801681020486009989D
:1095600000F0A0FCFFE7FFE79DF81E00C00778B100
:10957000FFE79DF818000007002808D5FFE70998C5
:10958000016808204860099800F0E8FDFFE7FFE760
:109590009DF81D000006002840F18D80FFE79DF832
:1095A00018004007002840F18180FFE79DF81D006A
:1095B000C00750B1FFE79DF80800C00728B1FFE7DA
:1095C000089840F001000890FFE79DF81D00800713
:1095D00000280BD5FFE79DF808008007002805D577
:1095E000FFE7089840F002000890FFE79DF81D0093
:1095F000400700280BD5FFE79DF80800400700282A
:1096000005D5FFE7089840F004000890FFE79DF8B3
:109610001D000007002848D5FFE79DF8080010F05E
:10962000700F42D0FFE7029800F0700001460191F0
:10963000102814D0FFE70198202815D0FFE70198E3
:10964000302816D0FFE70198402817D0FFE701988F
:10965000502818D0FFE70198602819D01DE008981D
:1096600040F00800089019E0089840F010000890B9
:1096700014E0089840F0200008900FE0089840F0AF
:10968000400008900AE0089840F08000089005E04B
:10969000089840F48070089000E0FFE7099801689E
:1096A000886920F070008861FFE7FFE7099801688A
:1096B00004204860FFE7089848B1FFE7089A099935
:1096C000486A104348620998FFF7D8FCFFE70AB0E0
:1096D00080BD000080B584B00290029820B9FFE7F9
:1096E00001208DF80F0063E20298006846F2004105
:1096F000C4F20001884209D0FFE70298006846F6EC
:109700000001C4F20001884201D1FFE708E045F200
:109710001E40C0F6020040F21D1114F00DFAFFE7E2
:109720000298007E28B1FFE70298007E012801D14F
:10973000FFE708E045F21E40C0F602004FF48F71CB
:1097400014F0FAF9FFE70298407E28B1FFE702988B
:10975000407E012801D1FFE708E045F21E40C0F637
:10976000020040F21F1114F0E7F9FFE70298807E33
:1097700028B1FFE70298807E012801D1FFE708E0C9
:1097800045F21E40C0F602004FF4907114F0D4F977
:10979000FFE70298C07E28B1FFE70298C07E01284B
:1097A00001D1FFE708E045F21E40C0F6020040F29A
:1097B000211114F0C1F9FFE70298007F28B1FFE7FB
:1097C0000298007F012801D1FFE708E045F21E4022
:1097D000C0F602004FF4917114F0AEF9FFE7029861
:1097E000407F28B1FFE70298407F012801D1FFE7C1
:1097F00008E045F21E40C0F6020040F2231114F0CA
:109800009BF9FFE70298806890B1FFE702988068B3
:10981000B0F1804F0CD0FFE702988068B0F1004FA4
:1098200006D0FFE702988068B0F1404F01D1FFE712
:1098300008E045F21E40C0F602004FF4927114F0A9
:109840007BF9FFE70298C06890B1FFE70298C06813
:10985000B0F1807F0CD0FFE70298C068B0F1007FC4
:1098600006D0FFE70298C068B0F1407F01D1FFE762
:1098700008E045F21E40C0F6020040F2251114F047
:109880005BF9FFE70298006900285AD0FFE70298C9
:109890000069B0F5803F54D0FFE702980069B0F549
:1098A000003F4ED0FFE702980069B0F5403F48D036
:1098B000FFE702980069B0F5802F42D0FFE70298D9
:1098C0000069B0F5A02F3CD0FFE702980069B0F521
:1098D000C02F36D0FFE702980069B0F5E02F30D0F6
:1098E000FFE702980069B0F5002F2AD0FFE7029841
:1098F0000069B0F5102F24D0FFE702980069B0F599
:10990000202F1ED0FFE702980069B0F5302F18D045
:10991000FFE702980069B0F5402F12D0FFE70298E8
:109920000069B0F5502F0CD0FFE702980069B0F540
:10993000602F06D0FFE702980069B0F5702F01D1C3
:10994000FFE708E045F21E40C0F602004FF49371B5
:1099500014F0F2F8FFE70298406950B3FFE702986D
:109960004069B0F5801F24D0FFE702984069B0F548
:10997000001F1ED0FFE702984069B0F5401F18D0C5
:10998000FFE702984069B0F5800F12D0FFE7029818
:109990004069B0F5A00F0CD0FFE702984069B0F520
:1099A000C00F06D0FFE702984069B0F5E00F01D183
:1099B000FFE708E045F21E40C0F6020040F2271122
:1099C00014F0BAF8FFE70298406838B1FFE7029850
:1099D0004068B0F5806F01D8FFE708E045F21E400F
:1099E000C0F602004FF4947114F0A6F8FFE7029855
:1099F00090F8200020B9FFE7029800F0DDF8FFE7BB
:109A000002980168086820F00200086001F028FF51
:109A10000190FFE70298006840688007002815D58C
:109A2000FFE701F01DFF0199401A0B280DD3FFE756
:109A30000299486A40F4003048620299052081F892
:109A4000200001208DF80F00B2E0E3E702980168E2
:109A5000086840F00100086001F002FF0190FFE794
:109A6000029800684068C007A8B9FFE701F0F8FE57
:109A70000199401A0B280DD3FFE70299486A40F478
:109A8000003048620299052081F8200001208DF8FD
:109A90000F008DE0E4E70298007E012807D1FFE780
:109AA00002980168086840F08000086006E00298AB
:109AB0000168086820F080000860FFE70298407E97
:109AC000012807D1FFE702980168086840F04000CC
:109AD000086006E002980168086820F0400008600D
:109AE000FFE70298807E012807D1FFE7029801680E
:109AF000086840F02000086006E0029801680868E5
:109B000020F020000860FFE70298C07E012807D1FE
:109B1000FFE702980168086820F01000086006E07E
:109B200002980168086840F010000860FFE702989A
:109B3000007F012807D1FFE702980168086840F01C
:109B40000800086006E002980168086820F0080034
:109B50000860FFE70298407F012807D1FFE70298DD
:109B60000168086840F00400086006E00298016897
:109B7000086820F004000860FFE7029B19685A6833
:109B80009868D3F80CC040EA0C00D3F810C040EA43
:109B90000C005B691843013A1043C8610299002028
:109BA0004862029A012182F820108DF80F00FFE729
:109BB0009DF80F0004B080BD80B594B013900020D4
:109BC0001290119010900F900E901398006846F22A
:109BD0000041C4F20001884253D1FFE740F21C501B
:109BE000C2F200000168013101600068012812D151
:109BF000FFE7FFE700200D9043F64000C4F20200AB
:109C0000016841F000710160006800F000700D9083
:109C10000D98FFE7FFE7FFE700200C9043F63000C8
:109C2000C4F20200016841F008010160006800F020
:109C300008000C900C98FFE703200E9002210F9172
:109C400000210791109111900920129040F60040D8
:109C5000C4F202000EA901F00DFA079A1420059033
:109C60000521069102F018FA059802F0FDF906990F
:109C7000079A1520089002F00FFA089802F0F4F9FC
:109C80006EE01398006846F60001C4F200018842B5
:109C900065D1FFE7FFE700200B9043F64000C4F2D8
:109CA0000200016841F080610160006800F080609E
:109CB0000B900B98FFE740F21C50C2F200000168C5
:109CC000013101600068012812D1FFE7FFE70020A1
:109CD0000A9043F64000C4F20200016841F00071AE
:109CE0000160006800F000700A900A98FFE7FFE743
:109CF000FFE70020099043F63000C4F2020001683B
:109D000041F002010160006800F00200099009982A
:109D1000FFE760200E9002200F900020039010902B
:109D2000032011900920129040F20040C4F202007A
:109D30000EA901F09FF9039A40200190052102919C
:109D400002F0AAF9019802F08FF90299039A4120D2
:109D5000049002F0A1F9049802F086F9FFE7FFE70A
:109D600014B080BD80B582B001900198F9F7F2FD82
:109D70008DF803009DF80300032819D0FFE79DF834
:109D8000030040F25842C2F20002342110FB0120CD
:109D9000C06960B1FFE79DF8030040F25842C2F28B
:109DA0000002342110FB0120C0698047FFE7FFE774
:109DB00002B080BD80B582B001900198F9F7CAFD6C
:109DC0008DF803009DF80300032819D0FFE79DF8E4
:109DD000030040F25842C2F20002342110FB01207D
:109DE000806960B1FFE79DF8030040F25842C2F27B
:109DF0000002342110FB012080698047FFE7FFE764
:109E000002B080BD80B582B001900198F9F7A2FD43
:109E10008DF803009DF80300032819D0FFE79DF893
:109E2000030040F25842C2F20002342110FB01202C
:109E3000406A60B1FFE79DF8030040F25842C2F269
:109E40000002342110FB0120406A8047FFE7FFE752
:109E500002B080BD80B582B001900198F9F77AFD1B
:109E60008DF803009DF80300032819D0FFE79DF843
:109E7000030040F25842C2F20002342110FB0120DC
:109E8000006A60B1FFE79DF8030040F25842C2F259
:109E90000002342110FB0120006A8047FFE7FFE742
:109EA00002B080BD80B582B001900198F9F752FDF3
:109EB0008DF803009DF80300032819D0FFE79DF8F3
:109EC000030040F25842C2F20002342110FB01208C
:109ED000806A60B1FFE79DF8030040F25842C2F289
:109EE0000002342110FB0120806A8047FFE7FFE772
:109EF00002B080BD80B584B00290029890F8200036
:109F000001282FD1FFE70299022081F82000029852
:109F10000168086820F00100086001F0A1FC0190D0
:109F2000FFE7029800684068C007A8B1FFE701F0AA
:109F300097FC0199401A0B280DD3FFE70299486A54
:109F400040F4003048620299052081F82000012089
:109F50008DF80F000FE0E4E70299002048628DF8C9
:109F60000F0008E00299486A40F40020486201208E
:109F70008DF80F00FFE79DF80F0004B080BD0000D2
:109F800080B582B001900198F9F7E4FC8DF80300E8
:109F90009DF80300032819D0FFE79DF8030040F265
:109FA0005842C2F20002342110FB0120C06860B1A7
:109FB000FFE79DF8030040F25842C2F2000234214C
:109FC00010FB0120C0688047FFE7FFE702B080BDBB
:109FD00080B582B001900198F9F7BCFC8DF80300C0
:109FE0009DF80300032817D0FFE79DF803003421F4
:109FF000414340F25840C2F20000405858B1FFE7D8
:10A000009DF803003421414340F25840C2F2000061
:10A0100040588047FFE7FFE702B080BD80B582B0BF
:10A0200001900198F9F796FC8DF803009DF8030064
:10A03000032819D0FFE79DF8030040F25842C2F20E
:10A040000002342110FB0120006960B1FFE79DF898
:10A05000030040F25842C2F20002342110FB0120FA
:10A0600000698047FFE7FFE702B080BD80B582B09E
:10A0700001900198F9F76EFC8DF803009DF803003C
:10A08000032819D0FFE79DF8030040F25842C2F2BE
:10A090000002342110FB0120406860B1FFE79DF809
:10A0A000030040F25842C2F20002342110FB0120AA
:10A0B00040688047FFE7FFE702B080BD80B582B00F
:10A0C00001900198F9F746FC8DF803009DF8030014
:10A0D000032819D0FFE79DF8030040F25842C2F26E
:10A0E0000002342110FB0120406960B1FFE79DF8B8
:10A0F000030040F25842C2F20002342110FB01205A
:10A1000040698047FFE7FFE702B080BD80B582B0BD
:10A1100001900198F9F71EFC8DF803009DF80300EB
:10A12000032819D0FFE79DF8030040F25842C2F21D
:10A130000002342110FB0120806860B1FFE79DF828
:10A14000030040F25842C2F20002342110FB012009
:10A1500080688047FFE7FFE702B080BD80B582B02E
:10A1600001900198F9F7F6FB8DF803009DF80300C4
:10A17000032819D0FFE79DF8030040F25842C2F2CD
:10A180000002342110FB0120C06A60B1FFE79DF896
:10A19000030040F25842C2F20002342110FB0120B9
:10A1A000C06A8047FFE7FFE702B080BD80B582B09C
:10A1B0000090009820B9FFE701208DF8070023E008
:10A1C0000098006843F20001C4F20201884201D104
:10A1D000FFE707E045F25640C0F60200682113F0A1
:10A1E000ABFCFFE70098407938B9FFE70099002001
:10A1F0000871009800F00CF8FFE700990120487101
:10A2000000208DF80700FFE79DF8070002B080BD31
:10A2100082B001900198006843F20001C4F202018B
:10A22000884212D1FFE7FFE70020009043F630009C
:10A23000C4F20200016841F480510160006800F43A
:10A24000805000900098FFE7FFE702B070470000E1
:10A2500080B584B002900298806D019001F000FBFF
:10A260000090029890F8350002280DD0FFE702997F
:10A2700080204865FFE70299002081F83400FFE75D
:10A2800001208DF80F0054E002980168086820F062
:10A290001600086002980168486920F08000486153
:10A2A0000298006C20B9FFE70298806C38B1FFE794
:10A2B00002980168086820F008000860FFE702982B
:10A2C0000168086820F001000860FFE70298006854
:10A2D0000068C007C0B1FFE701F0C2FA0099401A58
:10A2E000062810D3FFE7029920204865FFE702996E
:10A2F000002081F83400FFE70299032081F835003F
:10A300008DF80F0015E0E1E70298C16D3F2088400D
:10A3100001998860FFE70299002081F83400FFE787
:10A320000299012081F83500FFE700208DF80F0029
:10A33000FFE79DF80F0004B080BD000082B00090E0
:10A34000009890F83500022807D0FFE70099802098
:10A35000486501208DF807000EE00099052081F87E
:10A36000350000980168086820F001000860FFE7E8
:10A3700000208DF80700FFE79DF8070002B0704746
:10A3800080B586B005900020039040F22800C2F20C
:10A390000000006848F2B511C1F64E31A0FB011073
:10A3A000800A02900598806D0190019800680490E1
:10A3B00004980599C96DC840000700281AD5FFE721
:10A3C0000598006800684007002812D5FFE7059847
:10A3D0000168086820F0040008600598C16D082035
:10A3E0008840019988600599486D40F001004865F2
:10A3F000FFE7FFE704980599C96DC840C007A0B101
:10A40000FFE7059800684069000600280CD5FFE7C3
:10A410000598C16D01208840019988600599486DB3
:10A4200040F002004865FFE7FFE704980599C96D11
:10A43000C8404007002814D5FFE705980068006869
:10A44000800700280CD5FFE70598C16D04208840DF
:10A45000019988600599486D40F004004865FFE760
:10A46000FFE704980599C96DC840C006002847D584
:10A47000FFE7059800680068000700283FD5FFE760
:10A480000598C16D10208840019988600598006882
:10A490000068400300281AD5FFE7059800680068A7
:10A4A0000003002809D4FFE70598006C20B1FFE7FE
:10A4B0000598016C8847FFE708E00598806C20B19B
:10A4C000FFE70598816C8847FFE7FFE716E00598EE
:10A4D00000680068C005002807D4FFE705980168F8
:10A4E000086820F008000860FFE70598006C20B1BC
:10A4F000FFE70598016C8847FFE7FFE7FFE7FFE705
:10A5000004980599C96DC8408006002840F18D80E7
:10A51000FFE7059800680068C006002840F18480C5
:10A52000FFE70598C16D2020884001998860059853
:10A5300090F83500052834D1FFE7059801680868D0
:10A5400020F01600086005980168486920F0800036
:10A5500048610598006C20B9FFE70598806C38B118
:10A56000FFE705980168086820F008000860FFE729
:10A570000598C16D3F20884001998860FFE70599E3
:10A58000002081F83400FFE70599012081F83500AB
:10A590000598006D20B1FFE70598016D8847FFE73A
:10A5A0007BE0059800680068400300281AD5FFE7A3
:10A5B0000598006800680003002809D4FFE70598A3
:10A5C000406C20B1FFE70598416C8847FFE708E041
:10A5D0000598C06B20B1FFE70598C16B8847FFE77E
:10A5E000FFE720E0059800680068C005002811D446
:10A5F000FFE705980168086820F010000860FFE791
:10A600000599002081F83400FFE70599012081F8C1
:10A610003500FFE70598C06B20B1FFE70598C16BD7
:10A620008847FFE7FFE7FFE7FFE70598406DA0B326
:10A63000FFE70598406DC00730B3FFE70599052097
:10A6400081F8350005980168086820F0010008606D
:10A65000FFE70398013003900299884201D9FFE790
:10A6600007E0FFE7059800680068C0070028F0D100
:10A67000FFE7FFE70599002081F83400FFE705991F
:10A68000012081F83500FFE70598C06C20B1FFE795
:10A690000598C16C8847FFE7FFE706B080BD000062
:10A6A00080B586B004900020039001F0D9F80290A4
:10A6B000049820B9FFE701208DF8170087E204987D
:10A6C000006846F21001C4F20201884200F088805E
:10A6D000FFE70498006846F22801C4F202018842AC
:10A6E0007ED0FFE70498006846F24001C4F2020100
:10A6F000884275D0FFE70498006846F25801C4F21A
:10A70000020188426CD0FFE70498006846F27001AD
:10A71000C4F20201884263D0FFE70498006846F261
:10A720008801C4F2020188425AD0FFE70498006809
:10A7300046F2A001C4F20201884251D0FFE704981A
:10A74000006846F2B801C4F20201884248D0FFE72F
:10A750000498006846F21041C4F2020188423FD0DA
:10A76000FFE70498006846F22841C4F202018842DB
:10A7700036D0FFE70498006846F24041C4F2020177
:10A7800088422DD0FFE70498006846F25841C4F291
:10A790000201884224D0FFE70498006846F2704125
:10A7A000C4F2020188421BD0FFE70498006846F219
:10A7B0008841C4F20201884212D0FFE70498006881
:10A7C00046F2A041C4F20201884209D0FFE7049892
:10A7D000006846F2B841C4F20201884201D1FFE7A5
:10A7E00007E045F27330C0F60200B82113F0A4F977
:10A7F000FFE70498406850B3FFE704984068B0F161
:10A80000007F24D0FFE704984068B0F1806F1ED02D
:10A81000FFE704984068B0F1C06F18D0FFE70498D4
:10A820004068B0F1006F12D0FFE704984068B0F1C3
:10A83000206F0CD0FFE704984068B0F1406F06D05D
:10A84000FFE704984068B0F1606F01D1FFE707E0CF
:10A8500045F27330C0F60200B92113F06DF9FFE73D
:10A860000498806850B1FFE704988068402805D0BC
:10A87000FFE704988068802801D1FFE707E045F2F0
:10A880007330C0F60200BA2113F056F9FFE70498BE
:10A89000C068B0F5007F04D0FFE70498C06808B92D
:10A8A000FFE707E045F27330C0F60200BB2113F06A
:10A8B00043F9FFE704980069B0F5806F04D0FFE723
:10A8C0000498006908B9FFE707E045F27330C0F665
:10A8D0000200BC2113F030F9FFE70498406960B131
:10A8E000FFE704984069B0F5006F06D0FFE70498D1
:10A8F0004069B0F5805F01D1FFE707E045F27330B2
:10A90000C0F60200BD2113F017F9FFE70498806933
:10A9100060B1FFE704988069B0F5005F06D0FFE7FB
:10A9200004988069B0F5804F01D1FFE707E045F258
:10A930007330C0F60200BE2113F0FEF8FFE7049862
:10A94000C06958B1FFE70498C069B0F5807F05D0B1
:10A95000FFE70498C069202801D1FFE707E045F22E
:10A960007330C0F60200BF2113F0E6F8FFE7049849
:10A97000006A90B1FFE70498006AB0F5803F0CD000
:10A98000FFE70498006AB0F5003F06D0FFE704989F
:10A99000006AB0F5403F01D1FFE707E045F27330B0
:10A9A000C0F60200C02113F0C7F8FFE70498406A20
:10A9B00028B1FFE70498406A042801D1FFE707E0C7
:10A9C00045F27330C0F60200C12113F0B5F8FFE77D
:10A9D0000498406A00285BD0FFE70498806A78B149
:10A9E000FFE70498806A01280AD0FFE70498806A8C
:10A9F000022805D0FFE70498806A032801D1FFE709
:10AA000007E045F27330C0F60200C62113F094F857
:10AA1000FFE70498C06A90B1FFE70498C06AB0F5F8
:10AA2000000F0CD0FFE70498C06AB0F1807F06D019
:10AA3000FFE70498C06AB0F1C07F01D1FFE707E0EB
:10AA400045F27330C0F60200C72113F075F8FFE736
:10AA50000498006B90B1FFE70498006BB0F5001FFD
:10AA60000CD0FFE70498006BB0F5800F06D0FFE72D
:10AA70000498006BB0F5C00F01D1FFE707E045F285
:10AA80007330C0F60200C82113F056F8FFE7FFE765
:10AA9000FFE70499002081F83400FFE704990220C1
:10AAA00081F8350004980168086820F0010008600A
:10AAB000FFE7049800680068C00790B1FFE700F066
:10AAC000CFFE0299401A06280AD3FFE704992020F6
:10AAD00048650499032081F835008DF8170076E069
:10AAE000E7E70498006800680390039848F23F0184
:10AAF000CFF2100108400390049900914868D1F802
:10AB000008C0CB680A6940EA0C00184310434A6940
:10AB100010438A691043CA691043096A01430398C4
:10AB2000084303900498406A042808D1FFE7049979
:10AB3000C86A096B0143039808430390FFE7039831
:10AB400004990968086004980068406903900398B4
:10AB500020F0070003900498416A0398084303908B
:10AB60000498406A04281AD1FFE70498816A039880
:10AB7000084303900498C06A80B1FFE70498FCF78B
:10AB800075F850B1FFE70499402048650499012009
:10AB900081F835008DF8170019E0FFE7FFE703980B
:10ABA0000499096848610498FCF734F80190049806
:10ABB000C16D3F2088400199886004990020486554
:10ABC000049A012182F835108DF81700FFE79DF8EF
:10ABD000170006B080BD000080B588B006900591D2
:10ABE0000492039300208DF80B000698806D01906D
:10ABF000039828B1FFE7BDF80E0008B9FFE708E0A9
:10AC000045F27330C0F602004FF4E67112F094FF83
:10AC1000FFE7FFE7069890F83400012804D1FFE72A
:10AC200002208DF81F0045E00699012081F83400CC
:10AC3000FFE7FFE7069890F8350001282BD1FFE7E2
:10AC40000699022081F8350006990020486506988B
:10AC50000599049A039BFCF781F80698C16D3F2083
:10AC600088400199886006980168086840F01600DD
:10AC700008600698006C38B1FFE70698016808681C
:10AC800040F008000860FFE706980168086840F097
:10AC90000100086009E0FFE70699002081F8340010
:10ACA000FFE702208DF80B00FFE79DF80B008DF801
:10ACB0001F00FFE79DF81F0008B080BD80B584B07D
:10ACC000039000F0CDFD02900398019001980130AF
:10ACD00048B1FFE740F24040C2F20000017801981D
:10ACE00008440190FFE7FFE700F0BAFD0299401A1F
:10ACF0000199884201D2FFE7F6E704B080BD000069
:10AD000080B586B00490039101208DF80B000020DF
:10AD10000190FFE742F28060C2F20000007E01284D
:10AD200004D1FFE702208DF8170094E042F2806121
:10AD3000C2F2000101200876FFE7FFE704980068EF
:10AD400028B1FFE704980068012801D1FFE707E078
:10AD500045F2FD20C0F60200AB2112F0EDFEFFE748
:10AD60004CF25030FCF7A8FC8DF80B009DF80B005E
:10AD7000002863D1FFE703994FF0FF300860049883
:10AD80000068012814D1FFE70499087C4968FCF7A2
:10AD9000D3FA4CF25030FCF78FFC8DF80B0043F6E1
:10ADA0001041C4F20201086820F00400086042E08B
:10ADB00004988168C068084440B1FFE7049881683E
:10ADC000C06808440C2801D8FFE707E045F2FD20E1
:10ADD000C0F60200C32112F0AFFEFFE704988068BE
:10ADE0000190FFE7019804998A68C9681144884274
:10ADF00020D2FFE701980499097CFCF7B1F94CF2E5
:10AE00005030FCF759FC8DF80B0043F61041C4F2AA
:10AE10000201086820F0FA0008609DF80B0020B1DC
:10AE2000FFE701980399086004E0FFE7019801300B
:10AE30000190D7E7FFE7FCF72DFAFFE7FFE742F2C3
:10AE40008061C2F2000100200876FFE79DF80B0048
:10AE50008DF81700FFE79DF8170006B080BD0000D1
:10AE600043F61041C4F20201086840F00040086057
:10AE70000020704780B588B0069005910393029238
:10AE800001208DF80700FFE742F28060C2F2000067
:10AE9000007E012804D1FFE702208DF81F0069E041
:10AEA00042F28061C2F2000101200876FFE7FFE76D
:10AEB000069860B1FFE70698012808D0FFE70698DA
:10AEC000022804D0FFE70698032801D1FFE707E036
:10AED00045F2C320C0F60200A42112F02DFEFFE7C8
:10AEE0004CF25030FCF7E8FB8DF807009DF80700A6
:10AEF00098BBFFE7069830B9FFE705989DF8081062
:10AF0000FCF760FA1AE00698012806D1FFE70598D9
:10AF1000BDF80810FCF7D8FA0FE00698022805D112
:10AF2000FFE705980299FCF70FFB05E00598029AE8
:10AF3000039BFCF785FAFFE7FFE7FFE74CF2503091
:10AF4000FCF7BAFB8DF8070043F61041C4F202018A
:10AF5000086820F001000860FFE7FFE742F2806127
:10AF6000C2F2000100200876FFE79DF807008DF887
:10AF70001F00FFE79DF81F0008B080BD81B00020D2
:10AF80008DF8030043F61040C4F202000068C00FC1
:10AF9000D8B1FFE743F60441C4F2020140F22310A6
:10AFA000C4F26750086048F6AB10CCF6EF5008606A
:10AFB00043F61040C4F202000068C00F20B1FFE762
:10AFC00001208DF80300FFE7FFE79DF8030001B0C3
:10AFD0007047000080B582B0ADF8060000208DF803
:10AFE0000500FFE79DF805000F2824DCFFE7BDF80A
:10AFF00006009DF80510C840C007A8B1FFE79DF8FE
:10B00000051040F2DC40C2F2000050F8210050B1BF
:10B01000FFE79DF8051040F2DC40C2F2000050F856
:10B0200021008047FFE7FFE7FFE79DF805000130BB
:10B030008DF80500D6E702B080BD000080B582B073
:10B04000ADF8060043F61440C4F201000068BDF8F4
:10B05000061008420CD0FFE7BDF8060043F6144185
:10B06000C4F201010860BDF80600FFF7B3FFFFE777
:10B0700002B080BD80B58EB00D900C9100200A907A
:10B08000099008900D980021C4F20201884240D036
:10B09000FFE70D9840F20041C4F20201884238D027
:10B0A000FFE70D9840F60001C4F20201884230D05B
:10B0B000FFE70D9840F60041C4F20201884228D013
:10B0C000FFE70D9841F20001C4F20201884220D04E
:10B0D000FFE70D9841F20041C4F20201884218D006
:10B0E000FFE70D9841F60001C4F20201884210D03A
:10B0F000FFE70D9841F60041C4F20201884208D0F2
:10B10000FFE70D9842F20001C4F20201884201D12A
:10B11000FFE707E045F23A30C0F60200AC2112F03A
:10B120000BFDFFE70C98008828B1FFE70C984088DA
:10B1300008B9FFE707E045F23A30C0F60200AD215A
:10B1400012F0FAFCFFE70C984068002849D0FFE7AE
:10B150000C984068012844D0FFE70C9840681128FB
:10B160003FD0FFE70C98406802283AD0FFE70C98E0
:10B170004068122835D0FFE70C9840680021C1F2E2
:10B18000110188422DD0FFE70C9840680021C1F2E0
:10B190002101884225D0FFE70C9840680021C1F2C8
:10B1A000310188421DD0FFE70C9840680021C1F2B0
:10B1B0001201884215D0FFE70C9840680021C1F2C7
:10B1C000220188420DD0FFE70C9840680021C1F2AF
:10B1D0003201884205D0FFE70C984068032801D16E
:10B1E000FFE707E045F23A30C0F60200AE2112F068
:10B1F000A3FCFFE70C98806850B1FFE70C988068CB
:10B20000012805D0FFE70C988068022801D1FFE7EC
:10B2100007E045F23A30C0F60200AF2112F08CFC94
:10B22000FFE700200B90FFE70B980F2800F2B08299
:10B23000FFE70B99012088400A900C9800680A9952
:10B240000840099009980A99884240F09C82FFE7DB
:10B250000C98406800F00300012807D0FFE70C9825
:10B26000406800F0030002284BD1FFE70C98C0684B
:10B2700078B1FFE70C98C06801280AD0FFE70C9866
:10B28000C068022805D0FFE70C98C068032801D1E8
:10B29000FFE707E045F23A30C0F60200C12112F0A4
:10B2A0004BFCFFE70D98806808900B984100032045
:10B2B00000FA01F10898884308900C98C0680B992F
:10B2C000490000FA01F108980843089008980D9980
:10B2D00088600D98406808900B99012000FA01F1F0
:10B2E0000898884308900C984068C0F300100B99A8
:10B2F00000FA01F108980843089008980D994860F1
:10B30000FFE70C98406800F00300032818D0FFE71F
:10B310000D98C06808900B984100032000FA01F1D5
:10B320000898884308900C9880680B99490000FAA7
:10B3300001F108980843089008980D99C860FFE744
:10B340000C98406800F00300022840F0EE80FFE710
:10B350000C980069002800F0B980FFE70C9800699C
:10B36000092800F0B380FFE70C980069002800F07E
:10B37000AD80FFE70C980069002800F0A780FFE788
:10B380000C980069002800F0A180FFE70C98006984
:10B39000002800F09B80FFE70C980069012800F06E
:10B3A0009580FFE70C980069012800F08F80FFE787
:10B3B0000C980069022800F08980FFE70C9800696A
:10B3C000022800F08380FFE70C98006902287DD0F6
:10B3D000FFE70C980069032878D0FFE70C98006914
:10B3E000042873D0FFE70C98006904286ED0FFE7AB
:10B3F0000C980069042869D0FFE70C9800690528BB
:10B4000064D0FFE70C98006905285FD0FFE70C982F
:10B41000006909285AD0FFE70C980069062855D022
:10B42000FFE70C980069092850D0FFE70C980069E5
:10B4300007284BD0FFE70C980069072846D0FFE7A4
:10B440000C980069072841D0FFE70C98006908288C
:10B450003CD0FFE70C980069082837D0FFE70C982C
:10B460000069082832D0FFE70C98006909282DD020
:10B47000FFE70C980069092828D0FFE70C980069BD
:10B480000A2823D0FFE70C9800690A281ED0FFE79E
:10B490000C9800690B2819D0FFE70C9800690C285C
:10B4A00014D0FFE70C9800690C280FD0FFE70C9828
:10B4B00000690D280AD0FFE70C9800690C2805D018
:10B4C000FFE70C9800690F2801D1FFE707E045F27C
:10B4D0003A30C0F60200DC2112F02EFBFFE70D9897
:10B4E0000B996FF0030202EA51010844006A0890C8
:10B4F0000B9800F0070081000F2000FA01F1089876
:10B50000884308900C9800690B9901F007018900A5
:10B5100000FA01F108980843089008980D990B9BD0
:10B5200002EA530211440862FFE70D980068089090
:10B530000B984100032000FA01F108988843089015
:10B540000C98406800F003000B99490000FA01F1E3
:10B5500008980843089008980D9908600C98C079DD
:10B56000C006002840F10E81FFE7FFE700200790AA
:10B5700043F64400C4F20200016841F480410160D6
:10B58000006800F4804007900798FFE70B9820F0D0
:10B59000030043F60801C4F20101405808900B98DB
:10B5A00000F0030081000F2000FA01F108988843A1
:10B5B00008900D980021C4F20201884203D1FFE7F0
:10B5C000002006905EE00D9840F20041C4F20201B6
:10B5D000884203D1FFE70120059050E00D9840F626
:10B5E0000001C4F20201884203D1FFE70220049067
:10B5F00042E00D9840F60041C4F20201884203D1B6
:10B60000FFE70320039034E00D9841F20001C4F2FB
:10B610000201884203D1FFE70420029026E00D9842
:10B6200041F20041C4F20201884203D1FFE7052044
:10B63000019018E00D9841F60001C4F20201884221
:10B6400003D1FFE7062000900AE00D9941F6004281
:10B65000C4F202020820914208BF07200090FFE7D1
:10B6600000980190FFE701980290FFE7029803908D
:10B67000FFE703980490FFE704980590FFE705981B
:10B680000690FFE70698C0B20B9901F0030189000C
:10B6900000FA01F108980843089008980B9921F0E6
:10B6A000030143F60802C4F20102885043F6004049
:10B6B000C4F201000068089009990898884308902E
:10B6C0000C988079C00728B1FFE7099908980843CA
:10B6D0000890FFE7089843F60041C4F201010860B2
:10B6E00043F60440C4F201000068089009990898E4
:10B6F000884308900C9880798007002805D5FFE7DB
:10B700000999089808430890FFE7089843F6044110
:10B71000C4F20101086043F60840C4F20100006869
:10B72000089009990898884308900C988079C00679
:10B73000002805D5FFE70999089808430890FFE716
:10B74000089843F60841C4F20101086043F60C4032
:10B75000C4F201000068089009990898884308908D
:10B760000C9880798006002805D5FFE7099908988C
:10B7700008430890FFE7089843F60C41C4F2010122
:10B780000860FFE7FFE7FFE70B9801300B904BE500
:10B790000EB080BD80B582B00190ADF80210BDF84A
:10B7A000020020B1FFE7002008B9FFE708E045F2FA
:10B7B0003A30C0F602004FF4BD7112F0BDF9FFE758
:10B7C00001980069BDF80210084204D0FFE701208B
:10B7D0008DF8010003E000208DF80100FFE79DF8DF
:10B7E000010002B080BD000080B582B00190ADF8CC
:10B7F00002108DF80120BDF8020020B1FFE7002003
:10B8000008B9FFE708E045F23A30C0F6020040F21E
:10B810009B1112F091F9FFE79DF8010028B1FFE7B5
:10B820009DF80100012801D1FFE708E045F23A3018
:10B83000C0F602004FF4CE7112F07EF9FFE79DF8DA
:10B84000010028B1FFE7BDF802000199886105E019
:10B85000BDF80200000401998861FFE702B080BDD5
:10B8600049F6FC20C2F200000068704780B58EB037
:10B870000C900C9820B9FFE701208DF8370002E208
:10B880000C98006845F20041C4F20001884212D0D1
:10B89000FFE70C98006845F60001C4F200018842F9
:10B8A00009D0FFE70C98006845F60041C4F200019A
:10B8B000884201D1FFE708E045F28E40C0F6020061
:10B8C00040F2BF1112F038F9FFE70C98406850B110
:10B8D000FFE70C98406841F68021C0F206018842DB
:10B8E00001D8FFE708E045F28E40C0F602004FF4B1
:10B8F000E07112F021F9FFE70C98806830B1FFE7A2
:10B900000C988068B0F5804F01D1FFE708E045F260
:10B910008E40C0F6020040F2C11112F00DF9FFE7AF
:10B920000C98C068800A08B9FFE708E045F28E402D
:10B93000C0F602004FF4E17112F0FEF8FFE70C9838
:10B940000069B0F5804F06D0FFE70C980069B0F5AC
:10B95000404F01D1FFE708E045F28E40C0F60200FB
:10B9600040F2C31112F0E8F8FFE70C98406928B1E3
:10B97000FFE70C984069012801D1FFE708E045F294
:10B980008E40C0F602004FF4E27112F0D5F8FFE7E6
:10B990000C9880696FF0FE01084201D1FFE708E0D2
:10B9A00045F28E40C0F6020040F2C51112F0C4F814
:10B9B000FFE70C98C06928B1FFE70C98C0694028E0
:10B9C00001D1FFE708E045F28E40C0F602004FF4D7
:10B9D000E37112F0B1F8FFE70C98006A28B1FFE7B5
:10B9E0000C98006A802801D1FFE708E045F28E40FC
:10B9F000C0F6020040F2C71112F09EF8FFE70C9863
:10BA000090F83D0040B9FFE70C99002081F83C0018
:10BA10000C9800F03DF9FFE70C99242081F83D00D7
:10BA20000C980168086820F0010008600C98016813
:10BA3000086840F4004008600C980168086820F429
:10BA40000040086001F054FE0A900C98406848F2EB
:10BA5000A061C0F2010188420BD8FFE70A9948F2C1
:10BA60008042C0F21E020020914238BF012009909E
:10BA70000AE00A9940F60012C0F23D02002091420D
:10BA800038BF01200990FFE70998012804D1FFE79A
:10BA900001208DF83700F6E00A984DF68361C4F274
:10BAA0001B31A0FB0110800C0B900C9800684068C3
:10BAB00020F03F000B9908430C99096848600C98E6
:10BAC0000068006A20F03F0008900C98406848F237
:10BAD000A061C0F20101884204D8FFE70B98013051
:10BAE00007900EE00B984FF49671484344F6D351FB
:10BAF000C1F26201A0FB0101012000EB911007904F
:10BB0000FFE70898079908430C99096808620C98A0
:10BB10000068C0694CF6FF71884306900C98406835
:10BB200048F2A061C0F2010188421FD8FFE70A98DD
:10BB300001380C9949684900B0FBF1F001306FF30E
:10BB40001F30032803D8FFE7042005900BE00A9874
:10BB500001380C9949684900B0FBF1F001306FF3EE
:10BB60001F300590FFE7059804904CE00C98806822
:10BB700068B9FFE70A9801380C99496801EB41015F
:10BB8000B0FBF1F001306FF31F3003900DE00A9825
:10BB900001380C99496819225143B0FBF1F001308A
:10BBA000042161F31F300390FFE70398000518B9E3
:10BBB000FFE70120029023E00C98806868B9FFE756
:10BBC0000A9801380C99496801EB4101B0FBF1F08A
:10BBD00001306FF31F3001900DE00A9801380C9985
:10BBE000496819225143B0FBF1F00130042161F39F
:10BBF0001F300190FFE7019840F400400290FFE7FA
:10BC000002980490FFE70698049908430C99096884
:10BC1000C8610C980068006820F0C0000C9B19688F
:10BC2000DA691B6A1A43104308600C980068806840
:10BC300048F2FF3188430C9A1168D36812691A439D
:10BC4000104388600C980068C06820F0FF000C9BCF
:10BC500019685A699B691A431043C8600C980168B7
:10BC6000086840F0010008600C99002008640C9AF4
:10BC7000202182F83D100C9908630C9981F83E0050
:10BC80008DF83700FFE79DF837000EB080BD00004B
:10BC900080B594B0139000201290119010900F90E6
:10BCA0000E901398006845F20041C4F200018842EA
:10BCB00035D1FFE7FFE700200D9043F63000C4F2D6
:10BCC0000200016841F002010160006800F002001A
:10BCD0000D900D98FFE74FF440700E9012200F90DA
:10BCE00001201090032011900420129040F2004097
:10BCF000C4F202000EA9FFF7BDF9FFE700200C9087
:10BD000043F64000C4F20200016841F400110160F2
:10BD1000006800F400100C900C98FFE7FBE013980B
:10BD2000006845F60001C4F2000188425FD1FFE7D8
:10BD3000FFE700200B9043F63000C4F202000168D8
:10BD400041F020010160006800F020000B900B988A
:10BD5000FFE703200E9012210F9101211091119005
:10BD60000420129041F20040C4F202000EA9FFF735
:10BD700081F9FFE700200A9043F64000C4F2020078
:10BD8000016841F480010160006800F480000A90BD
:10BD90000A98FFE741F62020C2F20000069046F222
:10BDA000B801C4F2020101604FF0606141604021BE
:10BDB00081600021C1604FF4806202614161816154
:10BDC000C1614FF4003202624162FEF769FC18B1B2
:10BDD000FFE7FBF7C1F9FFE7FFE7139841F62021E2
:10BDE000C2F20001416313988863FFE792E0139861
:10BDF000006845F60041C4F20001884240F08980A5
:10BE0000FFE7FFE70020099043F63000C4F202008C
:10BE1000016841F004010160006800F0040009902D
:10BE20000998FFE7FFE70020089043F63000C4F2CE
:10BE30000200016841F001010160006800F00100AA
:10BE400008900898FFE74FF400700E9012200190C0
:10BE50000F90012002901090032003901190042075
:10BE60000490129040F60000C4F202000EA9059161
:10BE7000FFF700F9DDF804C0029B039A04980599C6
:10BE80004FF4807ECDF838E0CDF83CC0109311928D
:10BE900012900020C4F20200FFF7ECF8FFE7002048
:10BEA000079043F64000C4F20200016841F400012B
:10BEB0000160006800F4000007900798FFE741F672
:10BEC0008020C2F20000009046F24001C4F202015C
:10BED00001604FF0C061416000218160C1604FF49A
:10BEE0008062026141618161C16101624162FEF76C
:10BEF000D7FB18B1FFE7FBF72FF9FFE7FFE7139830
:10BF000041F68021C2F20001816313988863FFE744
:10BF1000FFE7FFE7FFE714B080BD000040F24040BC
:10BF2000C2F20000027849F6FC21C2F20001086862
:10BF3000104408607047000080B543F60041C4F229
:10BF40000201086840F400700860086840F48060EE
:10BF50000860086840F480700860032000F0D0F8A2
:10BF60000F2000F005F800F03BF8002080BD000035
:10BF700080B582B0009040F22800C2F20000006854
:10BF800040F24041C2F200010A784FF47A71B1FBED
:10BF9000F2F1B0FBF1F003F005FB20B1FFE7012067
:10BFA0008DF8070018E000980F280DD8FFE70099DA
:10BFB0004FF0FF30002200F06FF8009840F244414B
:10BFC000C2F20001086003E001208DF8070003E0E1
:10BFD00000208DF80700FFE79DF8070002B080BD44
:10BFE00080B582B0FFE70020019043F64400C4F220
:10BFF0000200016841F480410160006800F4804063
:10C0000001900198FFE7FFE70020009043F6400011
:10C01000C4F20200016841F080510160006800F044
:10C02000805000900098FFE76FF001000F21002280
:10C0300000F032F802B080BD80B582B08DF8070004
:10C040009DF90700002801D4FFE707E045F2AB3077
:10C05000C0F60200CE2111F06FFDFFE79DF9070049
:10C0600011F0CCFC02B080BD80B582B08DF8070025
:10C070009DF90700002801D4FFE707E045F2AB3047
:10C08000C0F60200BE2111F057FDFFE79DF9070041
:10C0900011F0D0FC02B080BD80B586B08DF81700DD
:10C0A000049103920020029003980F2801D8FFE723
:10C0B00007E045F2AB30C0F60200AA2111F03CFDCA
:10C0C000FFE704980F2801D8FFE707E045F2AB30FF
:10C0D000C0F60200AB2111F02FFDFFE711F0C2FC0A
:10C0E00002909DF91700019002980499039A07F0B5
:10C0F000C5FE0146019811F0BDFC06B080BD0000F0
:10C1000080B582B001900198072810D0FFE7019810
:10C1100006280CD0FFE70198052808D0FFE7019812
:10C12000042804D0FFE70198032801D1FFE707E0C6
:10C1300045F2AB30C0F60200922111F0FDFCFFE7A2
:10C14000019811F0DBFC02B080BD000082B00190CC
:10C150008DF8031002B0704782B00190ADF8021064
:10C16000BDF80200019909684862002002B07047DA
:10C1700084B003908DF80B10ADF808200398006888
:10C18000406A00909DF80B0048B9FFE7BDF8081021
:10C19000009840EA014003990968886233E00398F7
:10C1A0000068816A009800EB1140009000208DF833
:10C1B0000700FFE79DF807009DF80B100139884242
:10C1C00013D2FFE7039800689DF8071000EB810089
:10C1D000D0F80411009800EB11400090FFE79DF8A3
:10C1E000070001308DF80700E4E7BDF8081000985B
:10C1F00040EA0140039909689DF80B2001EB820198
:10C20000C1F80001FFE7002004B0704780B582B09C
:10C2100001900198D0F804040FF054FB02B080BDE7
:10C2200080B582B001908DF80310019AD2F8040411
:10C230009DF80310C1EBC10302EB8302926C0FF077
:10C240001FFA02B080BD000080B582B001908DF869
:10C250000310019AD2F804049DF80310C1EBC10346
:10C2600002EB8302D2F808220FF0B0FA02B080BDD0
:10C2700080B582B001900198D0F804040FF028FB3B
:10C2800002B080BD80B584B002908DF807109DF893
:10C290000700000600280FD5FFE702989DF8071059
:10C2A00001F00F01C1EBC10100EB81003C300090B7
:10C2B0000099012048700FE002989DF8071001F0E6
:10C2C0000F01C1EBC10100EB810000F5FE70009091
:10C2D000009900204870FFE79DF8070000F00F006C
:10C2E00000990870FFE7029890F8BC03012804D178
:10C2F000FFE702208DF80F0014E00299012081F879
:10C30000BC03FFE7FFE702980068009910F0A4FA69
:10C31000FFE70299002081F8BC03FFE700208DF8B9
:10C320000F00FFE79DF80F0004B080BD80B584B01A
:10C3300002908DF807109DF8070000F00F00029999
:10C340004968884204D9FFE701208DF80F004DE0CD
:10C350009DF80700000600280FD5FFE702989DF81A
:10C36000071001F00F01C1EBC10100EB81003C306F
:10C3700000900099012048700FE002989DF8071086
:10C3800001F00F01C1EBC10100EB810000F5FE706F
:10C390000090009900204870FFE700990020887005
:10C3A0009DF8070000F00F0000990870FFE7029861
:10C3B00090F8BC03012804D1FFE702208DF80F009C
:10C3C00014E00299012081F8BC03FFE7FFE702981F
:10C3D0000068009910F0C4FDFFE70299002081F881
:10C3E000BC03FFE700208DF80F00FFE79DF80F006A
:10C3F00004B080BD82B001908DF8031001989DF8C3
:10C40000031001F00F01C1EBC10100EB8100D0F876
:10C41000140202B07047000080B586B004908DF819
:10C420000F10ADF80C208DF80B3000208DF80A00AD
:10C430009DF80F00000600280FD5FFE704989DF82F
:10C440000F1001F00F01C1EBC10100EB81003C3086
:10C4500001900199012048700FE004989DF80F1099
:10C4600001F00F01C1EBC10100EB810000F5FE708E
:10C470000190019900204870FFE79DF80F0000F03F
:10C480000F0001990870BDF80C00019988609DF8B3
:10C490000B000199C8700198407820B1FFE701991D
:10C4A0000878C880FFE79DF80B00022804D1FFE759
:10C4B000019900200871FFE7FFE7049890F8BC039A
:10C4C000012804D1FFE702208DF8170015E0049938
:10C4D000012081F8BC03FFE7FFE704980068019999
:10C4E00010F076F8FFE70499002081F8BC03FFE71D
:10C4F0009DF80A008DF81700FFE79DF8170006B0B9
:10C5000080BD000080B586B005908DF813100392B1
:10C51000029305989DF8131001F00F01C1EBC101C2
:10C5200000EB810000F5FE70019003980199C8604E
:10C530000298019948610199002088610199487029
:10C540009DF8130000F00F0001990870059800692C
:10C55000012804D1FFE7039801990861FFE79DF8DE
:10C560001300000738B9FFE7059A10680199127C9B
:10C5700010F0AEFB06E0059A10680199127C10F0ED
:10C5800093FDFFE7002006B080BD000080B584B0B9
:10C5900002908DF807109DF8070000F00F00029937
:10C5A0004968884204D9FFE701208DF80F0058E060
:10C5B0009DF80700000600280FD5FFE702989DF8B8
:10C5C000071001F00F01C1EBC10100EB81003C300D
:10C5D00000900099012048700DE002989DF8071026
:10C5E000C1EBC10100EB810000F5FE7000900099E5
:10C5F00000204870FFE70099012088709DF807002F
:10C6000000F00F0000990870FFE7029890F8BC0353
:10C61000012804D1FFE702208DF80F0021E00299E4
:10C62000012081F8BC03FFE7FFE70298006800994A
:10C6300010F0E6FC9DF80700000740B9FFE7029AFA
:10C640001068117C02F5717210F03AFCFFE7FFE709
:10C650000299002081F8BC03FFE700208DF80F004D
:10C66000FFE79DF80F0004B080BD000080B586B0E4
:10C6700005908DF813100392029305989DF81310FE
:10C6800001F00F01C1EBC10100EB81003C300190D2
:10C6900003980199C86002980199486101990020A6
:10C6A00088610199012048709DF8130000F00F0087
:10C6B0000199087005980069012804D1FFE70398E3
:10C6C00001990861FFE79DF81300000738B9FFE7FB
:10C6D000059A10680199127C10F0FAFA06E0059AA2
:10C6E00010680199127C10F0DFFCFFE7002006B013
:10C6F00080BD000080B58CB00B900B9800680A904C
:10C700000A9809900B98006810F000FF002840F08C
:10C710001A83FFE70B98006810F064FF08B9FFE781
:10C7200011E30B98006810F05DFF8007002807D523
:10C73000FFE70B980168486900F002004861FFE7D5
:10C740000B98006810F04EFFC006002862D5FFE786
:10C750000B980168886920F0100088610A98006AC7
:10C7600003900B98039901F00F01C1EBC10100EB9D
:10C77000810000F5FE700290039800F4F011022091
:10C78000B0EB514F23D1FFE7BDF80C0047F6F07135
:10C7900008421BD0FFE70A980299C968039AC2F3BE
:10C7A0000A1210F02DFF039847F6F07100EA01031A
:10C7B000029AD06800EB1310D060039800EA0102DF
:10C7C0000299886900EB12108861FFE71BE003986B
:10C7D00000F4F0110620B0EB514F12D1FFE70A9898
:10C7E0000B9901F57171082210F00AFF039847F6C2
:10C7F000F07100EA01020299886900EB1210886169
:10C8000000E0FFE7FFE70B980168886940F010003F
:10C810008861FFE70B98006810F0E4FE0003002831
:10C8200070D5FFE7002005900B98006810F088FE97
:10C830000790FFE70798002863D0FFE79DF81C00EA
:10C84000C007002856D0FFE70B9800689DF8141029
:10C8500010F0B0FE06909DF81800C00760B1FFE729
:10C860000998059900EB41110120C1F8080B0B98BC
:10C87000059907F087FBFFE79DF8180000070028DF
:10C880000CD5FFE70998059900EB41110820C1F884
:10C89000080B0B98059907F02FFBFFE79DF8180090
:10C8A000C006002808D5FFE70998059900EB41115B
:10C8B0001020C1F8080BFFE79DF81800800600283B
:10C8C00008D5FFE70998059900EB41112020C1F830
:10C8D000080BFFE79DF819008006002809D5FFE73F
:10C8E0000998059900EB41114FF40050C1F8080B6D
:10C8F000FFE7FFE70598013005900798400807908B
:10C9000098E7FFE70B98006810F06CFE40030028E2
:10C9100040F1AC80FFE70B98006810F0FFFD079036
:10C9200000200590FFE70798002800F09E80FFE7B1
:10C930009DF81C00C007002800F09080FFE70B98CE
:10C9400000689DF8141010F00DFE06909DF8180078
:10C95000C00700283ED0FFE7059800F00F01012036
:10C9600000FA01F10491049B099AD2F83418994312
:10C97000C2F834180999059A01EB4211C1F8080967
:10C980000B98006901281FD1FFE70B980599C1EBAF
:10C99000C10100EB81014A6C886C104488640598E1
:10C9A00088B9FFE70B980599C1EBC10100EB810045
:10C9B000006D40B9FFE70B99086801F5717201211C
:10C9C00010F07EFAFFE7FFE70B989DF81410FFF7D1
:10C9D00027FCFFE79DF818000007002808D5FFE7AF
:10C9E0000998059900EB41110820C1F80809FFE7F3
:10C9F0009DF81800C006002808D5FFE7099805999A
:10CA000000EB41111020C1F80809FFE79DF818005C
:10CA10004006002808D5FFE70998059900EB411169
:10CA20004020C1F80809FFE79DF81800800700289A
:10CA300008D5FFE70998059900EB41110220C1F8DC
:10CA40000809FFE79DF818000006002805D5FFE754
:10CA50000B98059907F088FBFFE7FFE70598013081
:10CA600005900798400807905DE7FFE70B9800687E
:10CA700010F0B8FDC00F00B3FFE70999D1F8040822
:10CA800020F00100C1F804080B9890F8F403012885
:10CA900008D1FFE70B98002180F8F4130B98FFF7FB
:10CAA00055FB03E00B9800F061FBFFE70B98016872
:10CAB000486900F000404861FFE70B98006810F0FB
:10CAC00091FD0005002811D5FFE70998D0F8080866
:10CAD000C00720B1FFE70B9800F0D6FBFFE70B98EB
:10CAE0000168486900F400604861FFE70B9800683E
:10CAF00010F078FDC004002840F19080FFE709990C
:10CB0000D1F8040820F00100C1F804080B9800686F
:10CB1000102110F0ABFC00200890FFE708980B995B
:10CB2000496888423BD2FFE70998089900EB411118
:10CB30004FF67F30C1F808090999089A01EB4212B3
:10CB4000D2F8001921F40011C2F800190999089AC5
:10CB500001EB4212D2F8001941F00061C2F800194D
:10CB60000999089A01EB4211C1F8080B0998089934
:10CB700000EB4111D1F8000B20F40010C1F8000BBC
:10CB80000998089900EB4111D1F8000B40F00060C2
:10CB9000C1F8000BFFE7089801300890BEE709993B
:10CBA000D1F81C0840F00110C1F81C080B98006B6C
:10CBB00078B1FFE70999D1F8840840F00B00C1F87B
:10CBC00084080999D1F8440840F00B00C1F84408E2
:10CBD0000FE00999D1F8140842F22B021043C1F872
:10CBE00014080999D1F8100840F00B00C1F810089A
:10CBF000FFE70999D1F8000820F4FE60C1F80008A9
:10CC00000B9A1068117C02F5717210F059F90B98AB
:10CC10000168486900F480504861FFE70B9800689C
:10CC200010F0E0FC800400281FD5FFE70B98006897
:10CC30000FF03EFD0B98006810F042FC0B99C860A5
:10CC40000B980068019000F04DFD014601980B9A89
:10CC5000127B10F05BFD0B9800F05EFA0B980168F8
:10CC6000486900F400504861FFE70B98006810F035
:10CC7000B9FC000700280AD5FFE70B9800F080FAFE
:10CC80000B980168486900F008004861FFE70B98BD
:10CC9000006810F0A7FCC00200280ED5FFE70020B6
:10CCA00005900B989DF8141000F050F80B9801684F
:10CCB000486900F480104861FFE70B98006810F0A5
:10CCC00091FC800200280ED5FFE7002005900B980C
:10CCD0009DF8141000F048F80B980168486900F4BA
:10CCE00000104861FFE70B98006810F07BFC4000E3
:10CCF00000280AD5FFE70B98FFF788FA0B98016820
:10CD0000486900F080404861FFE70B98006810F028
:10CD100069FC4007002815D5FFE70B9800684068BC
:10CD200003909DF80C004007002804D5FFE70B98FE
:10CD3000FFF79EFAFFE7039A0B98016848681043D3
:10CD40004860FFE7FFE70CB080BD000080B582B00F
:10CD500001908DF803100198D0F804049DF8031099
:10CD60000EF048FE02B080BD80B582B001908DF813
:10CD700003100198D0F804049DF803100EF066FE2D
:10CD800002B080BD2DE9F04F97B01590159820B9ED
:10CD9000FFE701208DF85B0060E115980068B0F1B5
:10CDA000A04F08D0FFE7159800680021C4F20401E5
:10CDB000884201D1FFE707E045F25320C0F60200A8
:10CDC000872110F0B9FEFFE71598006814901598B8
:10CDD00090F8BD0340B9FFE71599002081F8BC0326
:10CDE000159800F041F9FFE71599032081F8BD037C
:10CDF0001498C06BC005002804D4FFE715990020E3
:10CE00000861FFE7159800680FF058FF159810901B
:10CE10000168119141688268C368D0F810C0446904
:10CE20008569C669076AD0F82480D0F82890D0F8C0
:10CE30002CA0D0F830B0D0F834E068461290C0F89A
:10CE400024E01198DDF848E0CEF820B0CEF81CA020
:10CE5000CEF81890CEF81480CEF81070CEF80C6092
:10CE6000CEF80850CEF80440CEF800C00FF036FCE3
:10CE700040B1FFE71599022081F8BD0301208DF82C
:10CE80005B00EBE01598006800210F9110F0E0FBCB
:10CE90000F988DF84F00FFE79DF84F0015994968EE
:10CEA000884245D2FFE715989DF84F10C1EBC101AC
:10CEB00000EB8101012081F83D009DF84F0015999C
:10CEC000C0EBC00201EB820181F83C009DF84F00ED
:10CED0001599C0EBC00201EB8201A1F84200159840
:10CEE0009DF84F10C1EBC10100EB8101002081F8DA
:10CEF0003F0015999DF84F20C2EBC20201EB820161
:10CF0000486415999DF84F20C2EBC20201EB8201E3
:10CF1000886415999DF84F20C2EBC20201EB820193
:10CF20000865FFE79DF84F0001308DF84F00B3E72B
:10CF300000208DF84F00FFE79DF84F0015994968D4
:10CF400088423ED2FFE715989DF84F10C1EBC10112
:10CF500000EB8101002081F8FD019DF84F10159A2A
:10CF6000C1EBC10302EB830282F8FC1115999DF815
:10CF70004F20C2EBC20201EB820181F8FF0115993B
:10CF80009DF84F20C2EBC20201EB8201C1F80402FE
:10CF900015999DF84F20C2EBC20201EB8201C1F846
:10CFA000080215999DF84F20C2EBC20201EB8201E5
:10CFB000C1F81002FFE79DF84F0001308DF84F00D7
:10CFC000BAE715980C9001680D9141688268C368B2
:10CFD000D0F810C044698569C669076AD0F8248012
:10CFE000D0F82890D0F82CA0D0F830B0D0F834E0A9
:10CFF00068460E90C0F824E00D98DDF838E0CEF8D1
:10D0000020B0CEF81CA0CEF81890CEF81480CEF840
:10D010001070CEF80C60CEF80850CEF80440CEF870
:10D0200000C00FF0E9FC40B1FFE71599022081F83C
:10D03000BD0301208DF85B0010E0159900200B90D6
:10D0400081F838001599012081F8BD031598006812
:10D050000FF0BCFC0B988DF85B00FFE79DF85B00C0
:10D0600017B0BDE8F08F000080B58AB009900020AD
:10D070000890079006900590049009980068B0F118
:10D08000A04F47D1FFE7FFE70020039043F63000B1
:10D09000C4F20200016841F001010160006800F083
:10D0A000010003900398FFE74FF4C0500490022062
:10D0B000059000200690032007900A200890002089
:10D0C000C4F2020004A9FDF7D5FFFFE743F63401DF
:10D0D000C4F20201086840F080000860FFE7002009
:10D0E000029043F64400C4F20200016841F480411A
:10D0F0000160006800F4804002900298FFE7FFE7BB
:10D100004320019005210022FEF7C6FF0198FEF79B
:10D11000ABFFFFE70AB080BD80B582B0019001206F
:10D120008DF803000198C06820B9FFE700208DF852
:10D1300003000CE00198C068022804D1FFE7012039
:10D140008DF8030002E0FAF707F8FFE7FFE7019820
:10D15000D0F804049DF803100EF076FD0198D0F885
:10D1600004040EF0E7FC02B080BD000080B582B080
:10D1700001900198D0F804040EF02CFD02B080BD9F
:10D1800080B582B001900198D0F804040EF034FD0F
:10D1900002B080BD80B584B002908DF80710FFE723
:10D1A000029890F8BC03012804D1FFE702208DF813
:10D1B0000F001AE00299012081F8BC03FFE7FFE7A6
:10D1C0009DF80700029981F83800029800689DF8E0
:10D1D000071010F06DFAFFE70299002081F8BC03F8
:10D1E000FFE700208DF80F00FFE79DF80F0004B067
:10D1F00080BD000080B582B001900199D1F804048F
:10D2000001F571710EF04AFD02B080BD80B584B0A9
:10D210000290029800680190FFE7029890F8BC0322
:10D22000012804D1FFE702208DF80F0027E00299C2
:10D23000012081F8BC03FFE7FFE70298806A01281C
:10D240000BD1FFE702988069012806D0FFE701991A
:10D25000886B40F480308863FFE70298006810F024
:10D26000D5F8029800680FF09BFBFFE702990020B9
:10D2700081F8BC03FFE700208DF80F00FFE79DF861
:10D280000F0004B080BD000080B582B0019001980D
:10D29000D0F804040EF084FD01980168D1F8000E66
:10D2A00040F00100C1F8000E0198006A48B1FFE7A4
:10D2B0004EF61051CEF20001086840F006000860FA
:10D2C000FFE702B080BD000080B584B002900191FC
:10D2D000029820B9FFE701208DF80F00FDE10298C8
:10D2E000006830B1FFE7029800680F2801D8FFE717
:10D2F00008E045F28B20C0F602004FF4177110F0E1
:10D300001BFCFFE70198E0B1FFE70198012818D066
:10D31000FFE70198022814D0FFE70198032810D0F6
:10D32000FFE7019804280CD0FFE70198052808D0F2
:10D33000FFE70198062804D0FFE70198072801D1EC
:10D34000FFE708E045F28B20C0F6020040F25D21C5
:10D3500010F0F2FBFFE7019843F60041C4F202012E
:10D36000096801F00701884212D9FFE7019943F6E5
:10D370000040C4F202000170006800F0070001994B
:10D38000884204D0FFE701208DF80F00A5E1FFE7F8
:10D39000029800788007002860D5FFE7029800789F
:10D3A0004007002809D5FFE743F60801C4F202014F
:10D3B000086840F4E0500860FFE702980078000732
:10D3C000002809D5FFE743F60801C4F20201086806
:10D3D00040F460400860FFE70298806840B3FFE7D0
:10D3E00002988068802823D0FFE702988068902800
:10D3F0001ED0FFE702988068A02819D0FFE70298A6
:10D400008068B02814D0FFE702988068C0280FD049
:10D41000FFE702988068D0280AD0FFE7029880686A
:10D42000E02805D0FFE702988068F02801D1FFE7E7
:10D4300008E045F28B20C0F602004FF4207110F096
:10D440007BFBFFE743F60801C4F20201086820F005
:10D45000F000029A926810430860FFE70298007893
:10D46000C007002800F08C80FFE70298406878B180
:10D47000FFE70298406801280AD0FFE70298406859
:10D48000022805D0FFE702984068032801D1FFE792
:10D4900008E045F28B20C0F6020040F2872110F030
:10D4A0004BFBFFE702984068012811D1FFE743F6E4
:10D4B0000000C4F20200006800F400310020B0EB6C
:10D4C000514F04D1FFE701208DF80F0005E12CE05A
:10D4D00002984068022805D0FFE7029840680328B8
:10D4E00011D1FFE743F60000C4F20200006800F02B
:10D4F00000710020B0EB516F04D1FFE701208DF8DF
:10D500000F00EAE010E043F60000C4F202000068F9
:10D5100000F002010020B0EB510F04D1FFE7012021
:10D520008DF80F00D9E0FFE7FFE743F60801C4F2EA
:10D530000201086820F00300029A52681043086054
:10D54000FEF78EF90090FFE743F60800C4F20200F0
:10D55000006800F00C0002994968B0EB810F0ED012
:10D56000FFE7FEF77DF90099401A41F289318842C0
:10D5700004D3FFE703208DF80F00AEE0E4E7FFE7F8
:10D58000019843F60041C4F20201096801F0070165
:10D59000884212D2FFE7019943F60040C4F202002C
:10D5A0000170006800F007000199884204D0FFE78D
:10D5B00001208DF80F0090E0FFE702980078400707
:10D5C000002832D5FFE70298C068C0B1FFE7029893
:10D5D000C068B0F5805F12D0FFE70298C068B0F570
:10D5E000A05F0CD0FFE70298C068B0F5C05F06D01E
:10D5F000FFE70298C068B0F5E05F01D1FFE708E0FF
:10D6000045F28B20C0F6020040F2C52110F094FADA
:10D61000FFE743F60801C4F20201086820F4E05075
:10D62000029AD26810430860FFE70298007800076A
:10D63000002833D5FFE702980069C0B1FFE70298E0
:10D640000069B0F5805F12D0FFE702980069B0F57D
:10D65000A05F0CD0FFE702980069B0F5C05F06D06C
:10D66000FFE702980069B0F5E05F01D1FFE708E04D
:10D6700045F28B20C0F602004FF4337110F05CFAD3
:10D68000FFE743F60801C4F20201086820F4604095
:10D69000029A126940EAC2000860FFE700F04CF805
:10D6A00043F60801C4F202010968C9B20A0944F646
:10D6B000C031C0F60201895CC84040F22801C2F2C4
:10D6C0000001086040F24440C2F200000068FEF72A
:10D6D0004FFC00208DF80F00FFE79DF80F0004B00D
:10D6E00080BD000040F22800C2F2000000687047D0
:10D6F00080B5FFF7F7FF43F60801C4F2020109689D
:10D70000C1F3822244F6D031C0F60201895CC840E0
:10D7100080BD000080B5FFF7E5FF43F60801C4F2C5
:10D720000201096889B24A0B44F6D031C0F6020101
:10D73000895CC84080BD000080B586B0002005909F
:10D7400004900390029043F60800C4F202000068BF
:10D7500000F00C000146019140B1FFE70198042858
:10D760000AD0FFE7019808280CD04FE042F20040B1
:10D77000C0F2F40002904FE041F60030C0F2B70072
:10D78000029049E043F60400C4F20200016801F08F
:10D790003F01059100684002002813D5FFE743F6DA
:10D7A0000400C4F202000068C0F3881041F60031A2
:10D7B000C0F2B701A0FB0101059A0023F2F700FDBA
:10D7C000049012E043F60400C4F202000068C0F3C3
:10D7D000881042F20041C0F2F401A0FB0101059A59
:10D7E0000023F2F7EDFC0490FFE743F60400C4F2D7
:10D7F0000200006800F44031022000EBD1300390B9
:10D8000004980399B0FBF1F0029005E042F2004069
:10D81000C0F2F4000290FFE7029806B080BD00005D
:10D8200080B586B00490049828B9FFE701208DF8F0
:10D83000170000F048BC049800680F2801D8FFE7E3
:10D8400007E045F28B20C0F60200E82110F074F9E1
:10D85000FFE704980078C007002800F0BE80FFE7CB
:10D860000498406860B1FFE704984068B0F5803FD5
:10D8700006D0FFE704984068B0F5A02F01D1FFE77C
:10D8800007E045F28B20C0F60200ED2110F054F9BC
:10D89000FFE743F60800C4F20200006800F00C0045
:10D8A000042813D0FFE743F60800C4F20200006822
:10D8B00000F00C0008281ED1FFE743F60400C4F274
:10D8C000020000684002002815D5FFE743F600007B
:10D8D000C4F20200006800F400310020B0EB514FA8
:10D8E00008D0FFE70498406820B9FFE701208DF8D1
:10D8F0001700E8E370E0FFE704984068B0F5803F68
:10D9000009D1FFE743F60001C4F20201086840F4C0
:10D910008030086020E004984068B0F5A02F0DD159
:10D92000FFE743F60001C4F20201086840F48020DA
:10D930000860086840F4803008600CE043F600019D
:10D94000C4F20201086820F480300860086820F4FE
:10D9500080200860FFE7FFE7FFE704984068E8B130
:10D96000FFE7FDF77DFF0390FFE743F60000C4F2F9
:10D970000200006800F400310020B0EB514F0CD1E0
:10D98000FFE7FDF76DFF0399401A652804D3FFE711
:10D9900003208DF8170096E3E7E71CE0FDF760FF32
:10D9A0000390FFE743F60000C4F20200006800F4B1
:10D9B00000310020B0EB514F0CD0FFE7FDF750FFD6
:10D9C0000399401A652804D3FFE703208DF8170058
:10D9D00079E3E7E7FFE7FFE7FFE7049800788007D0
:10D9E000002840F1B880FFE70498C06828B1FFE73D
:10D9F0000498C068012801D1FFE708E045F28B20B8
:10DA0000C0F6020040F21F1110F096F8FFE70498EC
:10DA100000691F2801D8FFE708E045F28B20C0F617
:10DA200002004FF4907110F087F8FFE743F608000A
:10DA3000C4F20200006810F00C0F13D0FFE743F6A9
:10DA40000800C4F20200006800F00C0008282CD185
:10DA5000FFE743F60400C4F2020000684002002819
:10DA600023D4FFE743F60000C4F20200006800F090
:10DA700002010020B0EB510F09D0FFE70498C06805
:10DA8000012804D0FFE701208DF817001BE343F6BF
:10DA90000001C4F20201086820F0F800049A12693B
:10DAA00040EAC2000860FFE754E00498C06870B321
:10DAB000FFE70021C4F2472101200860FDF7D0FEF6
:10DAC0000390FFE743F60000C4F20200006800F094
:10DAD00002010020B0EB510F0CD1FFE7FDF7C0FEB3
:10DAE0000399401A032804D3FFE703208DF8170099
:10DAF000E9E2E7E743F60001C4F20201086820F01A
:10DB0000F800049A126940EAC200086021E000218E
:10DB1000C4F2472100200860FDF7A2FE0390FFE752
:10DB200043F60000C4F20200006800F00201002089
:10DB3000B0EB510F0CD0FFE7FDF792FE0399401AAE
:10DB4000032804D3FFE703208DF81700BBE2E7E7C3
:10DB5000FFE7FFE7FFE704980078000700285ED59D
:10DB6000FFE70498406928B1FFE70498406901285D
:10DB700001D1FFE708E045F28B20C0F602004FF428
:10DB8000B0710FF0D9FFFFE70498406918B3FFE7C1
:10DB900040F68061C4F2472101200860FDF760FE75
:10DBA0000390FFE743F67400C4F20200006800F03F
:10DBB00002010020B0EB510F0CD1FFE7FDF750FE42
:10DBC0000399401A032804D3FFE703208DF81700B8
:10DBD00079E2E7E722E040F68061C4F247210020C5
:10DBE0000860FDF73DFE0390FFE743F67400C4F2C2
:10DBF0000200006800F002010020B0EB510F0CD0D1
:10DC0000FFE7FDF72DFE0399401A032804D3FFE731
:10DC100003208DF8170056E2E7E7FFE7FFE70498D7
:10DC200000784007002840F1E680FFE700208DF8EB
:10DC300007000498806850B1FFE7049880680128C5
:10DC400005D0FFE704988068052801D1FFE708E0C8
:10DC500045F28B20C0F602004FF4C6710FF06CFF46
:10DC6000FFE743F64000C4F202000068C00000284D
:10DC700015D4FFE7FFE70020009043F64000C4F210
:10DC80000200016841F080510160006800F080509E
:10DC900000900098FFE701208DF80700FFE747F2AA
:10DCA0000000C4F200000068C005002822D4FFE78D
:10DCB00047F20001C4F20001086840F48070086077
:10DCC000FDF7CEFD0390FFE747F20000C4F200002D
:10DCD0000068C00500280CD4FFE7FDF7C1FD0399DB
:10DCE000401A032804D3FFE703208DF81700EAE168
:10DCF000EAE7FFE7FFE704988068012809D1FFE71A
:10DD000043F67001C4F20201086840F001000860A7
:10DD10001FE00498806805280DD1FFE743F67001E5
:10DD2000C4F20201086840F004000860086840F08E
:10DD3000010008600CE043F67001C4F202010868BB
:10DD400020F001000860086820F004000860FFE788
:10DD5000FFE7FFE704988068F8B1FFE7FDF780FD73
:10DD60000390FFE743F67000C4F20200006800F081
:10DD700002010020B0EB510F0ED1FFE7FDF770FD5F
:10DD80000399401A41F28931884204D3FFE7032006
:10DD90008DF8170097E1E5E71EE0FDF761FD0390C0
:10DDA000FFE743F67000C4F20200006800F00201D1
:10DDB0000020B0EB510F0ED0FFE7FDF751FD0399A6
:10DDC000401A41F28931884204D3FFE703208DF8DD
:10DDD000170078E1E5E7FFE79DF80700012809D182
:10DDE000FFE743F64001C4F20201086820F08050CA
:10DDF0000860FFE7FFE70498806950B1FFE70498E7
:10DE00008069012805D0FFE704988069022801D1C4
:10DE1000FFE708E045F28B20C0F6020040F2CF1188
:10DE20000FF08AFEFFE704988069002800F0478120
:10DE3000FFE743F60800C4F20200006800F00C009F
:10DE4000082800F0F080FFE704988069022840F07D
:10DE5000C780FFE70498C06930B1FFE70498C06944
:10DE6000B0F5800F01D1FFE708E045F28B20C0F646
:10DE700002004FF4EC710FF05FFEFFE70498006AB8
:10DE80003F2801D8FFE708E045F28B20C0F60200EA
:10DE900040F2D9110FF050FEFFE70498406A322893
:10DEA00007D3FFE70498406AB0F5D87F01D8FFE7B1
:10DEB00008E045F28B20C0F602004FF4ED710FF040
:10DEC0003BFEFFE70498806A02280FD0FFE7049822
:10DED000806A04280AD0FFE70498806A062805D0E3
:10DEE000FFE70498806A082801D1FFE708E045F2BF
:10DEF0008B20C0F6020040F2DB110FF01DFEFFE7A1
:10DF00000498C06A022806D3FFE70498C06A0F2865
:10DF100001D8FFE708E045F28B20C0F602004FF47D
:10DF2000EE710FF009FEFFE76021C4F247210020E7
:10DF30000860FDF795FC0390FFE743F60000C4F28C
:10DF40000200006800F000710020B0EB516F0CD0AF
:10DF5000FFE7FDF785FC0399401A032804D3FFE788
:10DF600003208DF81700AEE0E7E70499C869D1F8FF
:10DF700020C04B6A8A6A40EA0C0040EA8310D20350
:10DF80004FF6FF739A43A2F580321043C96A40EA04
:10DF9000016043F60401C4F2020108606021C4F28A
:10DFA000472101200860FDF75BFC0390FFE743F683
:10DFB0000000C4F20200006800F000710020B0EB25
:10DFC000516F0CD1FFE7FDF74BFC0399401A032872
:10DFD00004D3FFE703208DF8170074E0E7E721E0A2
:10DFE0006021C4F2472100200860FDF739FC03904E
:10DFF000FFE743F60000C4F20200006800F0007181
:10E000000020B0EB516F0CD0FFE7FDF729FC03991E
:10E01000401A032804D3FFE703208DF8170052E0CD
:10E02000E7E7FFE74AE004988069012804D1FFE7A9
:10E0300001208DF8170046E043F60400C4F2020008
:10E040000068029004988069012831D0FFE70298A7
:10E0500000F480000499C969884229D1FFE7029839
:10E0600000F03F000499096A884221D1FFE7029835
:10E0700047F6C07108400499496AB0EB811F17D177
:10E08000FFE7029800F440300499896AC9034FF60B
:10E09000FF729143A1F58031884209D1FFE70298D0
:10E0A00000F070600499C96AB0EB016F04D0FFE71B
:10E0B00001208DF8170006E0FFE7FFE7FFE70020EB
:10E0C0008DF81700FFE79DF8170006B080BD00002F
:10E0D00080B582B00090009820B9FFE701208DF84C
:10E0E00007002EE00098006840F60001C5F2060126
:10E0F000884201D1FFE707E045F2C640C0F60200C2
:10E10000A3210FF019FDFFE70098407938B9FFE728
:10E11000009900200871009800F018F8FFE70099B6
:10E120000220487100980168086840F00400086007
:10E130000099012048710099002088608DF807003F
:10E14000FFE79DF8070002B080BD000082B001909B
:10E150000198006840F60001C5F20601884212D11C
:10E16000FFE7FFE70020009043F63400C4F202000E
:10E17000016841F040010160006800F0400000903B
:10E180000098FFE7FFE702B07047000080B582B05B
:10E190000190019808F084FC8DF803009DF80300BD
:10E1A00003281BD0FFE7019808F07AFC014640F2F3
:10E1B000A050C2F2000000EB4110806968B1FFE797
:10E1C000019808F06DFC014640F2A050C2F2000038
:10E1D00000EB411080698047FFE7FFE702B080BD98
:10E1E00080B584B00290029820B9FFE701208DF835
:10E1F0000F00D2E10298006843F20001C4F201016D
:10E20000884212D0FFE70298006843F60001C4F28A
:10E210000001884209D0FFE70298006843F60041F8
:10E22000C4F20001884201D1FFE708E045F2FE4058
:10E23000C0F602004FF4A1710FF07EFCFFE70298D8
:10E24000406830B1FFE702984068B0F5827F01D1A5
:10E25000FFE708E045F2FE40C0F6020040F243113D
:10E260000FF06AFCFFE70298806860B1FFE7029850
:10E270008068B0F5806F06D0FFE702988068B0F53F
:10E28000004F01D1FFE708E045F2FE40C0F6020072
:10E290004FF4A2710FF050FCFFE70298C068B0F590
:10E2A000006F04D0FFE70298C06808B9FFE708E0F4
:10E2B00045F2FE40C0F6020040F245110FF03CFC72
:10E2C000FFE702988069B0F5007F0AD0FFE7029867
:10E2D000806930B1FFE702988069B0F5802F01D1E5
:10E2E000FFE708E045F2FE40C0F602004FF4A371DC
:10E2F0000FF022FCFFE70298C06918B3FFE702980D
:10E30000C06908281ED0FFE70298C069102819D0FC
:10E31000FFE70298C069182814D0FFE70298C06987
:10E3200020280FD0FFE70298C06928280AD0FFE70D
:10E330000298C069302805D0FFE70298C0693828E4
:10E3400001D1FFE708E045F2FE40C0F6020040F2CE
:10E3500047110FF0F1FBFFE70298006A28B1FFE7D1
:10E360000298006A802801D1FFE708E045F2FE40EC
:10E37000C0F602004FF4A4710FF0DEFBFFE7029835
:10E38000406A28B1FFE70298406A102801D1FFE7F0
:10E3900008E045F2FE40C0F6020040F249110FF0DD
:10E3A000CBFBFFE70298406A002863D1FFE70298A1
:10E3B000006928B1FFE702980069022801D1FFE750
:10E3C00008E045F2FE40C0F602004FF4A6710FF0DF
:10E3D000B3FBFFE70298406928B1FFE70298406964
:10E3E000012801D1FFE708E045F2FE40C0F6020037
:10E3F00040F24D110FF0A0FBFFE702984068B0F526
:10E40000827F32D1FFE70298C06918B3FFE7029814
:10E41000C06908281ED0FFE70298C069102819D0EB
:10E42000FFE70298C069182814D0FFE70298C06976
:10E4300020280FD0FFE70298C06928280AD0FFE7FC
:10E440000298C069302805D0FFE70298C0693828D3
:10E4500001D1FFE708E045F2FE40C0F6020040F2BD
:10E4600051110FF069FBFFE703E002990020C8613A
:10E47000FFE736E00298C06918B3FFE70298C06969
:10E4800008281ED0FFE70298C069102819D0FFE7BE
:10E490000298C069182814D0FFE70298C0692028A4
:10E4A0000FD0FFE70298C06928280AD0FFE702983A
:10E4B000C069302805D0FFE70298C069382801D12B
:10E4C000FFE708E045F2FE40C0F6020040F25B11B3
:10E4D0000FF032FBFFE702990020086102994861C2
:10E4E000FFE7029900208862029890F8510040B935
:10E4F000FFE70299002081F85000029800F052F8DE
:10E50000FFE70299022081F851000298016808682B
:10E5100020F040000860029A019211685068D2F819
:10E5200008C0D36800F482700CF4044C604403F417
:10E5300000631844136903F002031844536903F09D
:10E5400001031844936903F400731844D36903F07A
:10E5500038031844136A03F080031843926A02F4E4
:10E56000005210430860029A508B00F004001168BA
:10E57000526A02F010021044486002980168C869AB
:10E5800020F40060C861029900204865029A0121C8
:10E5900082F851108DF80F00FFE79DF80F0004B0CE
:10E5A00080BD000080B592B01190002010900F90B7
:10E5B0000E900D900C901198006843F20001C4F287
:10E5C0000101884240F0B680FFE7FFE700200B9092
:10E5D00043F64400C4F20200016841F48051016036
:10E5E000006800F480500B900B98FFE7FFE70020D5
:10E5F0000A9043F63000C4F20200016841F00201C3
:10E600000160006800F002000A900A98FFE7FFE747
:10E610000020099043F63000C4F20200016841F086
:10E6200001010160006800F0010009900998FFE70E
:10E6300018200C90022001900D90012002900E9065
:10E64000032003900F9005200490109040F20040AA
:10E65000C4F202000CA90591FCF70CFDDDF804C022
:10E66000029B039A049805994FF0800ECDF830E094
:10E67000CDF834C00E930F9210900020C4F2020027
:10E68000FCF7F8FC41F6E020C2F20000069046F2EA
:10E690004041C4F2020101604FF0C06141600021BD
:10E6A0008160C1604FF48062026141618161C1613A
:10E6B0004FF4403202624162FBF7F2FF18B1FFE70C
:10E6C000F8F74AFDFFE7FFE7119841F6E021C2F2B3
:10E6D0000001C16411988863FFE741F64030C2F23F
:10E6E0000000009046F25841C4F2020101604FF070
:10E6F000C0614160402181600021C1604FF48062AF
:10E70000026141618161C1614FF400320262416284
:10E71000FBF7C6FF18B1FFE7F8F71EFDFFE7FFE7BD
:10E72000119841F64031C2F200018164119888636A
:10E73000FFE73EE01198006843F60001C4F20001D3
:10E74000884235D1FFE7FFE70020089043F64000FC
:10E75000C4F20200016841F480410160006800F4E5
:10E76000804008900898FFE7FFE70020079043F6F5
:10E770003000C4F20200016841F00201016000684B
:10E7800000F0020007900798FFE74FF460400C90FC
:10E7900002200D9001200E9003200F900520109074
:10E7A00040F20040C4F202000CA9FCF763FCFFE752
:10E7B000FFE712B080BD000080B588B006900591DB
:10E7C000ADF81220039300208DF8070006984068EA
:10E7D000B0F5827F16D1FFE70698806890B9FFE711
:10E7E0000699042081F851000698059ABDF8123068
:10E7F0000399EC46CCF80010114600F089FB8DF827
:10E800001F00EDE0FFE7069890F85000012804D1C2
:10E81000FFE702208DF81F00E2E00699012081F851
:10E820005000FFE7FFE7FDF71BF80290069890F80D
:10E830005100012804D0FFE702208DF80700C0E056
:10E84000059820B1FFE7BDF8120020B9FFE70120CD
:10E850008DF80700B5E00699042081F8510006996B
:10E86000002048650599069A9163BDF81210069A32
:10E870009187BDF81210069AD18706990863069908
:10E8800088860699C8860699086406994864069899
:10E890008068B0F5004F0DD1FFE706980168086861
:10E8A00020F04000086006980168086820F4804065
:10E8B0000860FFE706980068006800F04000402804
:10E8C00007D0FFE706980168086840F0400008603C
:10E8D000FFE70698C06880BBFFE7FFE70698C08F98
:10E8E00050B3FFE7069800688068C00778B1FFE77B
:10E8F00006980068007B0699896B08700699886BFA
:10E90000013088630699C88F0138C88713E0FCF787
:10E91000A7FF0299401A0399884204D3FFE703989E
:10E92000013018B9FFE7039820B9FFE703208DF8FD
:10E93000070046E0FFE7D1E72FE0FFE70698C08F2A
:10E9400050B3FFE7069800688068C00778B1FFE71A
:10E9500006980068C0680699896B08800699886BDC
:10E96000023088630699C88F0138C88713E0FCF726
:10E9700077FF0299401A0399884204D3FFE703986E
:10E98000013018B9FFE7039820B9FFE703208DF89D
:10E99000070016E0FFE7D1E7FFE706980399029A20
:10E9A00007F0BAFF20B1FFE7069920204865FFE78E
:10E9B0000698406D20B1FFE701208DF80700FFE7C2
:10E9C000FFE70699012081F85100FFE70699002032
:10E9D00081F85000FFE79DF807008DF81F00FFE762
:10E9E0009DF81F0008B080BD80B584B002900191F1
:10E9F000ADF8022000208DF801000298C06C08B12B
:10EA0000FFE708E045F2FE40C0F6020040F2CA61AE
:10EA10000FF092F8FFE70298806810BBFFE70298BA
:10EA20004068B0F5827F1CD1FFE70299042081F88D
:10EA300051000298806C08B1FFE708E045F2FE4003
:10EA4000C0F6020040F2D1610FF076F8FFE70298BD
:10EA5000019ABDF80230114600F01CFC8DF80F0041
:10EA6000A8E0FFE7029890F85000012804D1FFE7E2
:10EA700002208DF80F009DE00299012081F85000DE
:10EA8000FFE7FFE7029890F85100012804D0FFE764
:10EA900002208DF8010082E0019820B1FFE7BDF867
:10EAA000020020B9FFE701208DF8010077E002990C
:10EAB000042081F851000299002048650199029ACA
:10EAC0009163BDF80210029A9187BDF80210029A74
:10EAD000D18702990864029948640299888602994C
:10EAE000C88602988068B0F5004F0DD1FFE7029804
:10EAF0000168086820F04000086002980168086812
:10EB000020F480400860FFE70298C16C46F2BD70B7
:10EB1000C0F6010008640298C16C46F2ED70C0F6C0
:10EB20000100C8630298C16C46F28970C0F601000A
:10EB3000C8640298C16C00200865029B19689A6B32
:10EB4000D86C0C31DB8FFCF747F860B1FFE7029916
:10EB5000486D40F01000486501208DF801000299D1
:10EB600081F851001BE002980068006800F0400046
:10EB7000402807D0FFE702980168086840F040008D
:10EB80000860FFE702980168486840F0200048608C
:10EB900002980168486840F001004860FFE7FFE71D
:10EBA0000299002081F85000FFE79DF801008DF8E0
:10EBB0000F00FFE79DF80F0004B080BD80B582B064
:10EBC0000190019807F06CFF8DF803009DF8030099
:10EBD00003281BD0FFE7019807F062FF014640F2CF
:10EBE000A050C2F2000000EB4110406868B1FFE79E
:10EBF000019807F055FF014640F2A050C2F2000014
:10EC000000EB411040688047FFE7FFE702B080BD9E
:10EC100080B582B00190019807F042FF8DF80300A3
:10EC20009DF8030003281BD0FFE7019807F038FF89
:10EC3000014640F2A050C2F2000000EB4110006912
:10EC400068B1FFE7019807F02BFF014640F2A050A2
:10EC5000C2F2000000EB411000698047FFE7FFE7C8
:10EC600002B080BD80B588B006900591ADF8122045
:10EC7000039300208DF807000698806830B1FFE705
:10EC800006988068B0F5004F01D1FFE708E045F233
:10EC9000FE40C0F6020040F20A310EF04DFFFFE7E1
:10ECA000FFE7069890F85000012804D1FFE7022002
:10ECB0008DF81F0028E10699012081F85000FFE738
:10ECC000FFE7FCF7CDFD0290BDF81200ADF804009F
:10ECD000069890F85100012804D0FFE702208DF833
:10ECE000070002E1059820B1FFE7BDF8120020B946
:10ECF000FFE701208DF80700F7E00699032081F86F
:10ED000051000699002048650599069A1163BDF8DF
:10ED10001210069A9186BDF81210069AD1860699AD
:10ED20008863069988870699C88706994864069972
:10ED3000086406988068B0F5004F0DD1FFE706988B
:10ED40000168086820F040000860069801680868BB
:10ED500040F480400860FFE706980068006800F013
:10ED60004000402807D0FFE706980168086840F097
:10ED700040000860FFE70698C068B0F5006F47D113
:10ED8000FFE70698406828B1FFE7BDF804000128B6
:10ED90000ED1FFE706980168006B0088C8600699ED
:10EDA000086B023008630699C88E0138C886FFE7F1
:10EDB000FFE70698C08E50B3FFE7069800688068AA
:10EDC000800700280ED5FFE706980168006B0088D1
:10EDD000C8600699086B023008630699C88E01382E
:10EDE000C88613E0FCF73CFD0299401A039988425B
:10EDF00004D3FFE70398013018B9FFE7039820B95F
:10EE0000FFE703208DF807006FE0FFE7D1E746E05A
:10EE10000698406828B1FFE7BDF8040001280ED12C
:10EE2000FFE706980168006B007808730699086B85
:10EE3000013008630699C88E0138C886FFE7FFE7EE
:10EE40000698C08E50B3FFE7069800688068800778
:10EE500000280ED5FFE706980168006B007808735C
:10EE60000699086B013008630699C88E0138C88678
:10EE700013E0FCF7F5FC0299401A0399884204D389
:10EE8000FFE70398013018B9FFE7039820B9FFE7BF
:10EE900003208DF8070028E0FFE7D1E7FFE7069899
:10EEA0000399029A07F0AAFD20B1FFE706992020F6
:10EEB0004865FFE70698806870B9FFE7FFE7002024
:10EEC000009006980068C068009006980068806806
:10EED00000900098FFE7FFE70698406D20B1FFE73C
:10EEE00001208DF80700FFE7FFE70699012081F870
:10EEF0005100FFE70699002081F85000FFE79DF8D8
:10EF000007008DF81F00FFE79DF81F0008B080BDC7
:10EF100080B58EB0DDF840C00C900B910A92ADF830
:10EF200026300120059000208DF813000C98806891
:10EF300008B9FFE708E045F2FE40C0F6020040F2E3
:10EF40007E410EF0F9FDFFE7FFE70C9890F85000C6
:10EF5000012804D1FFE702208DF8370095E10C99D4
:10EF6000012081F85000FFE7FFE7FCF779FC0690ED
:10EF70000C9890F851008DF81F000C98406808908C
:10EF8000BDF82600ADF824009DF81F00012812D01E
:10EF9000FFE70898B0F5827F09D1FFE70C988068F9
:10EFA00028B9FFE79DF81F00042804D0FFE70220DE
:10EFB0008DF813005AE10B9838B1FFE70A9820B199
:10EFC000FFE7BDF8260020B9FFE701208DF8130008
:10EFD0004CE10C9890F85100042805D0FFE70C99FB
:10EFE000052081F85100FFE70C99002048650A9937
:10EFF0000C9A9163BDF826100C9AD187BDF82610A3
:10F000000C9A91870B990C9A1163BDF826100C9AF3
:10F01000D186BDF826100C9A91860C9908640C993B
:10F0200048640C980068006800F04000402807D051
:10F03000FFE70C980168086840F040000860FFE7AF
:10F040000C98C068B0F5006F76D1FFE70C98406867
:10F0500028B1FFE7BDF8240001280ED1FFE70C9886
:10F060000168006B0088C8600C99086B0230086367
:10F070000C99C88E0138C886FFE7FFE70C98C18E4F
:10F080000120029039B9FFE70C98C08F002818BF03
:10F0900001200290FFE70298C00700284BD0FFE74D
:10F0A0000C98006880688007002818D5FFE70C9846
:10F0B000C08EA0B1FFE70598012810D1FFE70C989A
:10F0C0000168006B0088C8600C99086B0230086307
:10F0D0000C99C88E0138C88600200590FFE70C986F
:10F0E00000688068C007A8B1FFE70C98C08F88B19E
:10F0F000FFE70C980068C0680C99896B08800C9930
:10F10000886B023088630C99C88F0138C88701204A
:10F110000590FFE7FCF7A4FB0699401A1099884276
:10F1200008D3FFE71098013020B1FFE703208DF8E6
:10F1300013009BE0A2E778E00C98406828B1FFE755
:10F14000BDF8240001280ED1FFE70C980168006B80
:10F15000007808730C99086B013008630C99C88E0D
:10F160000138C886FFE7FFE70C98C18E01200190A7
:10F1700039B9FFE70C98C08F002818BF0120019013
:10F18000FFE70198C00700284ED0FFE70C98006801
:10F1900080688007002818D5FFE70C98C08EA0B1C2
:10F1A000FFE70598012810D1FFE70C980168006B74
:10F1B000007808730C99086B013008630C99C88EAD
:10F1C0000138C88600200590FFE70C980068806829
:10F1D000C007A8B1FFE70C98C08F88B1FFE70C9873
:10F1E0000068C0680C99896B08700C99886B0130B5
:10F1F00088630C99C88F0138C88701200590FFE704
:10F20000FCF72EFB0699401A1099884204D3FFE7B9
:10F210001098013018B9FFE7109820B9FFE70320D4
:10F220008DF8130022E09FE7FFE70C981099069AEB
:10F2300007F0E4FB38B1FFE701208DF813000C99CB
:10F240002020486512E00C98806870B9FFE7FFE75E
:10F25000002003900C980068C06803900C98006828
:10F26000806803900398FFE7FFE7FFE70C99012010
:10F2700081F85100FFE70C99002081F85000FFE76A
:10F280009DF813008DF83700FFE79DF837000EB0AA
:10F2900080BD000080B588B0069005910492ADF85D
:10F2A0000E3000208DF806000698C06C08B1FFE70C
:10F2B00008E045F2FE40C0F602004FF4E8610EF0AF
:10F2C0003BFCFFE70698806C08B1FFE708E045F2D9
:10F2D000FE40C0F6020040F241710EF02DFCFFE747
:10F2E0000698806808B9FFE708E045F2FE40C0F6DE
:10F2F000020040F244710EF01FFCFFE7FFE70698A2
:10F3000090F85000012804D1FFE702208DF81F007B
:10F31000EFE00699012081F85000FFE7FFE706982B
:10F3200090F851008DF807000698406802909DF80B
:10F330000700012812D0FFE70298B0F5827F09D1BB
:10F34000FFE70698806828B9FFE79DF807000428C2
:10F3500004D0FFE702208DF80600BFE0059838B121
:10F36000FFE7049820B1FFE7BDF80E0020B9FFE7E2
:10F3700001208DF80600B1E0069890F851000428AD
:10F3800005D0FFE70699052081F85100FFE70699AF
:10F39000002048650599069A1163BDF80E10069A7B
:10F3A0009186BDF80E10069AD1860499069A91634B
:10F3B000BDF80E10069A9187BDF80E10069AD187F7
:10F3C0000699086406994864069890F85100042844
:10F3D0000FD1FFE70698C16C46F2BD70C0F6010080
:10F3E00008640698C16C46F2ED70C0F60100C8636F
:10F3F0000EE00698C16C46F2D570C0F601000864B4
:10F400000698C16C46F69100C0F60100C863FFE79C
:10F410000698C16C46F28970C0F60100C86406986F
:10F42000C16C00200865069B19689A6BD86C0C317A
:10F43000DB8FFBF7D1FB60B1FFE70699486D40F029
:10F440001000486501208DF80600069981F85100EA
:10F4500044E006980168486840F00100486006985A
:10F46000816C002008640699896CC8630699896CD0
:10F47000C8640699896C0865069B1A68196B986CB4
:10F480000C32DB8EFBF7A8FB60B1FFE70699486DF5
:10F4900040F01000486501208DF80600069981F8BB
:10F4A00051001BE006980068006800F0400040280A
:10F4B00007D0FFE706980168086840F04000086040
:10F4C000FFE706980168486840F020004860069809
:10F4D0000168486840F002004860FFE7FFE70699CE
:10F4E000002081F85000FFE79DF806008DF81F000E
:10F4F000FFE79DF81F0008B080BD000080B582B016
:10F500000190019807F0CCFA8DF803009DF80300F4
:10F5100003281BD0FFE7019807F0C2FA014640F22A
:10F52000A050C2F2000000EB4110806868B1FFE714
:10F53000019807F0B5FA014640F2A050C2F200006F
:10F5400000EB411080688047FFE7FFE702B080BD15
:10F5500080B582B00190019807F0A2FA8DF80300FF
:10F560009DF8030003281BD0FFE7019807F098FAE5
:10F57000014640F2A050C2F2000000EB4110406989
:10F5800068B1FFE7019807F08BFA014640F2A050FE
:10F59000C2F2000000EB411040698047FFE7FFE73F
:10F5A00002B080BD80B582B00190019808F02AF8C1
:10F5B00002B080BD81B0009001B0704781B0009072
:10F5C00001B0704780B584B0029001910020009096
:10F5D000029800680021C4F20101884209D0FFE7C7
:10F5E0000298006840F20041C4F20101884201D152
:10F5F000FFE708E045F26E50C0F6020040F2B47139
:10F600000EF09AFAFFE701980068B0F5006F04D099
:10F61000FFE70198006808B9FFE708E045F26E507F
:10F62000C0F6020040F2B5710EF086FAFFE70198CD
:10F630004068B0F5806F04D0FFE70198406808B9D2
:10F64000FFE708E045F26E50C0F6020040F2B671E6
:10F650000EF072FAFFE70198806890B1FFE7019819
:10F660008068B0F5807F0CD0FFE701988068B0F526
:10F67000007F06D0FFE701988068B0F5407F01D198
:10F68000FFE708E045F26E50C0F6020040F2B771A5
:10F690000EF052FAFFE70198C068FF2801D8FFE793
:10F6A00008E045F26E50C0F602004FF4F7610EF02C
:10F6B00043FAFFE701980069B0F5805F04D0FFE7E7
:10F6C0000198006908B9FFE708E045F26E50C0F6FE
:10F6D000020040F2B9710EF02FFAFFE7019840697D
:10F6E00030B1FFE701984069B0F5005F01D1FFE755
:10F6F00008E045F26E50C0F6020040F2BA710EF01A
:10F700001BFAFFE70198C069B0F5804F04D0FFE70E
:10F710000198C06908B9FFE708E045F26E50C0F6ED
:10F72000020040F2BB710EF007FAFFE7FFE7029814
:10F7300090F83C00012804D1FFE702208DF80F006B
:10F7400044E00299012081F83C00FFE7FFE70098C0
:10F7500020F0FF000199C96808430090009820F448
:10F7600040700199896808430090009820F48060F7
:10F770000199496808430090009820F400600199BD
:10F78000096808430090009820F4805001990969A5
:10F7900008430090009820F40050019949690843FB
:10F7A0000090009820F480400199C96908430090B6
:10F7B0000098029909684864FFE70299002081F8DF
:10F7C0003C00FFE700208DF80F00FFE79DF80F00D9
:10F7D00004B080BD80B586B00490039104980068A1
:10F7E0000021C4F2010188423CD0FFE70498006880
:10F7F000B0F1804F36D0FFE70498006840F2004136
:10F80000C4F2000188422DD0FFE70498006840F65A
:10F810000001C4F20001884224D0FFE70498006888
:10F8200040F60041C4F2000188421BD0FFE7049873
:10F83000006841F20001C4F20001884212D0FFE7E3
:10F840000498006841F20041C4F20001884209D0E6
:10F85000FFE70498006840F20041C4F201018842C9
:10F8600001D1FFE708E045F26E50C0F6020040F219
:10F8700077710EF061F9FFE70398006818B3FFE7AE
:10F880000398006810281ED0FFE70398006820281E
:10F8900019D0FFE703980068302814D0FFE70398D9
:10F8A000006840280FD0FFE70398006850280AD06E
:10F8B000FFE703980068602805D0FFE70398006819
:10F8C000702801D1FFE708E045F26E50C0F6020053
:10F8D0004FF4EF610EF030F9FFE70398406880289D
:10F8E00004D0FFE70398406808B9FFE708E045F255
:10F8F0006E50C0F6020040F279710EF01DF9FFE77C
:10F90000FFE7049890F83C00012804D1FFE70220AB
:10F910008DF817007EE00499012081F83C00FFE794
:10F92000FFE70499022081F83D00049800684068D0
:10F9300002900498006880680190029820F070009E
:10F940000290039801680298084302900298049973
:10F9500009684860049800680021C4F201018842E7
:10F960003CD0FFE704980068B0F1804F36D0FFE745
:10F970000498006840F20041C4F2000188422DD092
:10F98000FFE70498006840F60001C4F200018842D5
:10F9900024D0FFE70498006840F60041C4F200015B
:10F9A00088421BD0FFE70498006840F20041C4F28F
:10F9B0000101884212D0FFE70498006844F2000178
:10F9C000C4F20101884209D0FFE70498006841F6BB
:10F9D0000001C4F2000188420ED1FFE7019820F037
:10F9E00080000190039841680198084301900198B4
:10F9F000049909688860FFE70499012081F83D00B7
:10FA0000FFE70499002081F83C00FFE700208DF813
:10FA10001700FFE79DF8170006B080BD80B582B0E3
:10FA20000090009820B9FFE701208DF8070012E14F
:10FA3000009800680021C4F20101884272D0FFE7FB
:10FA400000980068B0F1804F6CD0FFE70098006824
:10FA500040F20041C4F20001884263D0FFE7009801
:10FA6000006840F60001C4F2000188425AD0FFE766
:10FA70000098006840F60041C4F20001884251D06D
:10FA8000FFE70098006841F20001C4F200018842DB
:10FA900048D0FFE70098006841F20041C4F200013D
:10FAA00088423FD0FFE70098006840F20041C4F26E
:10FAB0000101884236D0FFE70098006844F2000157
:10FAC000C4F2010188422DD0FFE70098006844F29B
:10FAD0000041C4F20101884224D0FFE70098006889
:10FAE00044F60001C4F2010188421BD0FFE70098F0
:10FAF000006841F60001C4F20001884212D0FFE71D
:10FB00000098006841F60041C4F20001884209D023
:10FB1000FFE70098006842F20001C4F20001884249
:10FB200001D1FFE708E045F23650C0F6020040F28E
:10FB300013110EF001F8FFE700988068A0B1FFE70D
:10FB40000098806810280FD0FFE700988068202870
:10FB50000AD0FFE700988068402805D0FFE70098AA
:10FB60008068602801D1FFE708E045F23650C0F612
:10FB700002004FF48A710DF0DFFFFFE70098006983
:10FB800060B1FFE700980069B0F5807F06D0FFE71D
:10FB900000980069B0F5007F01D1FFE708E045F269
:10FBA0003650C0F6020040F215110DF0C5FFFFE718
:10FBB0000098806928B1FFE700988069802801D10A
:10FBC000FFE708E045F23650C0F602004FF48B71B3
:10FBD0000DF0B2FFFFE7009890F83D0040B9FFE755
:10FBE0000099002081F83C00009800F039F8FFE708
:10FBF0000099022081F83D00009951F8040B07F0AC
:10FC0000B5FD0099012081F84600FFE70099012029
:10FC100081F83E00009981F83F00009981F840008A
:10FC2000009981F84100FFE7FFE70099012081F882
:10FC30004200009981F84300009981F8440000993E
:10FC400081F84500FFE70099012081F83D00002080
:10FC50008DF80700FFE79DF8070002B080BD0000A7
:10FC600080B58AB00990099800680021C4F20101AA
:10FC700088421BD1FFE7FFE70020089043F64400CD
:10FC8000C4F20200016841F001010160006800F067
:10FC9000010008900898FFE7182001900521002234
:10FCA000FCF7FAF90198FCF7DFF9B0E00998006871
:10FCB00040F20041C4F20001884212D1FFE7FFE7A1
:10FCC0000020079043F64000C4F20200016841F0B2
:10FCD00002010160006800F0020007900798FFE74A
:10FCE00094E00998006840F60001C4F200018842DF
:10FCF00012D1FFE7FFE70020069043F64000C4F270
:10FD00000200016841F004010160006800F0040095
:10FD100006900698FFE778E00998006840F60041F1
:10FD2000C4F20001884212D1FFE7FFE700200590EE
:10FD300043F64000C4F20200016841F0080101608E
:10FD4000006800F0080005900598FFE75CE009985E
:10FD5000006841F20041C4F2000188421BD1FFE774
:10FD6000FFE70020049043F64000C4F2020001685F
:10FD700041F020010160006800F020000490049828
:10FD8000FFE73720009005210022FCF785F9009855
:10FD9000FCF76AF937E00998006840F20041C4F2C4
:10FDA0000101884212D1FFE7FFE70020039043F6EC
:10FDB0004400C4F20200016841F0020101600068E1
:10FDC00000F0020003900398FFE71BE00998006829
:10FDD00044F20041C4F20101884212D1FFE7FFE77B
:10FDE0000020029043F64400C4F20200016841F48E
:10FDF00000310160006800F4003002900298FFE7D3
:10FE0000FFE7FFE7FFE7FFE7FFE7FFE7FFE70AB0EE
:10FE100080BD000080B584B0029002980068002187
:10FE2000C4F20101884272D0FFE702980068B0F185
:10FE3000804F6CD0FFE70298006840F20041C4F2A6
:10FE40000001884263D0FFE70298006840F6000195
:10FE5000C4F2000188425AD0FFE70298006840F6D9
:10FE60000041C4F20001884251D0FFE702980068C7
:10FE700041F20001C4F20001884248D0FFE7029835
:10FE8000006841F20041C4F2000188423FD0FFE720
:10FE90000298006840F20041C4F20101884236D065
:10FEA000FFE70298006844F20001C4F201018842B1
:10FEB0002DD0FFE70298006844F20041C4F201012E
:10FEC000884224D0FFE70298006844F60001C4F29B
:10FED000010188421BD0FFE70298006841F600014B
:10FEE000C4F20001884212D0FFE70298006841F690
:10FEF0000041C4F20001884209D0FFE7029800687F
:10FF000042F20001C4F20001884201D1FFE708E09B
:10FF100045F23650C0F6020040F2CF110DF00CFE53
:10FF2000FFE7029890F83D00012804D0FFE7012088
:10FF30008DF80F006AE00299022081F83D000298D6
:10FF40000168C86840F00100C8600298006800219C
:10FF5000C4F2010188423CD0FFE702980068B0F18A
:10FF6000804F36D0FFE70298006840F20041C4F2AB
:10FF7000000188422DD0FFE70298006840F600019A
:10FF8000C4F20001884224D0FFE70298006840F6DE
:10FF90000041C4F2000188421BD0FFE702980068CC
:10FFA00040F20041C4F20101884212D0FFE70298FA
:10FFB000006844F20001C4F20101884209D0FFE761
:10FFC0000298006841F60001C4F20001884212D193
:10FFD000FFE702980068806800F007000190019830
:10FFE000062807D0FFE702980168086840F0010082
:10FFF0000860FFE706E002980168086840F0010029
:020000040801F1
:100000000860FFE700208DF80F00FFE79DF80F0064
:1000100004B080BD80B586B004900391FFE70498DA
:1000200090F83C00012805D1FFE702208DF8170069
:1000300000F069BC0499012081F83C00FFE7FFE76C
:100040000499022081F83D0003980068B0F5805FB4
:100050002DD0FFE703980068B0F5005F27D0FFE7D9
:100060000398006818B3FFE70398006810281ED0B3
:10007000FFE703980068202819D0FFE7039800687D
:10008000302814D0FFE70398006840280FD0FFE71E
:100090000398006850280AD0FFE70398006860289A
:1000A00005D0FFE703980068702801D1FFE708E05A
:1000B00045F23650C0F6020041F222410DF03CFDFF
:1000C000FFE70498006880680290029820F07700AB
:1000D0000290029820F47F400290029804990968E7
:1000E0008860039800680190002800F0A883FFE76B
:1000F0000198102800F0A383FFE70198202800F062
:100100009E83FFE70198302800F09983FFE701986C
:10011000402800F00883FFE70198502800F0EB81A9
:10012000FFE70198602800F07282FFE701987028CD
:1001300000F09180FFE70198B0F5805F06D0FFE7FF
:100140000198B0F5005F00F03A81CDE304980068B3
:100150000021C4F20101884272D0FFE704980068D0
:10016000B0F1804F6CD0FFE70498006840F2004186
:10017000C4F20001884263D0FFE70498006840F6AB
:100180000001C4F2000188425AD0FFE704980068D9
:1001900040F60041C4F20001884251D0FFE70498C4
:1001A000006841F20001C4F20001884248D0FFE734
:1001B0000498006841F20041C4F2000188423FD037
:1001C000FFE70498006840F20041C4F20101884250
:1001D00036D0FFE70498006844F20001C4F2010140
:1001E00088422DD0FFE70498006844F20041C4F231
:1001F0000101884224D0FFE70498006844F600011A
:10020000C4F2010188421BD0FFE70498006841F660
:100210000001C4F20001884212D0FFE70498006890
:1002200041F60041C4F20001884209D0FFE704987A
:10023000006842F20001C4F20001884201D1FFE7E8
:1002400008E045F23650C0F6020041F22E410DF0B2
:1002500073FCFFE749E3049800680021C4F2010140
:1002600088423CD0FFE704980068B0F1804F36D058
:10027000FFE70498006840F20041C4F200018842A0
:100280002DD0FFE70498006840F60001C4F2000199
:10029000884224D0FFE70498006840F60041C4F289
:1002A000000188421BD0FFE70498006840F200413B
:1002B000C4F20101884212D0FFE70498006844F2BA
:1002C0000001C4F20101884209D0FFE704980068E8
:1002D00041F60001C4F20001884201D1FFE708E0C5
:1002E00045F23650C0F6020041F235410DF024FCD3
:1002F000FFE70398806890B1FFE703988068B0F546
:10030000805F0CD0FFE703988068B0F5005F06D0EF
:10031000FFE703988068B0F5405F01D1FFE708E090
:1003200045F23650C0F6020041F238410DF004FCAF
:10033000FFE703984068B0F5004F12D0FFE703983D
:10034000406870B1FFE70398406850B1FFE7039839
:100350004068022805D0FFE7039840680A2801D1C9
:10036000FFE708E045F23650C0F6020041F239419D
:100370000DF0E2FBFFE70398C0680F2801D8FFE704
:1003800008E045F23650C0F6020041F23A410DF065
:10039000D3FBFFE704980068039B5A689968DB6801
:1003A00007F052FB0498006880680290029840F0C1
:1003B00077000290029804990968886095E2049891
:1003C00000680021C4F2010188422AD0FFE70498A6
:1003D0000068B0F1804F24D0FFE70498006840F235
:1003E0000041C4F2000188421BD0FFE70498006876
:1003F00040F60001C4F20001884212D0FFE70498E1
:10040000006840F60041C4F20001884209D0FFE7CD
:100410000498006840F20041C4F20101884201D111
:10042000FFE708E045F23650C0F6020041F24D41C8
:100430000DF082FBFFE70398806890B1FFE7039817
:100440008068B0F5805F0CD0FFE703988068B0F556
:10045000005F06D0FFE703988068B0F5405F01D1E8
:10046000FFE708E045F23650C0F6020041F2504185
:100470000DF062FBFFE703984068B0F5004F12D023
:10048000FFE70398406870B1FFE70398406850B1F8
:10049000FFE703984068022805D0FFE7039840680B
:1004A0000A2801D1FFE708E045F23650C0F6020005
:1004B00041F251410DF040FBFFE70398C0680F285F
:1004C00001D8FFE708E045F23650C0F6020041F2DD
:1004D00052410DF031FBFFE704980068039B5A6816
:1004E0009968DB6807F0B0FA04980168886840F4FE
:1004F00080408860F9E1049800680021C4F201019D
:1005000088423CD0FFE704980068B0F1804F36D0B5
:10051000FFE70498006840F20041C4F200018842FD
:100520002DD0FFE70498006840F60001C4F20001F6
:10053000884224D0FFE70498006840F60041C4F2E6
:10054000000188421BD0FFE70498006840F2004198
:10055000C4F20101884212D0FFE70498006844F217
:100560000001C4F20101884209D0FFE70498006845
:1005700041F60001C4F20001884201D1FFE708E022
:1005800045F23650C0F6020041F261410DF0D4FA56
:10059000FFE703984068B0F5004F12D0FFE70398DB
:1005A000406870B1FFE70398406850B1FFE70398D7
:1005B0004068022805D0FFE7039840680A2801D167
:1005C000FFE708E045F23650C0F6020041F2644110
:1005D0000DF0B2FAFFE70398C0680F2801D8FFE7D3
:1005E00008E045F23650C0F6020041F265410DF0D8
:1005F000A3FAFFE704980068039A5168D26807F0ED
:10060000D9FC04980068502107F038FA6DE104988D
:1006100000680021C4F2010188423CD0FFE7049841
:100620000068B0F1804F36D0FFE70498006840F2D0
:100630000041C4F2000188422DD0FFE70498006811
:1006400040F60001C4F20001884224D0FFE704987C
:10065000006840F60041C4F2000188421BD0FFE769
:100660000498006840F20041C4F20101884212D0AF
:10067000FFE70498006844F20001C4F201018842D7
:1006800009D0FFE70498006841F60001C4F20001B8
:10069000884201D1FFE708E045F23650C0F602007B
:1006A00041F271410DF048FAFFE703984068B0F558
:1006B000004F12D0FFE70398406870B1FFE703983E
:1006C000406850B1FFE703984068022805D0FFE773
:1006D000039840680A2801D1FFE708E045F2365048
:1006E000C0F6020041F274410DF026FAFFE70398CC
:1006F000C0680F2801D8FFE708E045F23650C0F681
:10070000020041F275410DF017FAFFE70498006806
:10071000039A5168D26807F075FC0498006860215C
:1007200007F0ACF9E1E0049800680021C4F201018F
:1007300088423CD0FFE704980068B0F1804F36D083
:10074000FFE70498006840F20041C4F200018842CB
:100750002DD0FFE70498006840F60001C4F20001C4
:10076000884224D0FFE70498006840F60041C4F2B4
:10077000000188421BD0FFE70498006840F2004166
:10078000C4F20101884212D0FFE70498006844F2E5
:100790000001C4F20101884209D0FFE70498006813
:1007A00041F60001C4F20001884201D1FFE708E0F0
:1007B00045F23650C0F6020041F281410DF0BCF91D
:1007C000FFE703984068B0F5004F12D0FFE70398A9
:1007D000406870B1FFE70398406850B1FFE70398A5
:1007E0004068022805D0FFE7039840680A2801D135
:1007F000FFE708E045F23650C0F6020041F28441BE
:100800000DF09AF9FFE70398C0680F2801D8FFE7B9
:1008100008E045F23650C0F6020041F285410DF085
:100820008BF9FFE704980068039A5168D26807F0D3
:10083000C1FB04980068402107F020F955E00498B6
:1008400000680021C4F2010188423CD0FFE704980F
:100850000068B0F1804F36D0FFE70498006840F29E
:100860000041C4F2000188422DD0FFE704980068DF
:1008700040F60001C4F20001884224D0FFE704984A
:10088000006840F60041C4F2000188421BD0FFE737
:100890000498006840F20041C4F20101884212D07D
:1008A000FFE70498006844F20001C4F201018842A5
:1008B00009D0FFE70498006841F60001C4F2000186
:1008C000884201D1FFE708E045F23650C0F6020049
:1008D00041F294410DF030F9FFE704980068039964
:1008E000096807F0CBF800E0FFE70499012081F8E0
:1008F0003D00FFE70499002081F83C00FFE700205D
:100900008DF81700FFE79DF8170006B080BD0000C6
:1009100081B0009001B0704780B582B0019001981D
:100920000068006900F002010020B0EB510F28D0F0
:10093000FFE701980068C06800F002010020B0EBFA
:10094000510F1DD0FFE7019801686FF002000861A8
:10095000019901200877019800688069800720B11B
:10096000FFE70198FFF7D4FF06E0019800F04CFA8A
:10097000019800F0A3FDFFE7019900200877FFE749
:10098000FFE701980068006900F004010020B0EB67
:10099000910F29D0FFE701980068C06800F00401BA
:1009A0000020B0EB910F1ED0FFE7019801686FF0B7
:1009B00004000861019902200877019800688069A5
:1009C00010F4407F04D0FFE70198FFF7A1FF06E095
:1009D000019800F019FA019800F070FDFFE7019905
:1009E00000200877FFE7FFE701980068006900F042
:1009F00008010020B0EBD10F28D0FFE70198006874
:100A0000C06800F008010020B0EBD10F1DD0FFE757
:100A1000019801686FF008000861019904200877C7
:100A200001980068C069800720B1FFE70198FFF7CF
:100A30006FFF06E0019800F0E7F9019800F03EFD35
:100A4000FFE7019900200877FFE7FFE701980068BA
:100A5000006900F010010020B0EB111F29D0FFE762
:100A600001980068C06800F010010020B0EB111F71
:100A70001ED0FFE7019801686FF01000086101992E
:100A80000820087701980068C06910F4407F04D0FE
:100A9000FFE70198FFF73CFF06E0019800F0B4F98A
:100AA000019800F00BFDFFE7019900200877FFE7B0
:100AB000FFE7019800680069C00780B1FFE701986F
:100AC0000068C068C00748B1FFE7019801686FF08F
:100AD00001000861019801F057F8FFE7FFE701986E
:100AE00000680069C1B20020B0EBD11F13D0FFE74E
:100AF00001980068C068C1B20020B0EBD11F09D0D6
:100B0000FFE7019801686FF0800008610198FEF727
:100B100051FDFFE7FFE701980068006900F0400120
:100B20000020B0EB911F14D0FFE701980068C06867
:100B300000F040010020B0EB911F09D0FFE70198C1
:100B400001686FF040000861019801F033F8FFE799
:100B5000FFE701980068006900F020010020B0EB79
:100B6000511F14D0FFE701980068C06800F0200111
:100B70000020B0EB511F09D0FFE7019801686FF02A
:100B8000200008610198FEF719FDFFE7FFE702B0BA
:100B900080BD000080B592B01190002010900F90A1
:100BA0000E900D900C90119800680021C4F2010184
:100BB000884222D1FFE7FFE700200B9043F6300088
:100BC000C4F20200016841F010010160006800F009
:100BD00010000B900B98FFE74FF4D4400C900221CB
:100BE0000D9101200E900F91109041F20000C4F27F
:100BF00002000CA9FAF73EFA03E11198006840F2EE
:100C00000041C4F20001884222D1FFE7FFE7002043
:100C10000A9043F63000C4F20200016841F004017A
:100C20000160006800F004000A900A98FFE74FF4A2
:100C300080700C9002200D9001210E910F90109069
:100C400040F60000C4F202000CA9FAF713FAD7E04C
:100C50001198006840F60001C4F20001884223D1D7
:100C6000FFE7FFE70020099043F63000C4F20200DE
:100C7000016841F008010160006800F00800099077
:100C80000998FFE74FF480400C9002200D9001215D
:100C90000E9103210F91109040F60040C4F2020023
:100CA0000CA9FAF7E7F9AAE01198006840F60041AC
:100CB000C4F20001884222D1FFE7FFE7002008903C
:100CC00043F63000C4F20200016841F08001016087
:100CD000006800F0800008900898FFE74FF4E050AB
:100CE0000C9002200D9001210E910F90109041F672
:100CF0000040C4F202000CA9FAF7BCF97EE011989A
:100D0000006840F20041C4F2010188424AD1FFE785
:100D1000FFE70020079043F63000C4F202000168AC
:100D200041F480710160006800F4807007900798BA
:100D3000FFE7FFE70020069043F63000C4F2020010
:100D4000016841F004010160006800F004000690B1
:100D50000698FFE7402000900C90022002900D9032
:100D6000012101910E910F9003200390109042F207
:100D70000000C4F202000CA90491FAF77BF9DDF837
:100D800000C0019B029A03980499CDF830C00D92DF
:100D90000E930F92109040F60000C4F20200FAF792
:100DA00069F92AE01198006844F20041C4F2010197
:100DB000884221D1FFE7FFE70020059043F630008D
:100DC000C4F20200016841F020010160006800F0F7
:100DD000200005900598FFE740200C9002200D9020
:100DE0000E900F900320109041F20040C4F20200D8
:100DF0000CA9FAF73FF9FFE7FFE7FFE7FFE7FFE797
:100E0000FFE712B080BD000081B0009001B07047D4
:100E100080B586B0049003910292029880B1FFE7FA
:100E2000029804280CD0FFE70298082808D0FFE7B2
:100E300002980C2804D0FFE702983C2801D1FFE774
:100E400008E045F23650C0F6020041F217010CF0FE
:100E500073FEFFE703980068602805D0FFE703985A
:100E60000068702801D1FFE708E045F23650C0F66F
:100E7000020041F218010CF05FFEFFE70398806862
:100E800028B1FFE703988068022801D1FFE708E056
:100E900045F23650C0F6020041F219010CF04CFE4A
:100EA000FFE70398006928B1FFE703980069042869
:100EB00001D1FFE708E045F23650C0F6020041F2EA
:100EC0001A010CF039FEFFE7FFE7049890F83C00A8
:100ED000012804D1FFE702208DF81700C3E104992F
:100EE000012081F83C00FFE7FFE7029801900C2801
:100EF00000F2AE810199DFE811F00D00AB01AB010A
:100F0000AB019800AB01AB01AB010001AB01AB0140
:100F1000AB015501049800680021C4F20101884228
:100F200060D0FFE704980068B0F1804F5AD0FFE727
:100F30000498006840F20041C4F20001884251D098
:100F4000FFE70498006840F60001C4F200018842FF
:100F500048D0FFE70498006840F60041C4F2000161
:100F600088423FD0FFE70498006840F20041C4F295
:100F70000101884236D0FFE70498006844F200017E
:100F8000C4F2010188422DD0FFE70498006844F2C2
:100F90000041C4F20101884224D0FFE704980068B0
:100FA00044F60001C4F2010188421BD0FFE7049817
:100FB000006841F60001C4F20001884212D0FFE748
:100FC0000498006841F60041C4F20001884209D04B
:100FD000FFE70498006842F20001C4F20001884271
:100FE00001D1FFE708E045F23650C0F6020041F2B9
:100FF00024010CF0A1FDFFE704980068039906F0B6
:1010000053FD04980168886940F0080088610498DD
:101010000168886920F004008861039802690498D7
:10102000016888691043886113E104980068002111
:10103000C4F2010188423CD0FFE704980068B0F197
:10104000804F36D0FFE70498006840F20041C4F2B8
:10105000000188422DD0FFE70498006840F60001A7
:10106000C4F20001884224D0FFE70498006840F6EB
:101070000041C4F2000188421BD0FFE704980068D9
:1010800040F20041C4F20101884212D0FFE7049807
:10109000006844F20001C4F20101884209D0FFE770
:1010A0000498006841F60001C4F20001884201D1B1
:1010B000FFE708E045F23650C0F6020041F2350184
:1010C0000CF03AFDFFE704980068039906F09EFDD6
:1010D00004980168886940F4006088610498016898
:1010E000886920F480608861039802690498016827
:1010F000886940EA02208861ABE00498006800211A
:10110000C4F2010188422AD0FFE704980068B0F1D8
:10111000804F24D0FFE70498006840F20041C4F2F9
:10112000000188421BD0FFE70498006840F60001E8
:10113000C4F20001884212D0FFE70498006840F62C
:101140000041C4F20001884209D0FFE7049800681A
:1011500040F20041C4F20101884201D1FFE708E0FA
:1011600045F23650C0F6020041F246010CF0E4FCB4
:10117000FFE704980068039906F0FEFD04980168F3
:10118000C86940F00800C86104980168C86920F087
:101190000400C8610398026904980168C869104393
:1011A000C86156E0049800680021C4F20101884239
:1011B0002AD0FFE704980068B0F1804F24D0FFE701
:1011C0000498006840F20041C4F2000188421BD03C
:1011D000FFE70498006840F60001C4F2000188426D
:1011E00012D0FFE70498006840F60041C4F2000105
:1011F000884209D0FFE70498006840F20041C4F239
:101200000101884201D1FFE708E045F23650C0F6FF
:10121000020041F257010CF08FFCFFE704980068D0
:10122000039906F05FFE04980168C86940F4006005
:10123000C86104980168C86920F48060C861039897
:10124000026904980168C86940EA0220C86100E0A8
:10125000FFE7FFE70499002081F83C00FFE700204A
:101260008DF81700FFE79DF8170006B080BD00005D
:1012700080B582B00090009820B9FFE701208DF87A
:10128000070012E1009800680021C4F201018842C1
:1012900072D0FFE700980068B0F1804F6CD0FFE794
:1012A0000098006840F20041C4F20001884263D017
:1012B000FFE70098006840F60001C4F20001884290
:1012C0005AD0FFE70098006840F60041C4F20001E0
:1012D000884251D0FFE70098006841F20001C4F253
:1012E0000001884248D0FFE70098006841F20041C1
:1012F000C4F2000188423FD0FFE70098006840F246
:101300000041C4F20101884236D0FFE7009800682E
:1013100044F20001C4F2010188422DD0FFE7009899
:10132000006844F20041C4F20101884224D0FFE782
:101330000098006844F60001C4F2010188421BD005
:10134000FFE70098006841F60001C4F200018842FE
:1013500012D0FFE70098006841F60041C4F2000196
:10136000884209D0FFE70098006842F20001C4F209
:101370000001884201D1FFE708E045F23650C0F68F
:10138000020040F20E510CF0D7FBFFE70098806896
:10139000A0B1FFE70098806810280FD0FFE7009801
:1013A000806820280AD0FFE700988068402805D090
:1013B000FFE700988068602801D1FFE708E045F268
:1013C0003650C0F6020040F20F510CF0B5FBFFE7BB
:1013D0000098006960B1FFE700980069B0F5807F70
:1013E00006D0FFE700980069B0F5007F01D1FFE764
:1013F00008E045F23650C0F602004FF4A2610CF04E
:101400009BFBFFE70098806928B1FFE7009880699F
:10141000802801D1FFE708E045F23650C0F602000F
:1014200040F211510CF088FBFFE7009890F83D0066
:1014300040B9FFE70099002081F83C00009800F0D7
:1014400039F8FFE70099022081F83D00009951F832
:10145000040B06F08BF90099012081F84600FFE7A4
:101460000099012081F83E00009981F83F00009921
:1014700081F84000009981F84100FFE7FFE70099FB
:10148000012081F84200009981F84300009981F819
:101490004400009981F84500FFE70099012081F898
:1014A0003D0000208DF80700FFE79DF8070002B01F
:1014B00080BD000081B0009001B0704781B0009005
:1014C00001B0704780B58CB00A9009910A98006805
:1014D0000021C4F20101884214D1FFE709980028D5
:1014E00000F0E780FFE70998042800F0E280FFE7BA
:1014F0000998082800F0DD80FFE709980C2800F023
:10150000D880FFE70A980068B0F1804F14D1FFE758
:101510000998002800F0CD80FFE70998042800F022
:10152000C880FFE70998082800F0C380FFE7099802
:101530000C2800F0BE80FFE70A98006840F20041E6
:10154000C4F20001884214D1FFE70998002800F096
:10155000B080FFE70998042800F0AB80FFE7099806
:10156000082800F0A680FFE709980C2800F0A18069
:10157000FFE70A98006840F60001C4F200018842C3
:1015800014D1FFE70998002800F09380FFE709983D
:10159000042800F08E80FFE70998082800F0898071
:1015A000FFE709980C2800F08480FFE70A9800689C
:1015B00040F60041C4F20001884210D1FFE70998CB
:1015C000002876D0FFE70998042872D0FFE7099831
:1015D00008286ED0FFE709980C286AD0FFE70A9820
:1015E000006840F20041C4F20101884210D1FFE7D7
:1015F000099800285DD0FFE70998042859D0FFE733
:101600000998082855D0FFE709980C2851D0FFE722
:101610000A98006844F20001C4F20101884208D12E
:10162000FFE70998002844D0FFE70998042840D034
:10163000FFE70A98006844F20041C4F201018842C1
:1016400003D1FFE70998A0B3FFE70A98006844F6C2
:101650000001C4F20101884203D1FFE7099840B3B9
:10166000FFE70A98006841F60001C4F200018842D1
:1016700007D1FFE70998E0B1FFE70998042818D0DF
:10168000FFE70A98006841F60041C4F20001884271
:1016900003D1FFE7099860B1FFE70A98006842F2BA
:1016A0000001C4F20001884204D1FFE7099808B99B
:1016B000FFE708E045F23650C0F6020040F29451D0
:1016C0000CF03AFAFFE7099828B9FFE70A9890F872
:1016D0003E0007901CE00998042805D1FFE70A980E
:1016E00090F83F00069010E00998082805D1FFE720
:1016F0000A9890F84000059004E00A9890F841009C
:101700000590FFE705980690FFE706980790FFE72A
:101710000798012804D0FFE701208DF82F00AFE0E3
:10172000099828B9FFE70A99022081F83E001EE0D7
:101730000998042806D1FFE70A99022081F83F00A2
:10174000049012E00998082806D1FFE70A990220C0
:1017500081F84000039005E00A99022081F84100D9
:101760000390FFE703980490FFE70498FFE70A98C7
:10177000006809990122019206F0C6F801980A99B9
:1017800009680022C4F20102914202900CD0FFE7E6
:101790000A9800684FF60041CBF6FE710844B0FA93
:1017A00080F040090290FFE70298C00738B1FFE7D8
:1017B0000A980168486C40F400404864FFE70A98C2
:1017C00000680021C4F2010188423CD0FFE70A987A
:1017D0000068B0F1804F36D0FFE70A98006840F209
:1017E0000041C4F2000188422DD0FFE70A9800684A
:1017F00040F60001C4F20001884224D0FFE70A98B5
:10180000006840F60041C4F2000188421BD0FFE7A7
:101810000A98006840F20041C4F20101884212D0E7
:10182000FFE70A98006844F20001C4F2010188420F
:1018300009D0FFE70A98006841F60001C4F20001F0
:10184000884212D1FFE70A980068806800F007001C
:1018500008900898062807D0FFE70A9801680868EA
:1018600040F001000860FFE706E00A980168086898
:1018700040F001000860FFE700208DF82F00FFE72F
:101880009DF82F000CB080BD80B586B00590049106
:10189000059800680021C4F20101884214D1FFE7D5
:1018A0000498002800F0E780FFE70498042800F07F
:1018B000E280FFE70498082800F0DD80FFE7049845
:1018C0000C2800F0D880FFE705980068B0F1804F41
:1018D00014D1FFE70498002800F0CD80FFE70498BA
:1018E000042800F0C880FFE70498082800F0C380AF
:1018F000FFE704980C2800F0BE80FFE70598006819
:1019000040F20041C4F20001884214D1FFE704987C
:10191000002800F0B080FFE70498042800F0AB80B6
:10192000FFE70498082800F0A680FFE704980C2839
:1019300000F0A180FFE70598006840F60001C4F2BE
:101940000001884214D1FFE70498002800F093803A
:10195000FFE70498042800F08E80FFE70498082829
:1019600000F08980FFE704980C2800F08480FFE7EE
:101970000598006840F60041C4F20001884210D189
:10198000FFE70498002876D0FFE70498042872D077
:10199000FFE7049808286ED0FFE704980C286AD067
:1019A000FFE70598006840F20041C4F20101884257
:1019B00010D1FFE7049800285DD0FFE704980428C1
:1019C00059D0FFE70498082855D0FFE704980C2861
:1019D00051D0FFE70598006844F20001C4F201010C
:1019E000884208D1FFE70498002844D0FFE7049814
:1019F000042840D0FFE70598006844F20041C4F293
:101A00000101884203D1FFE70498A0B3FFE70598DE
:101A1000006844F60001C4F20101884203D1FFE7E7
:101A2000049840B3FFE70598006841F60001C4F24E
:101A30000001884207D1FFE70498E0B1FFE704986E
:101A4000042818D0FFE70598006841F60041C4F269
:101A50000001884203D1FFE7049860B1FFE70598D1
:101A6000006842F20001C4F20001884204D1FFE79D
:101A7000049808B9FFE708E045F23650C0F60200C6
:101A80004FF4B9610CF058F8FFE705980068049925
:101A9000002205F039FF0598016801200022C4F2F8
:101AA0000102914203900CD0FFE7059800684FF6C1
:101AB0000041CBF6FE710844B0FA80F04009039073
:101AC000FFE70398C007D8B1FFE7FFE70598006874
:101AD000006A41F21111084210D1FFE70598006831
:101AE000006A40F24441084207D1FFE705980168C7
:101AF000486C20F400404864FFE7FFE7FFE7FFE79A
:101B0000FFE705980068006A41F21111084210D100
:101B1000FFE705980068006A40F24441084207D197
:101B2000FFE705980168086820F001000860FFE7FA
:101B3000FFE7FFE7049828B9FFE70599012081F83E
:101B40003E001EE00498042806D1FFE70599012015
:101B500081F83F00029012E00498082806D1FFE7C0
:101B60000599012081F84000019005E005990120C8
:101B700081F841000190FFE701980290FFE7029889
:101B8000FFE7002006B080BD81B00090009800689B
:101B900041F20041C4F20001884208D1FFE741F65A
:101BA0007C61C2F20001086801300860FFE701B003
:101BB0007047000081B0009001B0704782B0019082
:101BC000ADF8021002B0704780B582B00190019864
:101BD00007F0A0FE8DF803009DF8030004281BD039
:101BE000FFE79DF8030000EBC00140F22060C2F265
:101BF000000000EB8100C06968B1FFE79DF80300B9
